:100000000C94B50E0C94DD0E0C94DD0E0C94DD0EEC
:100010000C94DD0E0C94DD0E0C94DD0E0C94DD0EB4
:100020000C94DD0E0C94DD0E0C94DD0E0C943E67EA
:100030000C94D46A0C946B670C94DD0E0C945718D6
:100040000C9445180C94DD0E0C94EF6D0C94DD0EA1
:100050000C94DD0E0C94DD0E0C94DD0E0C94DD0E74
:100060000C94946A0C94B3180C94D6670C94A368FF
:100070000C94DD0E0C94DD0E0C94DD0E0C94DD0E54
:100080000C94DD0E0C94DD0E0C94DD0E946C986CCB
:10009000A06CAA6CC16CDB6CF06CFF6C146D2B6DEA
:1000A000356D536D596D5E6D646D6A6DC46DCE6D49
:1000B000736D796D7F6D886D8C6D916D996DAB6D84
:1000C000B16DB76DBC6D9C6C9C6DA16DA66D256E00
:1000D000346F436E486E346F5E6E636E346F796E4C
:1000E0007E6E346F946E996E346FAF6EB46E346FF3
:1000F000CA6ECE6EE56EE76EE96EEB6EEF6E537014
:100100006C61736800804000000000000000000087
:1001100000000000000000000000000000000000DF
:1001200000000000000000000000000000000000CF
:1001300000000000000000000000000000000000BF
:1001400000000000000000000000000000000000AF
:10015000000080C0E0E0F0F8F8FCFCFCF8F8F8F0F3
:1001600040000000000080808000000000000000CF
:1001700000000000000000000000000080C0C0E09F
:10018000E0E0F0F0F0E0C00000000000C0F8FFFF89
:100190009F8783838383838383838383838383830F
:1001A00083838383838383830383808383838383A2
:1001B000838383838383838383838383838383830F
:1001C0008383C3E3733F1F0000000080E0F0F8FC6E
:1001D000FEFFFFFFFF7F3F1F1F0F0783C3E1E1E02B
:1001E000E0C0000E1F3F7F7FFFF3E0E080000000D3
:1001F0000000000000000080F0FCFEFFFFFFFF7F1A
:100200003F0F0301010100000080F0FEFFFFC7C1A6
:10021000C1C1C1C1C1C1C1C1C1C1C1C1C1C1C1C1CE
:10022000C1C1C1C1C101C1F0FEFF3F0F070F0D0DDC
:100230000D1D191919193131313171616161E1C136
:10024000C1C18100000080E0F8FCFFFFFFFF2F1715
:100250000F038180C0E0F0F8FCFEFFFFFFFFFFFF0F
:100260007F010000000000000001010307070E1ECF
:100270001C3870E0F0F8FEFFFF7F1F0F0300010045
:10028000000000000000000000000000000000006E
:10029000000000000000000000000000000000005E
:1002A000000000000000000000000000000000004E
:1002B000000000000000000000000000000000003E
:1002C00000000000007EFFFFFFFFFFFFFBF8FCFCCB
:1002D000FEFF7F3F1F0F07C3FFFFFFFFFFFF7F07EB
:1002E0000000000000000000000000000000C0E06E
:1002F000F8FEFFFF7F1F0F1F3D7CF8F8F0E0800045
:1003000000000000000000000000000000000000ED
:1003100000000000000000000000000000000000DD
:1003200000000000000000000000000000000000CD
:1003300000000000000000000000000000000000BD
:100340000000000000000001010101010307070790
:100350000301000000E0FCFFFFFFFFFF1F030000A0
:10036000000000000000000000C0F078DE27130944
:100370000E0703000000000000000001030F7FFFD4
:10038000FC7878F800000000000000000000008009
:10039000808080808080808000808000808000005D
:1003A00000000000008080808080808080808080CD
:1003B00080808080808080000000000000000000BD
:1003C000000000000000000000000000000000002D
:1003D000000080F0FEFFFFFFFF3F0F010000000064
:1003E00000000000C0E0381E0F0300010000000004
:1003F00000000000000000000000000000000000FD
:100400000000030301000000000000000000000ED7
:100410000E02020202020303000F0F000F0F080872
:1004200008080808080F0F08080808080F0F000040
:1004300000000F0F0000000000000000000000009E
:1004400000000000000000000000000000000000AC
:10045000C0F8BFFFFFFF1F7F010000000000000089
:1004600000F0FCFF7F78300000000000000000007A
:10047000000000000000000000000000000000007C
:10048000000000000000000000000000000000006C
:10049000000000000000000000000000000000005C
:1004A000000000000000000000000000000000004C
:1004B000000000000000000000000000000000003C
:1004C0000000000000000000000000000000301CE0
:1004D000070E0F07010000000000000000000000F0
:1004E000000000000000000000000000000000000C
:1004F00000000000000000000000000000000000FC
:1005000000000000000000001B1E272D36394B4E56
:10051000636C7278878D939CB1B4C6C9D2D8E1E47C
:1005200001020304010302040402030104030201A3
:1005300003010200040506076D656E75537461635F
:100540006B206F766572666C6F77006D656E7553A4
:100550007461636B20756E646572666C6F77007092
:100560007265737320616E79204B657900414C454B
:100570005254004D455353414745004C4F41444967
:100580004E47002020202020202020202020202036
:1005900020202020202020202000506C65617365E1
:1005A00020526573657420537769746368657300BE
:1005B0005377697463686573205761726E696E67FB
:1005C00000204F6C642056657273696F6E2045453C
:1005D00050524F4D202020434845434B2053455413
:1005E00054494E47532F43414C494200416C61727C
:1005F0006D732044697361626C6564005265736554
:1006000074207468726F74746C65005468726F74CF
:10061000746C65206E6F742069646C65005072653F
:10062000737320616E79206B657920746F20736B12
:10063000697000414C45525400454550524F4D2081
:100640006C6F77206D656D004F46464142535255A1
:1006500073525525454C73454C25544873544825D1
:10066000414C73414C25503120503125503220509F
:1006700032255033205033250054485252554445BA
:100680004C4549443049443149443241494C47453D
:100690004154524E535731535732535733535734B3
:1006A0005357355357365357375357385357395392
:1006B0005741535742535743004F4646004F4E2031
:1006C000002D2D2D004348002D2D2D200052554486
:1006D00020454C45205448522041494C200050317F
:1006E000202050322020503320204D4158204655A4
:1006F0004C4C43594331435943324359433350508F
:100700004D3150504D3250504D3350504D3450506B
:100710004D3550504D3650504D3750504D38434860
:100720003120434832204348332043483420434853
:100730003520434836204348372043483820434833
:1007400039204348313043483131434831324348FE
:100750003133434831344348313543483136002D35
:100760002D2D2D00564552533A2056312E35343911
:10077000382D6572657A00444154453A2031312E56
:1007800030322E323031320054494D453A2031302A
:100790003A31303A3331002053564E3A206572399F
:1007A000782D7237303800204D4F443A2041524462
:1007B000552020200012081200081C0808081C08F8
:1007C0000000082200490022080000000000227FEB
:1007D0002200000008220049002208000008220030
:1007E00049002208000000227F22000000000008CB
:1007F0002200490022080000081C0808081C080004
:1008000062319D438142E62BCE24CB54AD51D14879
:100810006B4AD450104BCE1D891FBF1F5F20DA21B9
:1008200054546D00457870457846466E654D656454
:1008300043727300544F540053544B1153542500CA
:10084000544D45115453570053544154005B4D458A
:100850004E555D20746F2072656672657368005333
:100860007461636B0F6200746D61696E0F6D73006C
:10087000746D7231204A69747465720F75730074F7
:100880006D72314C6174206D696E0F757300746DFB
:1008900072314C6174206D61780F7573005354414F
:1008A0005432004D6F64650042616E6447617000B0
:1008B000506F745363726F6C6C00416C61726D2089
:1008C0005761726E696E67004D656D6F7279205762
:1008D00061726E696E670054524530313241470093
:1008E00054524530313241470044656661756C743D
:1008F00020537700537769746368205761726E697B
:100900006E67005468726F74746C65205761726E04
:10091000696E670053706C617368204E616D65008D
:1009200053706C6173682073637265656E004F4627
:1009300046004C69676874206F6E2053746B204DBD
:1009400076004C69676874206F666620616674651E
:1009500072004C6967687420737769746368004635
:100960006C617368206F6E2062656570004265651A
:100970007020636F756E74646F776E004D696E756D
:1009800074652062656570005468726F74746C657C
:1009900020726576657273650053494E474F534D1B
:1009A0005046494C540046696C746572204144437A
:1009B00000496E616374697669747920616C617253
:1009C0006D0042617474657279207761726E696E30
:1009D0006700436F6E74726173740048617074696C
:1009E0006320537472656E67746800537065616B41
:1009F0006572205069746368004265657065725065
:100A00006953706B7200536F756E64204D6F64652F
:100A1000005175696574204E6F4B65792078536875
:100A20006F727453686F7274204E6F726D20204C19
:100A30006F6E672020784C6F6E672000426565708E
:100A40006572004F776E6572204E616D6500524190
:100A500044494F2053455455500043616C004D7537
:100A60006C7469706C6965720063683163683263C5
:100A70006833636834006F6666202B3D203A3D0082
:100A80006D6F64650A2520737263202073770053AD
:100A90006C61766500545241494E45520000030393
:100AA00003030056455253494F4E005472696D2D51
:100AB000202B00204D656E75204578697420446FA9
:100AC000776E20202055705269676874204C6566E7
:100AD00074004449414700424700414E41005B4D8C
:100AE000454E555D205748454E20444F4E45004DDC
:100AF0004F564520535449434B532F504F545300A6
:100B0000534554204D4944504F494E54005B4D4588
:100B10004E555D20544F205354415254005354417C
:100B200052542043414C4942524154494F4E004394
:100B3000414C4942524154494F4E0066726565002E
:100B40004D4F44454C53454C00434F4C2044697233
:100B5000656374696F6E0041494C20446972656336
:100B600074696F6E00454C45204469726563746911
:100B70006F6E0053776173682052696E6700436F30
:100B80006C6C656374697665002D2D2D20202031F5
:100B90003230202020313230582020313430202093
:100BA0002039302020202000537761736820547949
:100BB00070650048454C4920534554555000004449
:100BC000454C455445204D4F44454C0F5B4D454EDB
:100BD000555D0054325468547269670054726169FB
:100BE0006E657200452E204C696D69747300504F1C
:100BF000534E45470053686966742053656C004C3A
:100C000050342F4C5035202044534D326F6E6C7948
:100C10002044534D322F44534D580044534D2054DB
:100C20007970650053656E64205278204E756D6250
:100C30006572205B4D454E555D0050504D2046720B
:100C40004C656E0D6D536563002052784E756D00D6
:100C50003443482036434820384348203130434805
:100C600031324348313443483136434800755300EC
:100C7000755365630050504D202020505858202057
:100C80002044534D32202050504D313620005072B8
:100C90006F746F00524554413132330042656570C4
:100CA00020436E74005472696D205377004578704C
:100CB000202020457846696E6546696E6520204D86
:100CC000656469756D436F61727365005472696D17
:100CD00020496E6300542D4578706F00542D547276
:100CE000696D00436F756E7420446F776E436F7546
:100CF0006E7420557020200054696D657220005478
:100D00007269676765720054696D6572004E616D46
:100D100065005345545550000009010000000000D3
:100D2000000602004475706C69636174696E672027
:100D30006D6F64656C005B4D454E555D20205B45D5
:100D40005849545D005945530B4E4F0044454C459E
:100D50005445204D4F44454C004455504C49434167
:100D60005445204D4F44454C0020414243444546A4
:100D70004748494A4B4C4D4E4F505152535455568B
:100D80005758595A6162636465666768696A6B6C33
:100D90006D6E6F707172737475767778797A3031A1
:100DA00032333435363738395F2D2E006578702070
:100DB0002025202073773120737732004558504F1B
:100DC0002F4452000003445220486967680044528F
:100DD000204C6F77004452204D6964004472537771
:100DE0003200447253773100576569676874004573
:100DF00078706F004558504F2F445200002B2A52F4
:100E0000004D49584552005072657373205B455838
:100E100049545D20746F2061626F7274004D617877
:100E2000206D69786572732072656163683A20008D
:100E300044454C455445204D4958205B4D454E5541
:100E40005D00536C6F772020557000536C6F7720D6
:100E500020446F776E0044656C61792055700044C2
:100E6000656C617920446F776E00416464202020B6
:100E700020204D756C7469706C795265706C61637B
:100E80006520004D756C747078004F4646005761C0
:100E9000726E696E67005377697463680043757298
:100EA000766573004F4E204F4646005472696D00C0
:100EB0004F46464F4E2000466C4D6F646574726914
:100EC0006D004F666673657400466D5472696D56A9
:100ED000616C0057656967687400536F757263656C
:100EE0000045444954204D49582000494E5345522D
:100EF00054204D495820002D2D2D2D202020763EA8
:100F00006F66732020763C6F667320207C767C3E73
:100F10006F66737C767C3C6F6673414E4420202064
:100F2000204F522020202020584F52202020207671
:100F3000313D3D7632207631213D76322076313E8C
:100F40007632202076313C7632202076313E3D7656
:100F5000322076313C3D76322000535700435553C2
:100F6000544F4D20535749544348455300000253B2
:100F7000414645545920535749544348455300006E
:100F800002434C454152204D49584553205B4D4545
:100F90004E555D002052455441004368616E6E65B8
:100FA0006C204F726465720054454D504C4154455D
:100FB0005300434F5059205452494D205B4D454EEC
:100FC000555D002D2D2D494E56004C494D49545329
:100FD00000000303030303030303030303030303E7
:100FE00003030043560043555256455300505245A3
:100FF00053455400454449542D3E004355525645EF
:101000000009002D2D2D494E56004F46464F4E20CB
:10101000002D2D2D783E30783C307C787C663E303B
:10102000663C307C667C633120633220633320630E
:1010300034206335206336206337206338206339DA
:1010400020633130633131633132633133633134A2
:1010500063313563313600454550524F4D206F7630
:101060006572666C6F7700454550524F4D206F7624
:101070006572666C6F770067656E7772697465205C
:101080006572726F7200454550524F4D20466F7227
:101090006D617474696E67004261642045457072C9
:1010A0006F6D2044617461004D4F44454C202020F9
:1010B0002020004D45202020202020202000500806
:1010C0005000000000000000006F00000700070053
:1010D000147F147F14242A7F2A1223130864623693
:1010E000495522500005030000001C224100004128
:1010F000221C0014083E081408083E08080050305E
:1011000000000808080808006060000020100804BB
:1011100002003E49453E0000427F40006251494680
:101120000041494936001814127F0027454539000F
:101130003E49493200017905030036494936000627
:1011400049291E00003636000000563600000814FB
:1011500022411414141414412214080002015109EC
:101160000600060909067E0909097E7F49494936B4
:101170003E414141227F4141221C7F494949417FF3
:10118000090909013E4149497A7F0808087F004161
:101190007F41002040413F017F081422417F4040B1
:1011A00040407F020C027F7F0408107F3E41414196
:1011B0003E7F090909063E4151215E7F09192946F2
:1011C000264949493201017F01013F4040403F1F0C
:1011D0002040201F3F4030403F631408146307083D
:1011E0007008076151494543007F414100020408EE
:1011F00010200041417F00040201020440404040B1
:1012000040000102040020545454787F484444387C
:101210003844444420384444487F385454541808CF
:101220007E0901020C5252523E7F080404780044A9
:101230007D40002040443D007F1028440000417F55
:1012400040007C041804787C080404783844444442
:10125000387C14141408081414187C7C080404083E
:101260004854545420043F4440203C4040207C1CBF
:101270002040201C3C4020403C44281028440C5076
:1012800050503C4464544C44000836410000007FF8
:10129000000000413608000808221C08081C22082B
:1012A00008A06080000000000000000000000000B6
:1012B0000000FFFF0000000000001F3F00003F1F74
:1012C00000003030FFFF3030FFFF30303078CCCCC2
:1012D000FFFFCCCC8C0C060F0F86C0E070381C0CC6
:1012E0003CFEC7E3F33B1E0C00000000333B1F0F26
:1012F000000000000000F0F81C0E070300000000D2
:1013000003070E1CF8F000003030E0C0FCFCC0E029
:101310003030C0C0C0C0FCFCC0C0C0C00000000075
:10132000000000000000C0C0C0C0C0C0C0C0C0C03D
:101330000000000000000000000000000080C0E08D
:1013400070381C0C000000000000000000000000CD
:10135000000038380000000000000000000000001D
:10136000000003033F3F03033F3F03030C0C0C0C3F
:101370003F3F0C0C07030C0E07030100183C3C1800
:101380000F1F383133331E1E3333000000000000BE
:1013900000000000000003070E1C383000000000B1
:1013A00030381C0E07030000030301000F0F00017B
:1013B0000303000000000F0F000000000000333B9B
:1013C0001F0F0000000000000000000000000000EF
:1013D0000000183C3C18000000000C0E0703010040
:1013E000000000000000FCFE87C3E377FEFC000065
:1013F0000C0EFFFF0000000000000C0E0783C3E787
:101400007E3C00000303C3C3C3E7FE3C0000C0E012
:1014100070381C0EFFFF00003F3F33333373E3C3CC
:101420000000FCFEC7C3C3C78E0C00000303C3E368
:10143000733B1F0F00003CFEE7C3C3E7FE3C000008
:101440003C7EE7C3C3E7FEFC0000183C3C180000EC
:1014500000000000183C3C18000000000000C0E044
:10146000F0381C0E07033030303030303030303040
:1014700003070E1C38F0E0C000000C0E07030383C6
:10148000C3E77E3C00000F1F3B3130381F0F0000C8
:1014900030303F3F3030000000003C3E37333130C9
:1014A000303000003030303030391F0F000003037F
:1014B000030303033F3F00000C1C383030381F0F7C
:1014C00000000F1F383030391F0F000000003F3F71
:1014D0000000000000000F1F393030391F0F0000DE
:1014E000000030381C0E07030000060F0F06000036
:1014F00000000000333B1F0F00000000000000014F
:1015000003070E1C38300303030303030303030321
:1015100030381C0E070301000000000000003333C8
:101520000100000000003C7EE7C3C3E77E3CF0F80A
:10153000DCCEC7C7CEDCF8F0FFFFC3C3C3C3C3E72D
:10154000FE3CFCFE0703030303070E0CFFFF03032F
:1015500003070E1CF8F0FFFFC3C3C3C3C3C30303D9
:10156000FFFFC3C3C3C3C3C30303FCFE0703C3C35B
:10157000C3C7CECCFFFFC0C0C0C0C0C0FFFF0000CB
:101580000303FFFF03030000000000000303FFFF4D
:101590000303FFFFC0E0F0381C0E0703FFFF00004D
:1015A000000000000000FFFF0E1CF8F81C0EFFFFFB
:1015B000FFFF3870E0C08000FFFFFCFE070303035D
:1015C0000307FEFC000000000000000000003F3F99
:1015D0000000000000003F3F3F3F303030303039E6
:1015E0001F0F0F1F3830303030381C0C3F3F303069
:1015F00030381C0E07033F3F303030303030303051
:101600003F3F00000000000000000F1F3830303066
:1016100030303F3F3F3F0000000000003F3F0000F0
:1016200030303F3F303000000C1C383030381F0F56
:1016300000003F3F000103070E1C38303F3F3030B1
:101640003030303030303F3F0000000000003F3F7E
:101650003F3F0000000103033F3F0F1F3830303091
:1016600030381F0FFFFFC3C3C3C3C3E77E3CFCFE7C
:10167000070303030307FEFCFFFFC3C3C3C3C3E7A2
:101680007E3C3C7EE7C3C3C3C3C78E0C0303030386
:10169000FFFF03030303FFFF000000000000FFFF44
:1016A000FFFF000000000000FFFFFFFF0000000040
:1016B0000000FFFF0F1F38F0E0E0F0381F0F3F7F02
:1016C000E0C08080C0E07F3F03030383C3E3733B3C
:1016D0001F0F0000FFFF0303030300000C1C387002
:1016E000E0C080000000000003030303FFFF0000D0
:1016F00030381C0E07070E1C3830000000000000B8
:10170000000000003F3F00000000000000000F1F2D
:10171000383033371E1C3F333F3F000003070E1C99
:1017200038300C1C3830303030391F0F00000000CA
:101730003F3F000000000F1F3830303030381F0F9F
:1017400003070E1C38381C0E07030F1F38381F1FE5
:1017500038381F0F3C3E0703010103073E3C0000E1
:1017600000013F3F010000003C3E37333130303054
:10177000303000003F3F30303030000000000000CB
:10178000000103070E0C0000303030303F3F0000F6
:101790000000000000000000000030303030303029
:1017A00030303030000003070E1C383000000000DD
:1017B000303030303070E0C0FFFFC0E0703030704B
:1017C000E0C0C0E07030303030300000C0E0703039
:1017D0003070E0C0FFFFC0E0703030303070E0C0EB
:1017E000C0C0FCFEC7C303070E0CF0F89C0C0C0C29
:1017F0000C0CFCFCFFFFC0E070303070E0C000005B
:101800003030F3F300000000000000003030F3F34C
:101810000000FFFF0080C0E0703000000000030304
:10182000FFFF00000000F0F03070E0E07070E0C0FA
:10183000F0F0C0E070303070E0C0C0E070303030A8
:101840003070E0C0000000000000000000000C1E2E
:101850003F33333333333F3F3F3F30303030303826
:101860001F0F0F1F3830303030381C0C0F1F38302E
:10187000303030303F3F0F1F3B33333333330303BC
:1018800000003F3F0000000000000001333333330D
:10189000333B1F0F3F3F0000000000003F3F0000B0
:1018A00030303F3F303000000C1C383030381F0FD4
:1018B00000003F3F03070F1C3830000000003030AD
:1018C0003F3F303000003F3F0000030300003F3F38
:1018D0003F3F0000000000003F3F0F1F3830303016
:1018E00030381F0FF0F03030303030F0E0C0C0E062
:1018F000F0303030E0C0F0F0F0F0C0E07030307028
:10190000E0C0C0E0F0303030303000003030FFFF59
:10191000303000000000F0F0000000000000F0F0A7
:10192000F0F0000000000000F0F0F0F00000000017
:101930000000F0F03070E0C08080C0E07030F0F067
:10194000800000000000F0F03030303030B0F0F0B7
:1019500070300000C0E03C3E0703000000000000C3
:10196000FFFF00000000000003073E3CE0C0000055
:10197000C0C0C0C00C1CF8F0E0C0C0E0F0F81C0C07
:10198000C0C0C0C03F3F03030303030301000001C5
:101990000303030303033F3F3F3F00000000000039
:1019A0000000303133333333333F1E0C00000F1F40
:1019B000383030381C0C0F1F383030381C0C3F3F8B
:1019C00003070E1C38381C0E07030F1F38381C1C69
:1019D00038381F0F30381C0F07070F1C3830000134
:1019E00033333333333B1F0F30383C3E37333130E2
:1019F0003030000000010F1F3830000000000000F0
:101A00003F3F00000000000030381F0F01000000C1
:101A1000000000000C0E07030100000103070E0C7C
:101A20000000000040800804201002013C1A481AFF
:101A30004E1A5B1A621A6F1A7A1A851A53696D70F8
:101A40006C6520342D434800542D43757400537445
:101A500069636B7920542D43757400562D54616968
:101A60006C00456C65766F6E5C44656C7461004813
:101A7000656C69205365747570004779726F2053E7
:101A80006574757000536572766F205465737400C9
:101A90000000891112239B322446AD573665BF746E
:101AA000488CC19D5AAFD3BE6CCAE5DB7EE9F7F81E
:101AB0008110080193331A22A5562C47B7753E644E
:101AC000C99C408DDBBF52AEEDDA64CBFFF976E8FE
:101AD00002218B30100299132667AF763444BD552E
:101AE0004AADC3BC588ED19F6EEBE7FA7CC8F5D9DE
:101AF00083310A2091121803A7772E66B5543C450E
:101B0000CBBD42ACD99E508FEFFB66EAFDD874C9BD
:101B100004428D5316619F702004A9153227BB36ED
:101B20004CCEC5DF5EEDD7FC6888E1997AABF3BA9D
:101B300085520C4397711E60A1142805B3373A26CD
:101B4000CDDE44CFDFFD56ECE9986089FBBB72AA7D
:101B500006638F7214409D512225AB343006B917AD
:101B60004EEFC7FE5CCCD5DD6AA9E3B8788AF19B5D
:101B700087730E6295501C41A3352A24B11638078D
:101B8000CFFF46EEDDDC54CDEBB962A8F99A708B3D
:101B9000088481951AA793B62CC2A5D33EE1B7F06D
:101BA0004008C919522BDB3A644EED5F766DFF7C1D
:101BB000899400859BB712A6ADD224C3BFF136E04D
:101BC000C1184809D33B5A2AE55E6C4FF77D7E6CFD
:101BD0000AA583B4188691972EE3A7F23CC0B5D12D
:101BE0004229CB38500AD91B666FEF7E744CFD5DDD
:101BF0008BB502A499961087AFF326E2BDD034C10D
:101C0000C3394A28D11A580BE77F6E6EF55C7C4DBC
:101C10000CC685D71EE597F42880A1913AA3B3B2EC
:101C2000444ACD5B5669DF78600CE91D722FFB3E9C
:101C30008DD604C79FF516E4A9902081BBB332A2CC
:101C4000C55A4C4BD7795E68E11C680DF33F7A2E7C
:101C50000EE787F61CC495D52AA1A3B03882B193AC
:101C6000466BCF7A5448DD59622DEB3C700EF91F5C
:101C70008FF706E69DD414C5ABB122A0B99230838C
:101C8000C77B4E6AD5585C49E33D6A2CF11E780F3C
:101C900020415244552050494C4F54204D656761B6
:101CA000203F2F3820002052544C20446973746127
:101CB0006E636500204172647550696C6F74204DCD
:101CC0006F64650020506974636820416E676C65BD
:101CD0000020526F6C6C20416E676C650020436C75
:101CE000696D622052617465200020416972205341
:101CF0007065656420002044697374616E636520BB
:101D0000002057617920506F696E742023200020D5
:101D100042656172696E670020436F75727365007A
:101D200020416C74697475646520486F6C64002090
:101D3000416C7469747564650020436C696D622040
:101D400072617465002047726F756E6420737065F0
:101D5000656400204C6F6E67697475646500204C83
:101D600061746974756465003E1A11241FBECFEF5B
:101D7000D0E1DEBFCDBF11E0A0E0B1E0E8EDF5EECF
:101D800002C005900D92A434B107D9F71EE0A4E477
:101D9000B1E001C01D92AA39B107E1F71DE1CAE621
:101DA000DDE104C02297FE010E94A572C836D1076A
:101DB000C9F70E946E190C94EA720C9400003091DD
:101DC000B70422B78091B7043817C9F7932F80E082
:101DD00030E0282B392BC901089529E282029001B5
:101DE0001124359527953595279587FD815C86FBD0
:101DF000880F880B80F9992787FD9095281B390B50
:101E0000C9010895F8942091D70D3091D80D789498
:101E1000C9010895482F50E09A01220F331F63E053
:101E2000440F551F6A95E1F7240F351F22543E4F8A
:101E3000C901089590E09C01220F331F220F331F28
:101E4000280F391F22503D4FC9010895AF92BF920C
:101E5000CF92DF92EF92FF920F931F93CF93DF9376
:101E6000C82E162FEA01F22ED02E57FF10C022FFE7
:101E700002C08CE101C08FE09C2D981B892F612F3F
:101E80004DE22F2D0E942A5DD095C195DF4F2D2D5B
:101E90002F218C2D612F4AE30E942A5D8F2D90E027
:101EA000B4E0AB2EB12CA822B922F2FE02C0E2E0CF
:101EB00001C0E0E0CE016CE370E00E9453729B0130
:101EC000442737FD4095542F0F2D00618E2F8C0D28
:101ED000612FA2E0EA2E0E942A5FA114B10411F042
:101EE000ECE101C0E1E1CE016CE370E00E945372CD
:101EF0009C01442737FD4095542F0D2D00618E2FF6
:101F00008C0D612FF2E0EF2E0E942A5FDF91CF91BE
:101F10001F910F91FF90EF90DF90CF90BF90AF9007
:101F200008950F931F93062F122F206250E00E94F6
:101F3000606017FD07C08091A90D602F46E7212F33
:101F40000E942A5D1F910F910895242F409108014E
:101F50000E94910F08950F93022F442319F44FE527
:101F600057E020C04530A8F4E0918801F0E0EE0F82
:101F7000FF1FEE0FFF1F3197E40FF11DE05EFA4FD8
:101F8000449150E0440F551F440F551F4753594F7C
:101F900009C0453250F450E0440F551F440F551FFF
:101FA0004653594F24E00E94ED5D0F910895FF9232
:101FB0000F931F93182FF62E022F442321F448EC81
:101FC00056E024E00EC08A5E4A3008F485506F2D3A
:101FD00050E0202F0E946060812F6F2D45EC56E06D
:101FE00022E00E94ED5D1F910F91FF9008950F93E5
:101FF0001F93DF93CF9300D0CDB7DEB7382F162FC6
:10200000942F022F442329F0463139F04A3E81F4BF
:1020100008C08A5F41EC56E007C08A5F4DEB56E08E
:1020200003C08A5F49EB56E0202F0E941D5E28C046
:102030004095441F4427441F81E2841B482F832F6F
:1020400039839A830E942A5D3981832F8A5F9A811E
:10205000E92FFF27E7FDF095F7FF03C0F095E19525
:10206000FF4FFF27E7FDF0953197AF01440F551F54
:102070004E0F5F1F4758594F612F23E00E94ED5DBF
:102080000F900F90CF91DF911F910F91089589E7E5
:1020900096E00895DF92EF92FF920F931F93D82E50
:1020A000E62EF42E1091AF01E12FFF27E7FDF0950A
:1020B000F7FF03C0F095E195FF4FE031A4F483E012
:1020C000E802F0011124E85BF94F8D2D6E2DAF0170
:1020D00023E00F2D0E94ED5D1F3F3CF58D2D8650B6
:1020E0006E2D41E21FC08D2D8650E53264F411162D
:1020F0001CF4412F4F5002C0412F415F6E2D2F2DF8
:102100000E94F70F12C011161CF4412F445202C056
:10211000412F4C5D6E2D2F2D0E94F70F8D2D8E5E61
:102120006E2D4DE62F2D0E942A5D1F910F91FF907D
:10213000EF90DF9008958C3038F4E82FF0E0EE0F48
:10214000FF1FEF50FB4F2AC0803198F4E82FF0E0DA
:10215000DF01AA0FBB1FA257BB4FEE0FFF1FE25AB2
:10216000FE4F2D913C91119780819181281B390B55
:102170000AC0843158F4E82FF0E0EE0FFF1FE25759
:10218000FB4F20813181220F331F0DC0843248F470
:10219000E82FF0E0EE0FFF1FE952FB4F2081318165
:1021A00002C020E030E0C9010895AF92BF92DF92F3
:1021B000EF92FF920F931F93DF93CF9300D0CDB791
:1021C000DEB7F82E463008F0DEC0882309F4DEC002
:1021D000863119F08A3E19F4D6C061E0D7C099273C
:1021E00087FD90959C0197FF04C022273327281B69
:1021F000390B2A307CF41F144CF02DE030E0A9019B
:10220000481B590BCA010E94CA61BAC00D960E94B0
:10221000CA61BBC02A50A22EBB249501220F331FD6
:102220002A0D3B1D2C553E4FF901E85AFD4F5081B8
:10223000552309F4A8C0453029F4F501EE57FB4FAA
:1022400080819CC0F901EA5AFD4FD080295A3D4F48
:10225000F901E080553008F4A6C0583060F08D2DAB
:1022600081504A8359830E949B108C018E2D81508E
:102270000E949B10A2C020E030E000E010E0583047
:1022800088F4553088F5523009F462C0533020F498
:10229000513009F06EC057C05330D1F0543009F0BE
:1022A00068C01CC05A3009F44EC05B3038F4583056
:1022B00009F43FC0593009F05CC040C05C3009F4FB
:1022C0004CC05C3008F444C05D3009F052C04AC0D4
:1022D00017FF39C0109501951F4F35C017FF38C043
:1022E000109501951F4F34C0142F1F5F8D2D60E096
:1022F000412F0E94D510082F8E2D60E0412F0E94A3
:10230000D510F501EE0FFF1FEA0DFB1DE450FC4F49
:102310009081953029F4002361F1882341F52AC08A
:10232000963029F4002319F5882319F120C080275D
:1023300021C081E002171307E1F41CC081E00217FD
:102340001307C1F416C081E0201731079CF011C0BB
:1023500081E00217130774F00CC081E00217130725
:102360004CF407C081E02017310724F402C081E05B
:1023700001C080E0F501EE57FB4F80831F142CF065
:1023800061E0682703C060E001C0682F862F0F90CE
:102390000F90CF91DF911F910F91FF90EF90DF9001
:1023A000BF90AF9008958D2D81504A8359830E942C
:1023B0009B108C018E2D0E94ED0E9C014A8159814B
:1023C0005ECF86B380958E7708950E94E1118823B1
:1023D000E1F70E94396108958091750160E040E065
:1023E0000E94D510882331F480919F049091A0041D
:1023F000009711F0C79A0895C79808950F931F93F7
:10240000CF93DF93EC018B010E94C05C82E260E01D
:1024100043E356E024E00E941D5E80E2BE010E947C
:10242000445E88E2B8010E94445E80E36DE176E09C
:102430000E94445E0E94CA60809172010E94C06046
:102440000E94E511DF91CF911F910F9108950F9395
:10245000AB0160E123E000E00E94ED5D0F91089583
:10246000DF92EF92FF920F931F93CF93DF938091B0
:10247000870181FD83C080EB95E06AE975E00E94E9
:10248000FE1190919F01892F887341F0883131F0BE
:10249000883221F0803311F0883329F4892F877C2A
:1024A000886080939F0100E010E065E1E62EF12C4A
:1024B00008C0C701801B91090E94CA61110F182B27
:1024C0000F5F0830B0F3D0909F01D12680E060E12B
:1024D00043E855E026E100E00E94ED5DCD2DD0E01F
:1024E000CE0180FF05C082E069E776E00E942712F6
:1024F000C1FF05C087E16CE776E00E942712C2FFAA
:1025000005C08CE26FE776E00E942712CE01887347
:1025100090700097B1F0012F13FF05C081E462E8CD
:1025200076E00E94271204FF05C081E465E876E0AA
:102530000E94271205FF05C081E468E876E00E944A
:102540002712C6FF05C086E56BE876E00E942712D9
:10255000D7FE05C08BE66EE876E00E9427120E9447
:10256000CA6080919F01181749F00E94E1118823E9
:1025700029F40E94EC1100E010E09BCFDF91CF9195
:102580001F910F91FF90EF90DF9008951F93CF93CD
:10259000DF930E94E11120E030E011E0482F50E08D
:1025A0002F5F3F4FBA01022E02C0759567950A94BE
:1025B000E2F760FD03C01F5F183091F7115016302D
:1025C00030F5812F0E943B57882309F11093710148
:1025D000812F0E943F5781E00E940E580E94C05CEC
:1025E00086E160E04BE755E024E00E941D5EC4EA0E
:1025F000D1E01AE04991812F68E124E00E942A5D30
:10260000155F1837B9F70E94CA600E94E511DF9183
:10261000CF911F910895CF93DF93EC010E94C05C8E
:1026200082E260E043E755E024E00E941D5E88E11D
:10263000BE010E94445E0E94CA60809172010E94A5
:10264000C060DF91CF9108951F93CF93DF93EC018A
:10265000162F0E94C05C82E260E04DE655E024E067
:102660000E941D5E88E1BE010E94445E8CE168E329
:102670004FE555E00E944C5E0E94CA60112319F498
:102680008091720101C089E10E94C06082E10E94D4
:10269000E86D0E94E5110E94E1118823C9F4809140
:1026A0006B0E833019F4A89510926B0E8091750112
:1026B00060E040E00E94D510882331F480918C01C5
:1026C000882311F4112311F0C79AE5CFC798E3CFFF
:1026D000DF91CF911F91089580918104882351F05B
:1026E00081EC95E060E00E942413809181048E7F4C
:1026F0008093810408958091870187FD07C08873C6
:1027000029F48CEE95E060E00E94241308958091F6
:10271000870182FD0AC00E942F59883C910528F448
:1027200089E396E060E00E9424130895EF92FF92FF
:10273000CF93DF93A82FAF70A6509091B60192303F
:1027400074F0292F332727FD309521503040C1E008
:10275000D0E002C0CC0FDD1F2A95E2F79C2FA830F5
:1027600008F09CC06A2F659570E0FB01EE0FFF1F1B
:10277000E050FF4F0190F081E02DB081992379F472
:10278000CB2FDD27C7FDD095D7FF03C0D095C195CE
:10279000DF4F9C2FC7FD9D5F959595959F5F40915D
:1027A000880150E04170507022E030E0241B350B6E
:1027B0002617370769F42091B5012F7009F473C00B
:1027C00021E094E030918A0130FF03C0919501C06F
:1027D00020E04B2F552747FD5095C92FDD27C7FD1A
:1027E000D095A0FF03C0C40FD51F04C0BA016C1B55
:1027F0007D0BEB01209729F07E019F2D9B2797FFF2
:102800000BC0222349F4BB2339F010820E942962B5
:1028100086E10E94E86D41C0CE0184589F4F893FF8
:102820009105B8F4C08386E00E940E58CE0183580B
:102830009F4F8B3F910588F5D7FF03C0D095C19579
:10284000DF4FD595C795D595C795BE01645C462FDA
:102850001FC01C161D0614F48DE701C083E8808399
:1028600086E00E940E58CE0183589F4F8B3F910502
:10287000A0F4CE01D7FF03C0909581959F4F64E0EF
:1028800070E00E945372709561957F4F462F445CB3
:1028900089E494E065E10E94756C80E0DF91CF915E
:1028A000FF90EF90089520E08DCF8F929F92AF928E
:1028B000BF92CF92DF92EF92FF920F931F93CF932D
:1028C000DF93182FEB015A016901802E84FF06C0A7
:1028D0001F70106694E0992E05E003C085E0982EE5
:1028E00004E0802F8066181761F0802F806418172D
:1028F00041F080912005882369F0133611F01334DC
:1029000049F47E010894E11CF11C83E10E94E86D0A
:10291000892D18C0992D9066191761F0992D906432
:10292000191741F0882309F474C0123619F01234D3
:1029300009F06FC07E010894E108F10884E10E946B
:10294000E86D802F90E00E94CA61882351F0EE2448
:10295000FF24EC1AFD0A892D0E942962802F0E9413
:102960002962A114B10491F481E0C816D10471F474
:10297000103661F41092200501E0E02EF12C209732
:1029800011F0EE24FF2480E60E94296220919C042D
:1029900030919D04E21AF30ACE14DF0444F4812F2F
:1029A0000E94296283E10E94E86D76010AC0EA1460
:1029B000FB043CF4812F0E94296284E10E94E86DAF
:1029C0007501EC16FD06A9F0E114F10451F4812F14
:1029D0000E941A62D7FF02C083E101C084E10E9415
:1029E000E86D882D83700E940E5881E080939904D1
:1029F00002C010929904C701DF91CF911F910F91EE
:102A0000FF90EF90DF90CF90BF90AF909F908F900E
:102A100008957E01A6CF0F93772767FD7095552700
:102A200047FD5095332727FD30950E9455140F918F
:102A300008950F93772767FD7095552747FD5095AB
:102A4000332727FD309502E00E9455140F91089519
:102A50000F93772767FD7095552747FD50953327CE
:102A600027FD309501E00E9455140F910895E091E3
:102A70009804F0E0EE0FFF1FE057FB4F808191813B
:102A8000089590919804992319F4882331F418C07B
:102A9000882319F4892F815001C080E08093980425
:102AA00087E10E94E86DE0919804F0E0EE0FFF1FCF
:102AB000E257FB4F0190F081E02D8EEB09950895D0
:102AC0008BE495E060E00E9424130895FC01A0913E
:102AD0009804B0E0AA0FBB1FA257BB4F8D939C93E5
:102AE0008FEB099587E10E94E86D0895CF93DF93FE
:102AF000EC0180919804982F9F5F909398049530F3
:102B000040F08093980488E395E060E00E942413ED
:102B10000FC087E10E94E86DE0919804F0E0EE0FAD
:102B2000FF1FE257FB4FD183C0838FEBFE01099556
:102B3000DF91CF91089589E494E00E94746B88231B
:102B400011F084E105C08091B804882321F0815000
:102B50008093B80407C09091630081E091FF80E00A
:102B60008093B9048091B90408951092A30410923F
:102B7000A5041092A4041092A204089520919F0429
:102B80003091A0042115310531F0215030403093AF
:102B9000A00420939F04882369F040918C0150E0A9
:102BA00084EF91E0489F9001499F300D589F300D70
:102BB000112402C020E030E08091A104882369F054
:102BC0006091940170E044EF51E0649FC001659F03
:102BD000900D749F900D112402C080E090E0409110
:102BE0009F045091A0044217530720F43093A0048F
:102BF00020939F0420919F043091A0042817390747
:102C000020F49093A00480939F040E94EC110895F7
:102C1000E82FF0E0E05DFA4FE491F0E0EE0FFF1FE7
:102C2000E454FB4F20813181C9010895CF92DF9296
:102C3000EF92FF920F931F93DF93CF930F92CDB735
:102C4000DEB720E0CC24DD24822F29830E940816E1
:102C5000092F10E0C00ED11E29812F5F2430A1F76B
:102C6000C6010F90CF91DF911F910F91FF90EF90D0
:102C7000DF90CF9008951F930E94020F41E02091B2
:102C8000EF043091F0048217930709F440E0409379
:102C90009E040E94020F9093F0048093EF0485E25B
:102CA00095E060E00E94A43580919E04882309F499
:102CB000CBC08091A20480FF14C08091A304982F00
:102CC0009F5F9093A304943660F083568093A3048F
:102CD0008091A4049091A50401969093A5048093FB
:102CE000A40480E00E941C580E94C05C0E943C61C9
:102CF0000E949613182F0E94BE152091FD0430915A
:102D0000FE0480919A0490919B04821B930B60E2D5
:102D100070E00E94537270939D0460939C0461154F
:102D2000710591F08091ED049091EE04821B930B5C
:102D300062E070E00E94537270939D0460939C0463
:102D400030939B0420939A043093EE042093ED0477
:102D500080918A0185FF04C010929D0410929C040A
:102D6000E0919804F0E0EE0FFF1FE257FB4F019057
:102D7000F081E02D812F09950E94CA600E949B1569
:102D8000882321F0809165008F7E03C080916500CB
:102D90008061809365000E94020F8F719070823075
:102DA000910509F04FC087E00E9408169C01E4E0FD
:102DB000220F331FEA95E1F768E070E00E9453723A
:102DC00040917401552747FD50954A5F5F4F649FBE
:102DD000C001659F900D749F900D1124820F931F69
:102DE00020918A0126FD05C06091090170910A01B8
:102DF00002C060EF70E02091080130E02F5F3F4F8C
:102E00000E943F72260F371F3595279520930801A2
:102E10008091EC04805E8093EC04882399F4809187
:102E20007301281778F4223368F081E10E94E86D7D
:102E300080918A0183FF06C082E390E09093A00412
:102E400080939F041092A1041F910895ACEBB4E00D
:102E5000ECECF4E060E0862F806487B9369A408914
:102E600051898D919C91119796958795840F951F07
:102E70008E7F11969C938E9320813181C901840F9E
:102E8000951F96958795918B808B349BFECF349AB6
:102E900084B195B1820F931F9695879581939193F5
:102EA0006F5F12966830B9F60895EF92FF920F9314
:102EB0001F93CF93DF9380918A0184FD44C00E94C9
:102EC000EC110E94C05C80E060E045E051E020E051
:102ED00000E00E94CB5C8091900184FD08C080E0FE
:102EE00068E345E951E02AE000E10E94ED5D0E94BF
:102EF000CA60809172010E94C0600E94E51100E2E8
:102F00000E9426170150E1F70E9416168C010E94BC
:102F1000020FEC01C057DE4F0DC00E9426170E9421
:102F200016167C010E94E111882369F4E016F1066F
:102F300051F406C00E94020FC817D90771F703C0E9
:102F40000E94EC11F7CFDF91CF911F910F91FF906D
:102F5000EF900895ECEBF4E040E012C067B9369AC8
:102F6000349BFECF349A24B135B1820F931F515058
:102F7000A9F796958795819391934F5F483031F0EB
:102F800054E080E090E0642F6064E8CF0895ECEBBB
:102F9000F4E020E0822F806487B9369A349BFECF1C
:102FA000349A84B195B1880F991F819391932F5FC3
:102FB000283081F70895FF920F931F93CF93DF93EB
:102FC0008091870180FD3AC08091880190E08170F6
:102FD000907002E010E0081B190BF801EE0FFF1FC4
:102FE000EC5BFE4FC181D281609687859089C81BBA
:102FF000D90B0E94C717F02E802F0E940816C81701
:10300000D907E4F40E94E1118823C1F40DC00E94A5
:10301000C7178F2D0E940816C817D9077CF40E9485
:10302000E111882341F00AC08BE096E06CEF75E077
:103030000E94FE11ECCF0E94EC11E9CFDF91CF91FD
:103040001F910F91FF9008958EE587B9369A349BB2
:10305000FECF349A84B195B1049640910901509104
:103060000A019A0163E0220F331F6A95E1F7241BDE
:10307000350B820F931F23E0969587952A95E1F7EC
:1030800090930A0180930901089578941F920F92FA
:103090000FB60F9211248F938091B7048F5F8093A6
:1030A000B7048F910F900FBE0F901F9018957894D2
:1030B0001F920F920FB60F9211242F933F934F93AD
:1030C0005F936F937F938F939F93AF93BF93EF9390
:1030D000FF93F89487B78D7F87BF789481B78E5F11
:1030E00081BF90914B0480914D04882379F08091A9
:1030F0009301882349F0813051F48091990E890F12
:103100008093990E87FF02C01B9A01C01B98809183
:103110000B01982F915090930B01882371F48DE44B
:1031200080930B0189E494E00E94886B0E943A62CC
:1031300080916B0E826080936B0EF89487B78260EB
:1031400087BF7894FF91EF91BF91AF919F918F913D
:103150007F916F915F914F913F912F910F900FBE93
:103160000F901F90189578941F920F920FB60F92A0
:1031700011241F932F933F934F935F936F937F93EC
:103180008F939F93AF93BF93EF93FF932091800012
:1031900030918100F89480917D008F7D80937D0037
:1031A00078948091BA049091BB04A901481B590BF3
:1031B000CA01969587953093BB042093BA04109169
:1031C000B604212F2150283058F59C01215233405C
:1031D00055E02737350708F5E12FF0E0EE0FFF1F28
:1031E000EC55FB4FAC014C5D554020918E013327CF
:1031F00027FD3095265F3F4F429FC001439F900DB2
:10320000529F900D11246AE070E00E945372718306
:1032100060831F5F1093B6040CC01092B60409C0FF
:10322000815A9F402EE28F3D920718F481E08093EF
:10323000B604F89480917D00806280937D0078943C
:10324000FF91EF91BF91AF919F918F917F916F917E
:103250005F914F913F912F911F910F900FBE0F9053
:103260001F901895EBE9FEE09F0181918535E1F310
:103270002A593E40C9010895CF93DF930E94DF0E83
:10328000EC0180918B01813019F40E94261707C050
:10329000823019F40E94AA1702C00E94C7178EE557
:1032A00087B90E943B160E94241880916B0E8330D0
:1032B00019F4A89510926B0E0E94DF0E8C1B9D0BCB
:1032C0002091C7063091C8062817390720F490933B
:1032D000C8068093C706DF91CF9108951F938FEFA3
:1032E0008ABB1BBA91E897BB9EE798BB9EE394BB51
:1032F00091EC95BB11BA82BB88E082B987EF83B9A4
:10330000109261001092620084E1809364008BEF60
:10331000809365000E948A600E94486F80E487B9AC
:1033200085E886B987E083BF8CE981BF87B7836072
:1033300087BF1FBC8AE08EBD10928B0082E880930D
:103340008A0080917D00806280937D00EDB7FEB79A
:10335000329785E502C0808331979EE0EA39F9070C
:1033600009F0C8F7789482E89FE390938F048093E4
:103370008E0489E10E94C0600E94C75710917101BC
:103380000E94C612809172010E94C06050918C010F
:1033900040919401451778F4652F70E024EF31E0F7
:1033A000629FC001639F900D729F900D11249093B6
:1033B000A00480939F04541770F450E024EF31E090
:1033C000429FC001439F900D529F900D11249093F6
:1033D000A00480939F040E94EC118091930181309E
:1033E00039F480918A0184FD03C087E00E94E86D72
:1033F0000E9455170E9487130E94C7170E94DB176F
:103400000E9430120E947B130E946C130E94E511EF
:1034100080EF90E090930A01809309010E94DF6998
:103420002DE088E190E00FB6F894A89581BD0FBE1D
:1034300021BD85E295E060E00E94A43582E691E33B
:103440000E94761581E00E944115809172010E94D0
:10345000C06080917101181729F081E00E940E5818
:103460000E94AA5880ED97E09BBD8ABD80E186BF8F
:1034700087B7806187BF0E943C19FDCF89E494E043
:103480000E94716B089529E2820290011124359502
:1034900027953595279587FD815C86FB880F880BDE
:1034A00080F9992787FD9095281B390BC90108954C
:1034B0009C01E5E035952795EA95E1F7AC01440FCD
:1034C000452F441F550B280F391F892F990F990B32
:1034D0008595280F391F241B350BC9010895F894D1
:1034E0002091D70D3091D80D7894C9010895AC0181
:1034F00080E060E021E00E941D5E08950F931F931D
:10350000CF93DF93182F88E498E00E94771A113642
:1035100058F0133628F0133639F489E19BE102C0E4
:1035200082E89FE30E94661586E068E040E458E088
:103530000E944C5E40913F06509140068AE268E04E
:1035400020E000E00E94260F409141065091420683
:103550008EE468E020E00E94260F86E060E148E308
:1035600058E00E944C5E40914306509144068AE226
:1035700060E120E00E94260F4091450650914606EA
:10358000F4E056954795FA95E1F78EE460E120E086
:103590000E94260F86E660E044E358E00E944C5EFD
:1035A00040913D0650913E068EE460E020E00E948E
:1035B000260F8091C3069091C4068937910528F0A3
:1035C0008091C206C82FD0E002C0C0E0D0E082E007
:1035D0006CE34EE70E94CA5E85E06CE143E20E9424
:1035E000CE5E1BE0812F6BE343E00E94CE5E1A5F4C
:1035F0001338C1F716E00CE3FE01E65BF94F40819A
:10360000602F641B812F0E94CE5E2196C837D105A2
:1036100010F0C0E0D0E02091C20630E0C217D3071E
:1036200019F01F5F1E3741F7DF91CF911F910F9166
:1036300008951F93182F8DE998E00E94771A12368B
:10364000E1F0133628F4103631F01136E9F418C0E1
:103650001336D1F415C08FEF97E090930D0180934E
:103660000C011092C6061092C5061092C806109260
:10367000C70687E10E94E86D07C08EE79AE102C0A5
:1036800082E89FE30E94661588E06EE878E00E9479
:10369000445E4091C5065091C6065695479584E50F
:1036A00068E00E94706080E16FE778E00E94445E0D
:1036B00040910C0150910D015695479584E560E1CC
:1036C0000E94706088E160E778E00E94445E40916B
:1036D000C5065091C60680910C0190910D01481BC2
:1036E000590B5695479584E568E10E94706080E229
:1036F00067E678E00E94445E2091C7063091C806D4
:1037000084E690E0289FA001299F500D389F500D1E
:103710001124A4E056954795AA95E1F784E560E267
:1037200020E30E94606088E26FE578E00E94445EDA
:103730000E943219AC018FE368E20E94505E82E180
:1037400068E34DE458E00E944C5E1F91089581E1CA
:1037500090E108950F9393E0499FA0011124465FE3
:103760005F4E01E0222309F400E023E00E94ED5DBA
:103770000F9108950F9393E0499FA00111244D5F8D
:103780005F4E01E0222309F400E023E00E94ED5D9A
:103790000F910895FF920F931F93F82E062F142F69
:1037A00080E860E0402F50E0212F0E9460600A30E6
:1037B00010F00FE601C005E7802F60E04FE2212FF7
:1037C0000E942A5D4F2D50E04F5F5F4F802F60E0D9
:1037D000212F0E9460601F910F91FF9008956F92BA
:1037E0007F928F929F92AF92CF92DF92EF92FF9251
:1037F0000F931F93CF93DF93EC01162FD42E490123
:103800006090F9047090FA048091C8089091C908FA
:103810008619970920E430E0B9010E945372462FBF
:1038200060932305E091FB04F091FC048091C608AD
:103830009091C7088E1B9F0BB9010E945372862F6F
:1038400060932405442321F07092C9086092C8084F
:10385000882321F0F093C708E093C60880912205E1
:10386000882321F480918A0185FF06C010922305E8
:10387000109224051092220560912305662351F4CD
:1038800080912405882331F480919C0490919D04BB
:10389000009781F040918C0150E024EF31E0429F8D
:1038A000C001439F900D529F900D11249093A0044E
:1038B00080939F048114910409F456C08881882361
:1038C00009F04BC0662331F180912005882311F562
:1038D000ED2DE61BE7FDE0E0202F30E08E2F99274D
:1038E00087FD90958217930714F0E02FE150FF2792
:1038F000E7FDF0958D2D90E0E817F90749F0EE0F00
:10390000FF1FE80DF91D25913491C9010E9466152C
:1039100010922305153641F4DD2011F0ED2D01C084
:10392000E02FF0E031970FC01436C9F42D2D30E0B0
:10393000802F90E00197281739071CF4ED2DEF5FD9
:1039400001C0E0E0F0E0EE0FFF1FE80DF91D25914A
:103950003491C9010E94661502C040E001C041E0F7
:103960008D2D602F0E94CA1BE114F10451F0988143
:103970008C2D9C1508F4892FF701E80FF11D549147
:1039800001C050E080912005882309F04FC080914C
:103990002405882329F14881481B47FD40E0242F56
:1039A000332727FD30958A2D90E0281739070CF032
:1039B0004A2D48838981E114F10459F0C41608F4B2
:1039C0004C2DF701E40FF11DE4918E1718F4E82F48
:1039D00001C0E0E0E98380E68093D90D10922405D0
:1039E0008881882319F1909123059923F9F0498161
:1039F000E114F104B1F0491B47FD40E09C2D8C150A
:103A000008F4982FF701E90FF11DE491242F3327D3
:103A100027FD30958E2F90E0281739071CF04E2F88
:103A200001C040E0498380E68093D90D103651F102
:103A3000113690F4133409F480C0143430F4113288
:103A400079F1123409F09CC06AC0143409F43FC003
:103A5000153409F095C04FC01436E9F1153638F425
:103A6000123609F45FC0133609F08AC069C01138F4
:103A7000A1F01F3B21F0153609F082C040C0198229
:103A8000188212C0552309F47BC081E09091200573
:103A9000911180E08093200573C0109220050DC025
:103AA00080912005882319F01092200569C0888133
:103AB000882319F08114910421F480E00E944115BB
:103AC0005FC087E10E94E86D1982188256C0898123
:103AD000851709F455C0E114F10409F451C080912F
:103AE0002005882309F04CC08981851710F48F5F69
:103AF00012C0198242C08981882309F441C0E114AF
:103B0000F10409F43DC0809120058823C9F589811D
:103B1000882319F08150898330C059832EC0888151
:103B20008A1571F180912005882351F588818A15C5
:103B300010F48F5F0DC018820EC08881882301F1B8
:103B4000809120058823E1F48881882319F0815031
:103B5000888301C0A8828981E114F10461F0988111
:103B60009C1508F4C92EEC0CF11CF70194918917EF
:103B700018F4982F01C090E0998380E68093D90DC6
:103B8000DF91CF911F910F91FF90EF90DF90CF9039
:103B9000AF909F908F907F906F9008954F925F921B
:103BA0006F927F928F929F92AF92BF92CF92DF924D
:103BB000EF92FF920F931F93DF93CF930F92CDB7A6
:103BC000DEB7D82E85E99AE00E94771A8AE498E059
:103BD0006D2D41E024E138E006E05DE9E52E5AE094
:103BE000F52E15E0C12EB6E0AB2E0E94EF1B8090A3
:103BF0004A0890904B088091630081FF07C08AE2D9
:103C000068E14FE85AE00E944C5E60C182E168E0E2
:103C100040E85AE00E944C5E8A94809120058823F7
:103C200019F0A2E0CA2E02C0CC24C394EE24FF24D3
:103C300010E1A82CBB24A7FCB094F4E06F2E712CEB
:103C40002701440C551C8EE791E0480E591E4E2D5D
:103C50004F5F80E0612F20E00E94AB0FAE14BF04E5
:103C600011F491E0911090E0F201218122952695C6
:103C70002695237030E0A901440F551F420F531FB2
:103C80004A58554F992311F400E001C00C2D88E1EA
:103C9000612F23E099830E94ED5D99819923C1F002
:103CA000809120058823A1F0F201618162956695DB
:103CB000669563708D2D40E022E00E942815829564
:103CC000880F880F807CF20191819F73982B9183DC
:103CD000AE14BF0421F401E0F92DF13009F000E049
:103CE000F2018181880F880F85958595FDE08F020F
:103CF000C0011124B3010E945372AB01002311F4DF
:103D000020E001C02C2D82E4612F0E94606000231E
:103D1000A9F080912005882389F0F2016181660F66
:103D2000660F659565958D2D41EE2FE10E94281552
:103D30008F73F2019181907C982B9183AE14BF0414
:103D400021F491E0F92DF23009F090E0F2012081A8
:103D5000277030E0A901440F551F420F531F4759E8
:103D6000554F992311F400E001C00C2D88E4612F18
:103D700023E099830E94ED5D9981992391F08091D0
:103D80002005882371F0F201608167708D2D40E07D
:103D900023E00E9428158770F2019081987F982B6C
:103DA0009083AE14BF0421F401E0F92DF33009F043
:103DB00000E0F2014081459545954595002311F4B9
:103DC00020E001C02C2D8AE5612F0E94F70F00230F
:103DD000B1F080912005882391F0F2016081659512
:103DE000659565958D2D4AEE26E10E942815880F70
:103DF000880F880FF20190819770982B9083185F3D
:103E00000894E11CF11C103309F01ACF80E36EE531
:103E10007AE00E94445E40918E01552747FD5095FF
:103E2000465F5F4FF82DF43011F421E201C020E22B
:103E30008EE460E30E946060282D243049F48D2DCB
:103E400060918E0146EF28E20E94281580938E0132
:103E5000EE24E394882D853009F0EE2480E068E3B9
:103E60004AE55AE02E2D0E941D5E46EAA42E44E04B
:103E7000B42E06E711E090E3F501419151915F0105
:103E8000F801219131918F01421B530B440F551FB3
:103E9000892F68E320E299830E9460609981985E8F
:103EA000903951F7EE2091F0FD2DF03679F4A6E728
:103EB000B1E0E6EAF4E088E001900D928150E1F78C
:103EC00081E00E940E5887E10E94E86D0F90CF912B
:103ED000DF911F910F91FF90EF90DF90CF90BF90F7
:103EE000AF909F908F907F906F905F904F900895CC
:103EF000AF92CF92EF92FF920F93AE2CEE24FF245D
:103F0000CC240E94EF1B0F91FF90EF90CF90AF90C9
:103F10000895EF920F93DF93CF930F92CDB7DEB753
:103F2000682F83EA9AE069830E94771A8CE498E00C
:103F3000698142E024E138E006E0EE240E94781F27
:103F400080E167E977E00E94445E88E164E677E01B
:103F50000E94445E80E267E777E00E94445E88E268
:103F600068E877E00E94445E80E367EA77E00E94B9
:103F7000445E0F90CF91DF910F91EF900895CF9213
:103F8000DF92EF92FF920F931F93DF93CF9300D0B6
:103F9000CDB7DEB7682F82ED9AE069830E94771A69
:103FA0008EE498E0698143E024E138E006E0EE2405
:103FB0000E94781FEEE0CE2ED12C00E010E01430ED
:103FC00020F078EFF72EF00E01C0F02EC6010E940F
:103FD000CA61E82E1F5F8AE26F2D412F20E00E9408
:103FE000F70F4E2D405D84E46F2D2E2D0E942A5D2B
:103FF000085F0894C11CD11C193009F708E3CC24D0
:10400000DD2410E0812F90E00E94CA61F82EA60105
:104010004D54554F80E0602F25E00E94175E4F2DD4
:10402000405D80E2602F2F2D0E942A5D1F5F85E09A
:1040300090E0C80ED91E0850163021F784E568E1DB
:104040004BEA5AE027E00E94175E66E0E62EF12C6C
:1040500010E230E084E5612F45EB57E0232F00E0CC
:104060003A830E94CB5CC7010E94CA61282FC70116
:10407000019629830E94CA61082F2981422F405D41
:104080008CE6612F0E942A5D402F405D88E7612FFA
:10409000202F0E942A5D3A813F5F185FE2E0F0E046
:1040A000EE0EFF1E3430B1F60F900F90CF91DF91DE
:1040B0001F910F91FF90EF90DF90CF9008958F9216
:1040C0009F92AF92BF92DF92EF92FF920F931F9356
:1040D000CF93DF93D82E8AED9AE00E94771A80E57D
:1040E00098E06D2D44E024E138E006E0EE24E3940E
:1040F0000E94781FF0905008C1EFD4E010E000E07B
:10410000812CF4E09F2EA12CB12C88E1612F41E499
:104110000E94E95D402F4F5C8EE1612F0E94E95DB6
:10412000802F0E940816AC018AE2612F0E94505E27
:104130000730B1F068817981882777FD8095982FC5
:1041400024E630E040E050E00E941472A5019401A2
:104150000E9488728AE5612FA9010E9470600AC0DE
:104160008F2D813011F040E201C041E28AE5612FDC
:104170000E94A50F0F5F185F2296083031F68CE67B
:1041800068E247ED5AE022E00E94175E4091090183
:1041900050910A0188E760E320E00E9460608F2D63
:1041A000813059F4F09222058D2D6091740141E81F
:1041B0002FE70E94281580937401DF91CF911F9102
:1041C0000F91FF90EF90DF90BF90AF909F908F90F6
:1041D0000895EF920F93E42E40E020E030E000E0FD
:1041E0000E94781F0F91EF900895AF92BF92CF92E7
:1041F000DF92EF92FF920F931F93DF93CF9300D044
:10420000CDB7DEB78FE161E247E10E94CE5E8FE17C
:1042100067E347E10E94CA5E85E361E247E10E94ED
:10422000CE5E8FE161E247E10E94CA5E8BE461E20B
:1042300047E10E94CE5E8BE467E347E10E94CA5EDD
:1042400081E661E247E10E94CE5E8BE461E247E1F4
:104250000E94CA5E8AE26BE243E00E94CE5E89E27F
:104260006CE243E00E94CA5E86E56BE243E00E9496
:10427000CE5E85E56CE243E00E94CA5E8091F10467
:104280009091F20451E7C52ED12CB6010E945372D1
:10429000262F8091F3049091F4040FE81FEFB801EA
:1042A0000E945372362F48E2E42EE20E9AE2F92E73
:1042B000F60E8E2D6F2D45E02A8339830E94CE5E47
:1042C0003981632F625D8E2D45E00E94CA5E2A818E
:1042D000822F845D6F2D45E00E94CE5E8E2D6F2D66
:1042E00045E00E94CA5E8091F7049091F804B601FF
:1042F0000E945372262F8091F5049091F604B80124
:104300000E945372062F84E5F82EF20E162F165DCA
:104310008F2D612F45E02A830E94CE5E602F625D63
:104320008F2D45E00E94CA5E2A81822F885A612F14
:1043300045E00E94CE5E8F2D612F45E00E94CA5E4F
:1043400019EFA12E14E0B12EBAE3FB2E0DE510E01B
:10435000A8E3EA2EF501819191915F0180509C4F75
:10436000B8010E945372D62ED394CE2CCD188F2D27
:104370006C2D4D2D0E94CE5E8F2D8F5F6C2D4D2D9F
:104380000E94CE5E8F2D8E5F6C2D4D2D0E94CE5ED5
:10439000F5E0FF0E8F2D8934E9F60F900F90CF9145
:1043A000DF911F910F91FF90EF90DF90CF90BF9022
:1043B000AF9008954F925F926F927F928F929F92EB
:1043C000AF92BF92CF92DF92EF92FF920F931F9323
:1043D000DF93CF930F92CDB7DEB7B82E8FE29BE07D
:1043E0000E94771A8DE798E06B2D45E024E138E0D4
:1043F00006E0EE24E3940E94781F10927D0811E6F7
:10440000E12E18E0F12EB3E5CB2EB8E0DB2E8601CD
:10441000470160E0862F69830E940816D4014D9100
:104420005C911197282F392F6981421753070CF49B
:104430009A01F401219331934F01D8014D915C9180
:104440001197282F392F241735070CF49A01F801FA
:10445000219331938F016F5F6730E1F680915208AD
:1044600080932205FB2DF03219F0FF3B71F40BC055
:104470008F5F80935208833041F487E10E94E86D9A
:1044800081E00E940E5810925208809152088130AB
:10449000B1F0813020F0823009F0A4C03FC08CE040
:1044A00060E14DE15BE021E100E00E94ED5D82E131
:1044B00068E14DE05BE02FE00E94ED5D93C08EE18E
:1044C00060E140E05BE02CE000E00E94ED5D82E115
:1044D00068E14EED5AE020E10E94ED5DAFE68A2EE4
:1044E000A8E09A2E20E008E91AE3F8E6AF2EF5ECF2
:1044F000BF2ED7010D931D937D01F601A192B192BC
:104500006F01822F29830E940816D4018D939D93F9
:104510004D0129812F5F273061F764C082E160E19E
:104520004FEE5AE020E100E00E94ED5D82E168E19B
:104530004EED5AE020E10E94ED5DEFE6AE2EE8E0A0
:10454000BE2E75E4472E71E0572EF20160E4862EF0
:10455000912CD7018D919D917D01D6016D907D901B
:104560006D019C012619370937FF03C0309521954D
:104570003F4F23333105DCF0D5012D913C91318340
:1045800020838901081B190BC801B4010E945372D2
:10459000061B170B17870687C301821B930B9C0111
:1045A000B4010E945372261B370B358F248FA2E073
:1045B000B0E0AA0EBB1E3296BFE6EB16B8E0FB06D3
:1045C00041F680E090E0F201219131912F01820FBC
:1045D000931FFDE54F16F1E05F06A9F79093700178
:1045E00080936F010E94F5200F90CF91DF911F9172
:1045F0000F91FF90EF90DF90CF90BF90AF909F9082
:104600008F907F906F905F904F900895282F30E0AB
:10461000C901880F991FA90163E0440F551F6A95CE
:10462000E1F7840F951FA9014F5F5F4FBA01660F35
:10463000771FA3E0440F551FAA95E1F7640F751F7C
:1046400062547E4F20953095205E3F4FA901440F64
:10465000551FE3E0220F331FEA95E1F7420F531F86
:1046600082549E4F0E94B8728AE0E4EFF2E0DF01CC
:104670001D928A95E9F782E00E940E580E94AA587E
:1046800008950F931F93CF93DF93282F30E0E90114
:10469000CC0FDD1FC90113E0880F991F1A95E1F7B0
:1046A000C80FD91F8E0102541E4FA9014F5F5F4FE3
:1046B000CA01880F991FA3E0440F551FAA95E1F77F
:1046C000840F951F20953095205E3F4FA901440F20
:1046D000551FE3E0220F331FEA95E1F7420F531F06
:1046E00082549E4FB8010E94B8728AE0D8011D9290
:1046F0008A95E9F78091A108CC55DE4F8A8F8B8F80
:1047000084E68C8F82E00E940E580E94AA58DF91A6
:10471000CF911F910F910895FF920F931F9385EFF3
:10472000E5E4F5E0DF011D928A95E9F780913A060C
:10473000AEEBB1E050E021E030E060E07C91772327
:1047400011F0472F01C040E1641738F5F22E032F16
:10475000162F1F5F802F90E0FC01EE0FFF1FEE0F62
:10476000FF1FE80FF91FEB5BFA4F912F9F738081BA
:10477000807C892B80648083F182F39453830F5F64
:10478000141738F3962F9095642F822F8F5F890F1F
:10479000390F340F290F240F840F772359F1832FFA
:1047A00090E0FC01EE0FFF1FEE0FFF1FE80FF91F57
:1047B000EB5BFA4F4F738081807C5483842B80683D
:1047C000808322832F5F1A968C911A97781719F499
:1047D0001182138205C021832F5F852F8F5F838312
:1047E000822F5F5F1A96503219F420933A0604C064
:1047F0003F5FA4CF80933A061F910F91FF900895D9
:10480000EEEBF1E080E090819150903108F48F5F01
:104810003A9692E0EE3FF907B1F708951F93182FEB
:1048200080E16DE17EE00E94445E0E940024482FFA
:1048300088E760E150E020E00E94606080E267E08D
:104840007EE00E94445E113651F481E60E942962A6
:1048500081E00E9441158EEC94E20E9476151F9132
:1048600008950E940024803230F08EE094E20E948D
:10487000761581E0089580E00895EF92FF920F93FE
:104880001F93DF93CF9300D0CDB7DEB7182F8132BF
:1048900008F07BC0882319F4442341F476C08032A9
:1048A00019F4442331F071C0442319F0012F0F5F34
:1048B00002C0012F0150812F4A8369830E940A0F91
:1048C0007C01802F0E940A0FFC01D7018C91982F48
:1048D00091504A816981903108F057C0208121317F
:1048E00008F053C06623A1F10E943124882309F007
:1048F0004CC0212F30E0A9014F5F5F4FCA01880FE4
:10490000991F13E0440F551F1A95E1F7840F951F67
:10491000B901660F771FA901A3E0440F551FAA959F
:10492000E1F7640F751F62547E4F20953095205E2D
:104930003F4FA901440F551FE3E0220F331FEA95B3
:10494000E1F7420F531F82549E4F0E94B8721DC060
:10495000281759F0442331F08031B8F48F5FF70104
:10496000808313C0D7019C9310C0D701CF010A9652
:1049700004C020813C9131932D93E817F907C9F7C2
:1049800082E00E940E580E94AA580F900F90CF917B
:10499000DF911F910F91FF90EF9008956F927F929A
:1049A0008F929F92AF92BF92CF92DF92EF92FF923F
:1049B0000F931F93CF93DF93182F81E09EE00E9407
:1049C000771AE0903A06EA9484EA98E0612F44E08E
:1049D00020E038E00AE00E94781FC090A408CC20B4
:1049E00011F41092A3081236D9F1133670F413346F
:1049F000A9F1143420F4123409F070C031C010361B
:104A0000C1F0113609F06AC045C0103809F452C02F
:104A1000113820F4133609F061C020C01E3BB9F1F3
:104A20001F3B09F05BC081E08093A2081092A308AD
:104A30002EC01C143CF481E09091A308911180E0F9
:104A40008093A3088091A3088093A20880919F0877
:104A5000882309F443C01092A30840C01092A20812
:104A60008091A3088823D1F141E0123609F040E09B
:104A70008091A0086091A2080E943D248091A20824
:104A8000882319F0133609F4CA941092A2080E94E0
:104A90008C2324C08091A308882301F18091A00871
:104AA0000E9406231092A3080E948C2381E60E9494
:104AB000296214C01C1494F480919F08882341F04B
:104AC0000E943124882321F48091A0080E94412370
:104AD0001092A30884E892E50E94761538E0D32E60
:104AE00077247A9423E6822E9924BB24BA946624F0
:104AF0006394E0901F05E90CFF24F701EE0FFF1F00
:104B0000EE0FFF1FEE0DFF1DEB5BFA4F4081842F70
:104B1000807C09F462C146FF06C04F7380E06D2DB2
:104B200020E00E94D70F1C14E4F4E701CC0FDD1F36
:104B3000CC0FDD1FCE0DDF1DCB5BDA4F8981C81690
:104B400081F46D2D695F80E048E10E94CA5E8B812F
:104B50008093A00888818F738093A10860929F083A
:104B6000B92CF701EE0FFF1FEE0FFF1FEE0DFF1D1B
:104B7000EB5BFA4F808187FF05C19481C92FDD2748
:104B8000C7FDD095AA24A3949281C912AA2486FDB8
:104B90001FC0FE01EE0FFF1FCE01A3E0880F991F7B
:104BA000AA95E1F7E80FF91FEB53FE4F40814695B8
:104BB000477050E04350524F8091A308882311F46E
:104BC00000E001C00A2D82E16D2D21E00E94ED5D23
:104BD000FE01EE0FFF1FCE0163E0880F991F6A955B
:104BE000E1F7E80FF91FEC55FE4F448D552747FDBF
:104BF00050958DE26D2D2A2D0E9460608091A30852
:104C0000882311F420E001C02A2D8DE26D2D45E2AC
:104C10000E942A5DFE01EE0FFF1FCE0143E0880FC8
:104C2000991F4A95E1F7E80FF91FEC55FE4F438DA8
:104C30008091A308882311F420E001C02A2D86E387
:104C40006D2D0E94AB0FFE01EE0FFF1FCE0123E082
:104C5000880F991F2A95E1F7E80FF91FEC55FE4FD1
:104C6000458D442359F08091A308882311F420E056
:104C700001C02A2D8EE46D2D0E94F70FFE01EE0F6C
:104C8000FF1FCE01B3E0880F991FBA95E1F7E80F37
:104C9000F91FEC55FE4F468D442391F023E0429FCF
:104CA000A00111244F5E5F4E8091A308882311F468
:104CB00000E001C00A2D86E66D2D23E00E94ED5D27
:104CC000FE01EE0FFF1FCE0173E0880F991F7A954A
:104CD000E1F7E80FF91FE254FE4F21E085818823B8
:104CE00009F420E0FE01EE0FFF1FCE0153E0880F14
:104CF000991F5A95E1F7E80FF91FE254FE4F86819C
:104D0000882329F0222309F498C04AE203C0222311
:104D100061F044E480912005882311F420E001C073
:104D20002A2D89E76D2D0E942A5D8A2D813051F54B
:104D30005E01AA0CBB1C33E0CC0FDD1F3A95E1F7F6
:104D4000AC0EBD1EE4EAF1E0AE0EBF1E812FF501F0
:104D5000648D43E82DE70E941915F501848FF70152
:104D6000EE0FFF1FEE0FFF1FEE0DFF1DEB5BFA4F67
:104D700084818093A00880818F738093A108109212
:104D80009F08B92CF701EE0FFF1FEE0FFF1FEE0D6E
:104D9000FF1DEB5BFA4F8181882331F088150CF4FD
:104DA000882E87150CF0782EF701EE0FFF1FEE0FFF
:104DB000FF1FEE0DFF1DEB5BFA4F8281882331F060
:104DC00088150CF4882E87150CF0782E9394F8E053
:104DD000DF0E292D273009F08CCECC20A1F08B2DB1
:104DE0008F3FF9F4C81464F480911F0590E0019797
:104DF000EFEF8F3F9E0711F480E090E080931F0556
:104E00007C14ECF414C0FB2DFF3F59F480911F0576
:104E100090E001972FEF8F3F920761F480E090E0E0
:104E200009C08B2D86305CF0992D983040F0809130
:104E30001F058F5F80931F0502C043E56BCFDF9195
:104E4000CF911F910F91FF90EF90DF90CF90BF9087
:104E5000AF909F908F907F906F9008952F923F9288
:104E60004F925F926F927F928F929F92AF92BF927A
:104E7000CF92DF92EF92FF920F931F935C01CC24AD
:104E8000DD243B018824992464E6262E312C412C14
:104E9000512CC201B1016619770988099909A60147
:104EA00095010E9414727B018C0182E390E0A0E0E6
:104EB000B0E0E80EF91E0A1F1B1FC601B5010E94D3
:104EC00014720E941472BC0188279927A4019301CF
:104ED0000E94147244E096958795779567954A9558
:104EE000D1F7E60EF71E081F191FC801B701A2016E
:104EF00091010E946672C9011F910F91FF90EF907E
:104F0000DF90CF90BF90AF909F908F907F906F90E9
:104F10005F904F903F902F9008951F93CF93DF9312
:104F20009C016115710511F1132F111F1127111F1C
:104F300019F0309521953F4F77FF0EC0C0E0D4E0C7
:104F4000709561957F4FCE01821B930B0E942E2797
:104F50009E01281B390B05C0C9010E942E27282F4E
:104F6000392F112319F0309521953F4FC901DF9159
:104F7000CF911F9108956F927F928F929F92AF92DF
:104F8000BF92CF92DF92EF92FF920F931F93DF9326
:104F9000CF93CDB7DEB7982E962F322F802F6E2D60
:104FA000222359F0442361F440919C0450919D04C4
:104FB0004115510539F421E001C020E0FF2405C06E
:104FC00022E001C021E0FF24F394332311F091117A
:104FD00021E04A2D433679F44C2D50E0440F551F03
:104FE0008A0173E0000F111F7A95E1F7041B150B7E
:104FF000065A1C4F11C0FA2DF236D9F44C2D50E050
:10500000440F551F8A0193E0000F111F9A95E1F795
:10501000041B150B055A1C4FF80140810E94F70F25
:10502000FF2009F463C0F8016081892D4AEE26E172
:1050300059C069887724BB24882051F54C2D50E055
:10504000440F551F6A01B3E0CC0CDD1CBA95E1F7A3
:10505000C41AD50AAA0CBB1CAA0CBB1CCA0CDB1CAC
:10506000C60CD71C4EE453E0C40ED51EF601408199
:10507000552747FD50950E946060FF20B9F1F60169
:105080006081892D4CE924E60E941915F6012DC096
:10509000DD24AA0CBB1CA601E3E0440F551FEA95D2
:1050A000E1F74C195D09A40EB51EA80CB11CAA0CA1
:1050B000BB1CF301EA0DFB1DE25BFC4F4081552751
:1050C00047FD50954C595F4F0E946060FF2071F082
:1050D0008501060D171D025B1C4F892DF8016081AB
:1050E0004CE920E00E941915F8018083CF91DF91EF
:1050F0001F910F91FF90EF90DF90CF90BF90AF90F6
:105100009F908F907F906F9008952F923F924F9233
:105110005F926F927F928F929F92AF92BF92CF9247
:10512000DF92EF92FF920F931F93DF93CF93CDB750
:10513000DEB72A970FB6F894DEBF0FBECDBFD82ECC
:1051400084EF9DE00E94771A8DE998E06D2D40E094
:1051500020E030E000E07CEFE72E7DE0F72ECC246D
:1051600053E0A52E0E94EF1B409195084F5F80E30E
:1051700060E020E00E94AB0FF0909D0880919508C0
:1051800090E0880F991FFC0123E0EE0FFF1F2A9586
:10519000E1F7E81BF90BE65AFC4F808160E040E044
:1051A0000E94D5108823C1F08091950890E0880F67
:1051B000991FFC0113E0EE0FFF1F1A95E1F7E81BA2
:1051C000F90BE55AFC4F808160E040E00E94D51069
:1051D000882321F411E003C010E001C012E06091C7
:1051E0009508462F50E0FA01EE0FFF1FEF50FB4FDE
:1051F000808191818A3191051CF010929C0807C032
:105200002FEF873E92071CF481E080939C08209149
:10521000880130E02170307082E090E0821B930BB7
:105220008417950741F4643030F48091B501807F94
:1052300011F010929C0880E16FEE7DE00E94445EC8
:105240000F92EDB7FEB7319621E0F11020E080918A
:105250009C0880838D2D61E041E006E3A0E1EA2E09
:10526000C0909508A12E88240E94BB270F9088E14A
:1052700068EE7DE00E94445E0F92EDB7FEB7319676
:1052800021E03F2D313009F020E080919C0880839F
:105290008D2D61E041E006E3F8E1EF2EC090950826
:1052A000A12E882483940E94BB270F9080E262EE97
:1052B0007DE00E94445E0F92EDB7FEB7319621E08B
:1052C0008F2D823009F020E010828D2D61E041E0C9
:1052D0000EE1E0E2EE2EC090950873E6A72E88243A
:1052E0000E94BB270F9088E26CED7DE00E94445E37
:1052F0000F92EDB7FEB7319621E09F2D933009F064
:1053000020E010828D2D61E041E00EE158E2E52EB3
:10531000C090950832E6A32E88240E94BB270F90E8
:10532000113019F0123049F404C080E365ED7DE0DE
:1053300007C080E36EEC7DE003C080E366EC7DE0B7
:105340000E94445E00919508402F50E0812F90E02C
:10535000880F991F880F991FBA01660F771F9B014D
:10536000B3E0220F331FBA95E1F7261B370B820FEC
:10537000931F8C559E4FFC01E655FE4FA081A983DB
:10538000FC01E555FE4FB081BA83FC01E455FE4FA8
:105390009080E4E69E0E83559E4FDC018C908E0E2D
:1053A0002091880130E02170307082E090E0821B13
:1053B000930B8417950709F062C0043008F05FC0B2
:1053C0008091B501807F09F45AC0EE24FF24870143
:1053D00020E030E0B9816B2E772467FC7094A1E265
:1053E0004A2E512C292C332427FC3094F0E4CF2E64
:1053F000D22ED801C701B595A79597958795B3018A
:1054000029873A870E948D27880F991FB2010E9431
:105410005372629DC001639D900D729D900D112489
:105420006FE3A62EAD0C64E670E00E943F72EC2D97
:10543000E61B6E2F8A2D0E947E5E29853A85C90162
:1054400083709070009761F48A2D6FE30E947E5EF6
:105450006D2D6695605E8FE30E947E5E3A8529859C
:105460002F5F3F4F81E290E0A0E0B0E0E80EF91E30
:105470000A1F1B1F2E33310509F0BACF7CC0DD2473
:105480009981492E552447FC509401E210E0A92D42
:10549000BB27A7FDB095BC83AB8354E6652E712C6A
:1054A00040E2A42EBA812B2E332427FC3094E82D21
:1054B000FF27E7FDF095FE83ED83FD2D21E2F29FAE
:1054C00070011124C701B2010E948D27B8010E940A
:1054D0005372AB81BC816A9FC0016B9F900D7A9F14
:1054E000900D11243EE5C32ECD0CB3010E943F72F6
:1054F000BA2DB61B6B2F8C2D0E947E5EED2DF0E039
:10550000E370F070F887EF83309749F48C2D60E2F8
:105510000E947E5E6D2D605E8EE50E947E5EC701FC
:10552000B1010E948D27B8010E9453722D813E81E6
:10553000629FC001639F900D729F900D11242EE514
:10554000F22EFD18B3010E943F72605E8F2D0E9403
:105550007E5E8F819885009749F48F2D60E20E94CE
:105560007E5E6A2D6D198EE50E947E5ED3949D2D20
:105570009F3109F0A2CFE0919508F0E0EE0FFF1FF8
:10558000EF50FB4F408051805201CC24B7FCC094B7
:10559000DC2CC601B50121E230E040E050E00E9481
:1055A0008872822F825A61E04EE30E94CE5E409163
:1055B00095082091880130E02170307082E090E001
:1055C000821B930B242F30E08217930709F050C001
:1055D000443008F04DC08091B501807F09F448C087
:1055E000C601B50160507C4F8F4F9F4F22E030E0E5
:1055F00040E050E00E948872A9816A2F772767FDFA
:105600007095C9010E948D27BC01660F771F8827FE
:1056100077FD8095982F292D97FC2D5F2595259551
:10562000332727FD3095432F532F0E94147229E111
:1056300030E040E050E00E94887279018A01CA019E
:10564000B9012FED3FEF4FEF5FEF0E948872622F9D
:10565000605C8FE34EE30E94CA5EC801B70122E09E
:1056600030E040E050E00E94887279018A013CC03D
:105670001A141B041C041D0414F4698101C06A81FE
:10568000772767FD7095C2010E948D279C014427F2
:1056900037FD4095542F1A141B041C041D0414F4E8
:1056A000692D01C0682D67FD6D5F6595659577274C
:1056B00067FD7095872F972F0E94147229E130E0C3
:1056C00040E050E00E94887279018A01CA01B90164
:1056D0002FED3FEF4FEF5FEF0E948872622F605E09
:1056E0008FE34EE30E94CA5EC601B50129E130E0B6
:1056F00040E050E00E941472612CB1E07B2E812CBE
:10570000912CA40193010E94887282E760E3A901B1
:1057100020E00E946060C801B70129E130E040E06C
:1057200050E00E941472A40193010E94887284E5E3
:1057300068E0A90120E00E9460601A141B041C04A8
:105740001D0474F4B9816B2F772767FD7095C20132
:1057500044970E948D27F701E81BF90BCF010BC07E
:10576000FA816F2F772767FD7095C20144960E94DA
:105770008D278E199F099C01220F331F220F331F83
:10578000280F391F442737FD4095542F84E560E1E9
:1057900000E3F3E0EF2E0E942A5F2A960FB6F894FA
:1057A000DEBF0FBECDBFCF91DF911F910F91FF9054
:1057B000EF90DF90CF90BF90AF909F908F907F90B1
:1057C0006F905F904F903F902F9008952F923F924F
:1057D0004F925F926F927F928F929F92AF92BF9201
:1057E000CF92DF92EF92FF920F931F93DF93CF93AD
:1057F000CDB7DEB72F970FB6F894DEBF0FBECDBF83
:10580000982E8CEB9DE00E94771A8AE998E0692D2A
:1058100043E020E038E00AE0F4ECEF2EFDE0FF2E5C
:10582000CC24C394E4E0AE2E0E94EF1BF0909A08C3
:10583000FA9430909B08292D203841F4F7FC06C0DB
:10584000F092950885E898E20E94761585E168E077
:105850004CEA5DE00E944C5E8AE593E09C838B837A
:1058600076E9472E78E0572EE1EFF4E0FB87EA87F0
:1058700010E1662477242F2D332727FD30953A83B6
:105880002983C901880F991FFC0153E0EE0FFF1F08
:105890005A95E1F7E81BF90BFE83ED83F62CEB81BB
:1058A000FC81808160E040E00E94D510882361F097
:1058B000EB81FC81818160E040E00E94D51088236B
:1058C00029F4BB24B39404C0BB2402C042E0B42E2C
:1058D0002B2D30E038872F83C901880F991F880F3F
:1058E000991FA301440F551F9A0103E0220F331F94
:1058F0000A95E1F7241B350B820F931F8C559E4FA1
:10590000DC01A355BE4FFC01E455FE4F3C912081C4
:10591000321751F4FC01E555FE4F86559E4F41E08C
:105920002081FC018081281340E0EA85FB8581917C
:105930009191FB87EA879C0197FF04C022273327B8
:10594000281B390B2A3131050CF040E0242E8A3116
:1059500091051CF0F201108207C0FFEF873E9F0700
:105960001CF421E0F20120838091880190E0817095
:105970009070E2E0F0E0E81BF90BE615F70551F452
:105980008091B501807F31F0F301EA56F74F108224
:10599000222423944F2D4F5F80E0612F20E00E944E
:1059A000AB0F5D864C86F2013081F1E0F987311151
:1059B000198680912005882351F4DD24D3948091A9
:1059C0009C0490919D04009721F4DD2402C0DD2405
:1059D000D39489819A818615970511F421E03110BD
:1059E00020E00F92EDB7FEB73183892D60E04D2D99
:1059F00007E2E12ECF2CAB2C88240E94BB270F900E
:105A000029813A812615370509F0D2C0332009F0E3
:105A1000CBC0DD2009F4CCC0222009F4C9C08F819D
:105A20009885880F991F880F991FED81FE818E0F31
:105A30009F1F8C559E4FF9858F0F911D86559E4F48
:105A40009F878E87892DEE85FF8560814CE924E64E
:105A50000E941915EE85FF858083AAC021E00F9270
:105A6000F2018081EDB7FEB78183892D60E04D2D75
:105A700009E3E12ECF2CAB2C882483940E94BB2712
:105A80000F9029813A812615370509F097C0332DEB
:105A9000313009F08FC0DD2009F490C0222009F4D4
:105AA0008DC08F819885880F991F880F991FED8170
:105AB000FE818E0F9F1F8C559E4FF9858F0F911D74
:105AC00084559E4F98878F83892DEF81F88560815B
:105AD0004CE920E00E941915EF81F88580836EC0A3
:105AE00021E00F92EDB7FEB71182892D60E04D2DB8
:105AF0000FE3E12ECF2CF3E6AF2E88240E94BB27C4
:105B00000F9029813A812615370521F421E0332DA4
:105B1000333009F020E00F92EDB7FEB71182892DE6
:105B200060E04D2D07E5E12ECF2CE2E6AE2E882475
:105B30000E94BB270894411C511C0F90EC85FD85E9
:105B40008081882319F4222031F008C0222031F40A
:105B50008AE34FE705C08BE34EE702C08AE34DE2DC
:105B6000612F0E94E95DFB2DF13019F0F23049F40C
:105B700004C085E7612F4DE407C085E7612F4CE441
:105B800003C085E7612F48E40E94E95D0894611C29
:105B9000711C2B813C81225F3F4F3C832B83185F1C
:105BA000103309F07BCE0CC0332D313009F456CFC1
:105BB00020E055CF832D823009F492CF20E091CFA1
:105BC0002F960FB6F894DEBF0FBECDBFCF91DF91F9
:105BD0001F910F91FF90EF90DF90CF90BF90AF900B
:105BE0009F908F907F906F905F904F903F902F90FD
:105BF000089520E030E0F901E759F24FE491E81709
:105C000011F4822F08952F5F3F4FEE23A1F780E01C
:105C10000895823430F4E82FF0E0E759F24F849190
:105C2000089580E20895EF92FF920F931F93182F2B
:105C3000F62EE22E862FBA010E94445E86E66F2D74
:105C4000412F2E2D0E94AA1BEE2039F0802F612FAC
:105C500040E021E00E942815182F812F1F910F91FD
:105C6000FF90EF900895FF920F931F93F82E1091DD
:105C7000AF01212F332727FD309537FF03C0309523
:105C800021953F4F022F25320CF43DC0209144084E
:105C9000309145088091420890914308282B392B78
:105CA0008091460890914708282B392B8091410814
:105CB00090E0282B392B40913E0850E0242B352BC7
:105CC0002115310531F4812F881F8827881F809383
:105CD0003E0811161CF4812F845202C0812F8C5D66
:105CE00060E040E00E94D510882359F090913E0872
:105CF000992339F491E020914108211190E090938B
:105D0000410880933E0820914408309145082F5F58
:105D10003F4F30934508209344082091420830912A
:105D200043082F0D311D30934308209342080E94F1
:105D3000020F2091460830914708821B930B84364E
:105D4000910508F471C12C593F4F309347082093B7
:105D500046082091420830914308E0914408F091B0
:105D60004508C901BF010E943F72F62E462F50E040
:105D70004E9FC0014F9F900D5E9F900D1124281BD8
:105D8000390B309343082093420810924508109233
:105D9000440800311CF4109241080FC005326CF425
:105DA00011161CF4812F8F5002C0812F815F60E09B
:105DB00040E00E94D5108093410880913D0690916B
:105DC0003E06019690933E0680933D0640913F0625
:105DD000509140064F5F5F4F5093400640933F06FF
:105DE000FF2049F0809143069091440601969093DC
:105DF00044068093430680914108882349F08091AE
:105E00004106909142060196909342068093410686
:105E1000F69420914506309146062F0D311D3093A2
:105E20004606209345068091B1019091B20190936E
:105E30004906809348066091AF01772767FD70950A
:105E400077FF03C0709561957F4F662319F4109218
:105E500047061EC0613019F4841B950B15C06031D4
:105E600068F460FF06C0A4E036952795AA95E1F78F
:105E700009C0209143063091440604C02091410698
:105E800030914206821B930B9093490680934806FB
:105E900080914706813051F0813018F0823049F509
:105EA00014C08091AF01882321F120C08091480661
:105EB0009091490618161906E4F08091B10190916D
:105EC000B2010097B1F082E012C080914806909133
:105ED00049062FEF853C92071CF483E08093470628
:105EE0008091B1019091B201009719F481E0809303
:105EF0004706809148069091490620913F083091CD
:105F000040082817390709F479C020914706213045
:105F100009F065C020918A0122FF45C02091B1019E
:105F20003091B20121153105F1F18E31910519F44D
:105F300089E10E94E86D809148069091490684317C
:105F4000910519F48AE10E94E86D809148069091CC
:105F500049068A30910519F48BE10E94E86D809121
:105F6000480690914906843091051CF48CE10E940A
:105F7000E86D80918A0183FF16C080914806909158
:105F800049068E31910549F08431910531F08A300E
:105F9000910519F08430910534F482E390E09093F8
:105FA000A00480939F0480918A0181FF27C0809183
:105FB000B001209148063091490680FF07C08091CA
:105FC000B1019091B201821B930B01C0C9016CE336
:105FD00070E00E943F72009789F480E003C0223095
:105FE00069F48CE10E94E86D80918A0183FF06C00C
:105FF00082E390E09093A00480939F042091480650
:10600000309149063093400820933F088091B001B9
:1060100080FF0AC08091B1019091B201821B930B65
:1060200090934906809348061F910F91FF90089521
:106030008091AF01992787FD909597FF03C09095B8
:1060400081959F4F982F823034F1803124F58595CA
:106050009A3024F40E944D6390E003C0992787FD95
:1060600090950197FC01EE0FFF1FEF50FB4F208131
:1060700031818091AF0187FF05C080E094E0821BF1
:10608000930B03C0C90180509C4F26E096958795DD
:106090002A95E1F702C080E090E00E94332E83E071
:1060A0000E944D63E82FF0E0EE0FFF1FE151FB4F20
:1060B0008081918180509C4FB6E096958795BA95E6
:1060C000E1F72091B00122FF0AC08530910538F038
:1060D0002091A204222319F423E02093A20420910A
:1060E0003A0830913B082F5F3F4F30933B08209395
:1060F0003A082091380830913908280F391F309319
:106100003908209338080E94020F20913C083091F2
:106110003D08821B930B23E0883E9207E8F10E9422
:10612000020F90933D0880933C088091B301823028
:1061300051F485E160E040E00E94D510882319F019
:1061400087E00E94E86D809138089091390860914D
:106150003A0870913B080E943F72109239081092E1
:10616000380810923B0810923A088091C30690912B
:10617000C40601969093C4068093C3068091C2061C
:10618000E82FF0E0E65BF94F60838F5F8093C206F3
:10619000883710F01092C2060895109247061092A8
:1061A000400610923F061092440610924306109249
:1061B0004206109241061092460610924506089536
:1061C0000F931F93182F80913B06882319F069E5E0
:1061D0007DE002C06CE47DE088E00E94445E81E0E6
:1061E00060E144EA51E02AE000E10E94ED5D82E4D2
:1061F00060E14FE30E94E95D82E168E245E45DE031
:106200000E944C5E82E160E346E35DE00E944C5EEA
:10621000113609F44AC01F3B21F0103609F04FC077
:1062200004C080E00E94E86D4AC080913B0688234C
:10623000A9F084E29DE00E940B1380913C060E942D
:106240007657882339F087E10E94E86D82E08093D9
:106250003B0629C080E00E94E86D25C08091710155
:106260008F5F0E943A5A1091710108C0115011318C
:1062700008F01FE080917101181739F0812F8F5FAE
:106280000E94ED59882391F301C010E01093710131
:1062900081E00E940E580E94AA58809171010E94CC
:1062A0003F570E94CD3080E601C081E60E942962FE
:1062B00081E00E94411582E691E30E9476151F91CC
:1062C0000F910895AF92BF92DF92EF92FF920F93DA
:1062D0001F93CF93DF93182F80E49BE00E94771ADF
:1062E000809120058823A1F4E0912305E7FF10C0E9
:1062F000E195EA3008F0E9E0F0E0EE0FFF1FE05032
:10630000F84F25913491C9010E946615109223051A
:10631000F0908F088FE898E0612F4FE00E94E9200D
:1063200086E360E04BE35BE00E944C5E0E942F59E5
:10633000AC0186E660E020E00E94606080E06AE0F8
:1063400041E00E94CA1BD0908F0880913B068230AA
:1063500021F410928E0810923B06163648F414363B
:1063600090F5103609F456C0113609F075C00AC010
:10637000113809F456C01F3B09F465C0103809F004
:106380006BC053C080918E088823E9F010928E086C
:1063900087E10E94E86D81E60E9429620E94AA5866
:1063A00080918F08809371010E943F570E94CD30E9
:1063B00081E00E940E580E94AA5882E00E940E5866
:1063C0000E94AA5849C0809171018D15B9F0812FA2
:1063D0000E94296280918F08809371010E94AA58BF
:1063E000809171010E943F570E94CD3081E00E9450
:1063F0000E580E94AA5881E00E94E86D153619F4E3
:1064000084ED90E504C0143639F58DE993E40E94DB
:10641000661522C081E080938E0887E10E94E86DB6
:106420001BC081E00E94411517C080918E0888230F
:1064300099F081E080933B06D0923C0680EE90E399
:106440000E94761509C010928E0880917101809388
:106450008F0881E00E941C5880918E08882341F0AB
:10646000FD1431F06D2D6F5F8F2D8F5F0E94FB59F2
:10647000CD2DDD27C7FDD09580911F059E01281BDE
:106480003109C901181619065CF0CE01019797FF72
:1064900002C080E090E080931F0510E1DD240BC076
:1064A00025303105D4F3CE0104978B3091059CF350
:1064B0008AE090E0F0CFF0901F05FD0CAF2CBB24DC
:1064C00095012F5F3F4F442737FD4095542FCA1544
:1064D000DB0511F401E101C000E182E1612F72E00E
:1064E000E72E0E942A5F80917101F81629F481E05D
:1064F000612F4AE20E94E95D8F2D6FE778E04FE05F
:106500000E94F756CA15DB0531F480918E08882366
:1065100011F001E101C000E188E1612F4FE758E08F
:106520002FE00E94ED5DD394185F3D2D363019F6B3
:10653000DF91CF911F910F91FF90EF90DF90BF906F
:10654000AF900895AF92BF92CF92DF92EF92FF92F9
:106550000F931F93CF93DF935B016C0110E1E12E4A
:10656000F12CC0E0D0E800E010E89E0140E050E0EF
:10657000CA01B9010E941472A616B706C806D90648
:1065800010F4C027D127169507950894E108F10863
:10659000E114F10461F4CE01DF91CF911F910F91CD
:1065A000FF90EF90DF90CF90BF90AF900895C02BF9
:1065B000D12BDBCFE1E0683068F4E0E070E09B01D4
:1065C000220F331F220F331F260F371FA9014657F3
:1065D0005C4F0EC070E0685070409B0153E0220F8A
:1065E000331F5A95E1F7260F371FA9014E545C4F10
:1065F000DA012C9180509C4F97FD0FC0B8E080309D
:106600009B078CF0EE2319F028E030E002C024E074
:1066100030E0240F351FF9012081332727FD309505
:10662000322F222730C0EE2329F0692F9070880F77
:10663000991F03C0692F66959170262F30E0FA01EB
:10664000E20FF31F6181772767FD7095AC015595C7
:106650004795649F9001659F300D749F300D112404
:106660006081772767FD709540E052E0481B590B29
:1066700055954795649FC001659F900D749F900D3F
:106680001124280F391FC90169E170E00E9453727B
:10669000CB0108952F923F924F925F926F927F921B
:1066A0009F92AF92BF92CF92DF92EF92FF920F93A1
:1066B0001F93DF93CF9300D00F92CDB7DEB7182F83
:1066C000992493948091A608883008F499248BEF3C
:1066D0009FE00E94771A992011F05AE001C056E01D
:1066E00084EC98E0612F40E020E030E000E071E0D1
:1066F000E72E70E1F72ECC24C394A52E0E94EF1B49
:106700004091A60850E04F5F5F4F84E260E021E0D7
:106710000E9460608091A608992079F090E0089727
:106720007C0103E0EE0CFF1C0A95E1F7E80EF91E70
:1067300022EB33E0E20EF31E0CC090E07C01EE0C85
:10674000FF1CEE0CFF1CE80EF91E8AE893E0E80E31
:10675000F91E0091C4080150D090C508113661F0AF
:10676000123628F41434D1F0153471F50EC01436F5
:10677000A9F0153649F509C0DD2031F11092C508A0
:1067800081E60E942962DD241FC0809120058823B4
:10679000D9F01D14CCF48D2D815014C080912005AA
:1067A000882391F02D2D332727FD3095992019F05E
:1067B00089E090E002C085E090E02817390724F4D2
:1067C0008D2D8F5F8093C5088091C508809320052B
:1067D000CE2C4F2C6E2C7F2C90E122243324A02E23
:1067E000BB24A7FCB094F30141913F01552747FD1D
:1067F000509521E0A214B30409F020E088E1692F4C
:1068000099830E9460600894211C311C9981985FD3
:10681000983349F7992001F1A5E06A2E712C6E0C8E
:106820007F1C90E1F5E02F2E312CF30141913F01C7
:10683000552747FD509521E0A214B30409F020E04C
:1068400080E3692F99830E9460600894211C311CA9
:106850009981985F903349F70F3F11F421E0D110EF
:1068600020E08CE068E044EF5FE00E941D5E99202C
:1068700019F089E090E002C085E090E021E0A816E0
:10688000B90609F020E08CE068E34DEE5FE00E947D
:106890001D5E992019F089E090E002C085E090E04B
:1068A000A816B90694F407FD4EC0A02EBB24A7FC81
:1068B000B094AE0CBF1C812FF50160814CE924E639
:1068C0000E941915F50180833EC01016E4F5812F52
:1068D0006091C3084CEF24E000E00E940B15809308
:1068E000C30890919904992371F1992021F050E106
:1068F00094E049E003C058E092E045E024E68202DB
:1069000030011124892F90E0909581959F4F869DAD
:106910009001879D300D969D300D1124EC2DF42DA6
:10692000A52E00E0C9016A2D702F0E945372619359
:10693000260D371D8E2F8C198417A0F382E00E943C
:106940000E580E94AA5880912005882351F0AA244D
:10695000ECE92E2EEFEF3E2E4D2C552447FC5094A3
:10696000A5C000E01CEFAA24BB2470E2D72EACC067
:10697000C90165E0880F991F6A95E1F7992019F020
:1069800064E070E002C062E070E00E945372462F43
:10699000062F055C37016A0C711CF3018081992771
:1069A00087FD909555E0880F991F5A95E1F7B10141
:1069B0000E945372562F90E2D92ED60E2F5F3F4F72
:1069C0008D2D90E09B838A834216530609F050C0B8
:1069D00082349105ACF48AE3C82EC40E625E8C2D1D
:1069E00045E059830E94CA5E5981EA81FB81E13406
:1069F000F10531F0652F615E8C2D45E00E94CA5E85
:106A0000FD2DF03430F4802F81506D2D45E00E9433
:106A1000CA5E2A813B812F33310594F401506D2DDC
:106A20006F5F802F45E00E94CA5E8A819B818E3312
:106A3000910531F06D2D6E5F802F45E00E94CA5E9A
:106A400080919C0490919D04009741F4123631F09E
:106A5000133621F0123411F0133439F5812FF3017C
:106A600060814CE924E60E941915F30180831DC062
:106A70002A813B81213431052CF4615E802F43E073
:106A80000E94CA5E3D2D303428F4802F6D2D43E0E6
:106A90000E94CA5E8A819B818F33910534F46D2DEB
:106AA0006F5F802F43E00E94CA5EA3942A2D30E0DE
:106AB000992019F089E090E002C085E090E0281765
:106AC00039070CF455CF4DCFC8016091A6080E943C
:106AD000DA32BCE3EB2EEA0C9C01A5E03695279553
:106AE000AA95E1F76D2D621B8E2D0E947E5E9501A9
:106AF000237030702115310521F48E2D60E20E9443
:106B00007E5E0894A11CB11C005E1F4F90E4A91684
:106B1000B104D1F68CE560E040E40E94CE5E0F90B7
:106B20000F900F90CF91DF911F910F91FF90EF90F9
:106B3000DF90CF90BF90AF909F907F906F905F90CD
:106B40004F903F902F9008952F923F924F925F92D7
:106B50006F927F928F929F92AF92BF92CF92DF926D
:106B6000EF92FF920F931F93DF93CF93CDB7DEB7D2
:106B7000A2970FB6F894DEBF0FBECDBF8F8F98A33C
:106B80006A8B80919E04882309F474C0809121054A
:106B9000882319F08150809321058091CB06909134
:106BA000CC062091C9063091CA06820F931F20910E
:106BB000CD063091CE06820F931F2091CF063091E3
:106BC000D006820F931F20915407309155072C0156
:106BD000421A530A920157FE03C0309521953F4F48
:106BE00041E0213034073CF09093550780935407DF
:106BF00081E08093A10480918901863FD9F1909131
:106C000008019233B8F1909151079F5F909351071B
:106C1000903160F020915207309153072F5F3F4F22
:106C20003093530720935207109251079091A1047B
:106C3000992321F010925307109252072091520786
:106C400030915307992787FD90950A9667E771E081
:106C5000869FA001879F500D969F500D11244217CB
:106C6000530740F4237030702130310519F480E16E
:106C70000E94E86D80918801582F51705F5F59879D
:106C800081FF02C01D8602C063E06D876090BC0179
:106C9000662009F44AC08985E82FF0E0EE0FFF1F57
:106CA000EF50FB4FA080B180CC24B7FCC094DC2C0B
:106CB0009D85E92FF0E0EE0FFF1FEF50FB4F208185
:106CC0003181442737FD4095542FCA01B9010E94F4
:106CD00014727B018C01C601B501A60195010E94C9
:106CE0001472E60EF71E081F191F662D70E080E073
:106CF00090E0EAE0660F771F881F991FEA95D1F7A9
:106D000024E630E040E050E00E948872B901CA01F8
:106D10000E9414726E157F058007910730F4C80138
:106D2000B7010E94A2324C0102C088249924B40108
:106D300080E090E024E630E040E050E00E941472F1
:106D40006B8F7C8F8D8F9E8F64E4662E61E0762E34
:106D5000A9ECB6E0BE8BAD8BFE013196F88FEF8BC0
:106D600050E0252E51E0352E24EA31E03F872E8772
:106D700041EF54E05A8F498F2901F98BE88BBC8B86
:106D8000AB8BEE24FF241B865A89517059A3AE2C7D
:106D90008E2D0E9408169C01D30111968D919C9115
:106DA0001297281B390BB901882777FD8095982FFA
:106DB0004AE0660F771F881F991F4A95D1F7121670
:106DC00013062CF45D962D913C915E9703C0F30160
:106DD000278530892436310514F424E630E0442731
:106DE00037FD4095542F0E9488728901FCEF2130B5
:106DF0003F072CF024E00030120724F405C000E027
:106E00001CEF02C000E014E080918A0180FF0FC0F7
:106E10008091880190E08170907042E050E0481BC2
:106E2000590BE416F50619F4109501951F4FA98D1D
:106E3000BA8D0D931D93BA8FA98FC8010F968F310C
:106E40009105F0F4B4E0EB16F1047CF48A2D8F5F29
:106E50000E944D6390E00197E1E0F0E002C0EE0F88
:106E6000FF1F8A95E2F7CF0108C081E090E00E2C69
:106E700002C0880F991F0A94E2F7FB85F82BFB8765
:106E80002A2D243008F07AC139A1332309F05FC0DC
:106E90008091B00181FF5BC06701CC0CDD1C4EE727
:106EA00051E0C40ED51ED60111968C911197807CAD
:106EB00009F44DC08C9185958595859561E040E0FC
:106EC0000E94D510882309F442C0D601EC91E770E6
:106ED000F0E0DF01AA0FBB1FAA55BB4FEE0FFF1F4B
:106EE000EA58FE4F8D919C91119720813181821B30
:106EF000930B62E070E00E945372F701EE0FFF1FE8
:106F0000E158FE4F2081422F440F440F459545958F
:106F1000552747FD5095649FC001659F900D749F54
:106F2000900D11246FE170E00E945372660F771F7D
:106F3000660F771F2295269526952370213019F02C
:106F4000223029F403C0060F171F01C08B018114E2
:106F5000910409F1B985AB1619F0ED85AE16D9F497
:106F60006091BC0170E080E090E04AE0660F771F1E
:106F7000881F991F4A95D1F79801442737FD4095FE
:106F8000542F0E9414722B8D3C8D4D8D5E8D0E946E
:106F90008872022F132FF201EA54FE4F808160E0C5
:106FA00040E00E94D510882369F0F201E954FE4FB9
:106FB000808160E040E00E94D510882329F4CC2431
:106FC000C39404C0CC2402C032E0C32E8091880157
:106FD00090E08170907022E0A22EB12CA81AB90A1C
:106FE000AE14BF0469F58091B501807F49F1C801F5
:106FF00080509C4F62E070E00E9453729B01EC2D28
:10700000F0E0EE0FFF1FEE0FFF1FA701440F551F0B
:10701000CA01A3E0880F991FAA95E1F7841B950B7D
:10702000E80FF91FE25BFC4F6081772767FD7095E1
:10703000C9010E948D27AC01440F551F30E028C0C4
:1070400031E0101611060CF430E08C2D90E0A70111
:10705000440F551FFA0163E0EE0FFF1F6A95E1F739
:10706000E41BF50B880F991F880F991FE80FF91F74
:10707000EC55FE4FE30FF11DE655FE4F608177277B
:1070800067FD7095C8013AA30E948D27AC013AA113
:10709000EC2DF0E0EE0FFF1FEE0FFF1FB701660FA4
:1070A000771FCB0113E0880F991F1A95E1F7861B14
:1070B000970BE80FF91FEC55FE4FE30FF11DE45558
:1070C000FE4F6081772767FD70956C597F4F882749
:1070D00077FD8095982FDA019D01442737FD409573
:1070E000542F0E94147224E630E040E050E00E94E9
:1070F0008872022F132FAE14BF0499F58091B50149
:10710000982F907F09F466C60050144063C6D101E1
:10711000ED91FC911197608180918A0180FD6195CC
:10712000772767FD7095872F972F63587F4F8F4F75
:107130009F4F20E034E0201B310B442737FD409562
:10714000542F0E94147220E038E040E050E00E948A
:1071500088722030B8E03B07B0E04B07B0E05B0737
:1071600039F4D101ED91FC912081332727FD309531
:10717000220F331FE889F98931832083AB89BC89C9
:107180000D931D93BC8BAB8B0894E11CF11CE2E0CA
:10719000F0E06E0E7F1E288939892E5F3F4F398BB4
:1071A000288B2E0E3F1E4EE050E0440E551E57E039
:1071B000E516F10409F0EBCD0091B9016B850623CA
:1071C000809156078095802319F088E10E94E86D30
:1071D0000093560780E094E09093D8068093D706FA
:1071E0009093DA068093D906E6EAF4E026E731E0E8
:1071F000A1EEB6E0BD0181919191D9014D915D91D2
:107200009D01841B950B880F991FDB018D939D9326
:10721000BD01B4E0EE3AFB0771F78091AE049091A6
:10722000AF04880F991F9093EA068093E906809136
:10723000B0049091B104880F991F9093EC0680934D
:10724000EB068091B2049091B304880F991F90933C
:10725000EE068093ED068091B4049091B504880FFA
:10726000991F9093F0068093EF06E1E1F7E0FC8729
:10727000EB8721EF36E04191519161917191D901F4
:107280004D935D939D01B7E0E135FB07A1F7C090F9
:10729000BC01CC2009F47AC0E985AE2EBB24AA0C2F
:1072A000BB1C29EC422E26E0522EA40CB51CD501A5
:1072B0002D903C90442437FC4094542CBD850B2FDA
:1072C00010E0000F111F0753194FF8012081318181
:1072D000442737FD4095542FCA01B9010E9414720A
:1072E0003B014C01C201B101A20191010E94147243
:1072F000660E771E881E991EDD24EE24FF248AE088
:10730000CC0CDD1CEE1CFF1C8A95D1F7C701B60121
:1073100024E630E040E050E00E948872B901CA01E2
:107320000E941472661577058805990578F5C401E1
:10733000B3010E94A232BC0180E090E024E630E07C
:1073400040E050E00E9414723B014C01C201B101C7
:10735000A70196010E941472A40193010E948872F1
:10736000D5012D933C93F80160817181882777FDC9
:107370008095982FA70196010E941472A401930191
:107380000E948872D80111963C932E93E090BA0126
:107390008E2D807E09F4DEC0B9852B2F30E0220FC0
:1073A000331FF901E753F94F40815181CE01019616
:1073B000280F391FD901ED91FC91BD856B2F70E02D
:1073C000660F771FDB01A753B94F2D913C91860FB4
:1073D000971FDC018D919C91BA89B1FD05C0E40F26
:1073E000F51F280F391F04C020E030E0E0E0F0E096
:1073F000A091BB01AA2349F0B0E0AA0FBB1FA9537B
:10740000B94F0D911C91119702C000E010E0E2FE0F
:1074100003C0F095E195FF4FE3FE03C03095219541
:107420003F4FE4FE03C0109501951F4F8091BA01B4
:10743000829586958770823071F1833020F4813097
:1074400009F088C007C0833009F459C0843009F0BE
:1074500081C06CC0C90168E070E00E9453727B017A
:10746000C90160E870E00E94537229014E185F085C
:107470007201E61AF70AC90160E072E00E945372D5
:10748000E61AF70AC8018E1B9F0B9093DC068093C7
:10749000DB06CF0120C0CF0168E070E00E9453728C
:1074A0007B01CF0160E870E00E9453723F016E18CB
:1074B0007F087301E61AF70ACF0160E072E00E94CC
:1074C0005372E61AF70AC801821B930B9093DC06ED
:1074D0008093DB06C90162E070E00E945372600F86
:1074E000711FCB018E0D9F1D9093DE068093DD06EC
:1074F0006E197F097093E0066093DF062BC0C80108
:107500008E1B9F0B9093DC068093DB06E00FF11F30
:10751000CF01820F931F9093DE068093DD06E21B5E
:10752000F30BF093E006E093DF0614C0C8018E1B56
:107530009F0B9093DC068093DB06C801820F931F9C
:107540009093DE068093DD06021B130B1093E0067A
:107550000093DF0680919E04882311F00E9418306A
:1075600080E4E1E1F7E0DF011D928A95E9F7BA894D
:10757000B1FF2DC08091880190E08170907022E071
:1075800030E0281B390B80E090E0ED89FE89AF895F
:10759000B88D2817390729F01182108211961C9294
:1075A0001E920196329612968430910591F71092B0
:1075B000E2061092E1061092E4061092E3061092A1
:1075C000E6061092E5061092E8061092E70686E8B5
:1075D00093E090930101809300019C012F5F3F4F46
:1075E00030930301209302019C012E5F3F4F3093A3
:1075F00005012093040103969093070180930601EF
:1076000027E1422E28E0522E97E9692E97E0792E45
:1076100087E5282E87E0382E19861D8689850E94E9
:107620000A0F7C01FC0180818150803108F0ADC2DD
:10763000838161E040E00E94D510D2019C918823B3
:10764000A1F4292F1C92F7019181892F8850823053
:1076500008F08AC287818E70843009F485C299301F
:1076600009F04BC000E01CEF4AC021E0911120E07E
:1076700081E0D2018C93D7011196EC913E2F3150CD
:10768000832F90E0DC01AA0FBB1FA753B94F0D91C8
:107690001C911197343160F0B9853B1748F4DC0137
:1076A000AA0FBB1FAA0FBB1FAF5EB84F0D911C9155
:1076B000D70117963C911797832F807381F0832F02
:1076C0008295837090E0019741E050E002C0440F42
:1076D000551F8A95E2F7CA015D85582B5D8736FFF5
:1076E0000EC0E53060F4F0E0EE0FFF1FE250FF4FF8
:1076F000C70108969183808302C000E010E0D701A3
:107700001796CC901797C6FC0BC018968C911897BB
:10771000882331F02AA30E94ED0E080F191F2AA119
:10772000F7018681882321F48581882309F458C1D3
:10773000D3016D917D918D919C911397222389F4B2
:1077400020E031E040E050E00E9488725095409582
:10775000309521953F4F4F4F5F4F4801820E931E4A
:107760005AC08C2D8E70843051F5D701EC91F0E029
:10777000EE0FFF1FE151F94F60817181882777FD7E
:107780008095982F20E034E640E050E00E9414728B
:10779000F3016083718382839383D70112962C91C6
:1077A0001297222361F0332727FD3095432F532F63
:1077B0000E948872F3012083318342835383D30173
:1077C0006D917D918D919C91139720E031E040E087
:1077D00050E00E94887250954095309521953F4F1A
:1077E0004F4F5F4F4801820E931E8114910499F010
:1077F000F701258197FE22952F7030E044E650E096
:10780000249FC001259F900D349F900D1124D1011C
:1078100011969C938E93F10180819181009799F04C
:1078200020919E04222319F0019791838083D10136
:107830008D919C911197009731F0F30160817181D6
:1078400082819381B7C08114910409F4C9C0D70122
:1078500016968C911697882309F4B4C080919E04E3
:10786000882309F476C012962C9112972223B1F046
:10787000332727FD309537FF03C0309521953F4FC3
:10788000332727FD3095432F532F60E070E080E2CF
:1078900093E00E94887259016A0106C0A12CB12CA4
:1078A000F0E2CF2EF3E0DF2EF701868118141904E1
:1078B000FCF48F7090E00097F1F144E650E0849F73
:1078C0009001859F300D949F300D1124442737FD82
:1078D0004095542FC601B5010E948872F301808142
:1078E0009181A281B381280F391F4A1F5B1F2CC0D1
:1078F00082958F7090E00097F1F044E650E0849F0D
:107900009001859F300D949F300D1124442737FD41
:107910004095542FC601B5010E94887259016A0131
:10792000D3012D913D914D915C9113972A193B09FB
:107930004C095D0909C09801442737FD4095542F33
:10794000542F432F322F2227F30120833183428388
:107950005383D3016D917D918D919C9120E031E015
:1079600040E050E00E948872C801AA2797FDA095C8
:10797000BA2F1814190434F482179307A407B50713
:1079800034F012C0281739074A075B076CF4222726
:1079900017FD2095322F322F212F102F0027F301B2
:1079A0000083118322833383D3016D917D918D9167
:1079B0009C91139720E031E040E050E00E948872F3
:1079C00089010EC0C801AA2797FDA095BA2FBA2F2A
:1079D000A92F982F8827F30180839183A283B383F3
:1079E000D70114966C911497633061F1643028F4D8
:1079F000613051F06230A0F444C0653069F1653007
:107A000038F1663081F52BC0F7018181893029F486
:107A100017FD35C0005012400EC017FF32C02CC0F9
:107A2000D70111968C911197893041F410161106E7
:107A300004F100501E4F000F111F23C01016110635
:107A4000DCF01FC017FF1DC0109501951F4F19C016
:107A50001016110674F010C017FF0EC010C01016DB
:107A600011063CF00CC06750C8010E94DA328C014C
:107A700008C000E014E005C000E010E002C000E033
:107A80001CEFF701878180FD13C0E181EE2381F0B7
:107A9000E53070F4F0E03197EE0FFF1F21E030E0A9
:107AA0002C0F3D1FE20FF31F80819181080F191FDA
:107AB000B801882777FD8095982FD70112962C91D1
:107AC0001297332727FD3095432F532F0E941472AE
:107AD000F701008110E001501040278126952770A2
:107AE000213071F0F801EE0FFF1FEE0FFF1F223063
:107AF00069F5EF5EF84F608371838283938334C0AE
:107B000024E630E040E050E00E948872E22EC32E6E
:107B1000DA01000F111F000F111F0F5E184FF8013F
:107B200020813181428153816E2D7C2DCD010E94B7
:107B3000147220E034E040E050E00E948872D801E6
:107B40002D933D934D935C9313970EC0EF5EF84FCA
:107B50002081318142815381260F371F481F591FD1
:107B60002083318342835383B985BF5FB9870894EB
:107B7000411C511CE4E0F0E06E0E7F1E22E030E07C
:107B8000220E331EB03209F049CD0E94020F8C0143
:107B9000ED84E0FE05C0882319F48EE10E94E86DB3
:107BA000E1FE0BC0C80190708034910519F0883453
:107BB000910519F48FE10E94E86DE2FE0DC010708E
:107BC0000038110531F00838110519F00039110598
:107BD00019F480E20E94E86DBFEF4B2EB4E05B2EFB
:107BE0003F8D28A1832F922F9A87898722243324BF
:107BF000598A488AAB85BC85ED90FD900D911C910A
:107C0000C801B70124E630E040E050E00E948872ED
:107C1000EB85FC852083318342835383A889B9890E
:107C20002D933D93B98BA88BEE85FF85E35AFE4FCC
:107C300080819181EE85FF85E55AFE4F2081BAE073
:107C40002B0260011124E8EEF3E0CE0EDF1EEE857C
:107C5000FF85E65AFE4F20812B0250011124A8E136
:107C60004A2EACEF5A2EA40CB51C96014C2D232F96
:107C70008C159D0514F4482F292F842E922E8A14DA
:107C80009B040CF44501E114F1040105110569F1AF
:107C90009401442737FD4095542F1E141F041006ED
:107CA000110654F4B601882777FD8095982F621B42
:107CB000730B840B950B0DC0C501AA2797FDA095EA
:107CC000BA2F29013A01481A590A6A0A7B0AC301E4
:107CD000B201A80197010E94147220EA36E841E03F
:107CE00050E00E94887279018A01C4010E94581AEA
:107CF0003C01882477FC8094982C6E0C7F1C801E9D
:107D0000911EC6010E94581A8C01C5010E94581A82
:107D1000222717FD2095322F06151705280539054E
:107D200014F438014901AA2797FDA095BA2F8401C0
:107D30007301681679068A069B0614F47C018D018E
:107D4000EE85FF85E45AFE4F8081882341F010952F
:107D50000095F094E094E11CF11C011D111DF4EA62
:107D6000CF2EF1E0DF2EC20CD31CF601E358FD4FFD
:107D70008081882389F060E040E00E94D51088234C
:107D800059F0F601E258FD4F80810E94ED0E7C0112
:107D90000027F7FC0095102FF894A985BA85ED927D
:107DA000FD92BA87A9877894EB85FC853496FC8789
:107DB000EB87E2E04E2E512C240C351C2E853F859E
:107DC0002B5F3F4F3F872E8730E22316310409F0A7
:107DD00011CF04C08F7009F09AC9C3C9A2960FB61B
:107DE000F894DEBF0FBECDBFCF91DF911F910F91F1
:107DF000FF90EF90DF90CF90BF90AF909F908F90CB
:107E00007F906F905F904F903F902F900895EF92EA
:107E1000FF920F931F93DF93CF93CDB7DEB7C0547C
:107E2000D0400FB6F894DEBF0FBECDBF8E010F5FFE
:107E30001F4FC80163E00E94A43581E2E82EF12CB7
:107E4000EC0EFD1EC70161E00E94A435E0E0F3E006
:107E5000418152816081D8012D913C91D7018D9152
:107E60009C911197662329F0B901681B790BCB010E
:107E700002C0821B930B840F951F73E0883E970707
:107E80002CF4ACEF89319A0724F005C088EE93E01A
:107E900002C088E19CEF9283818335960E5F1F4F6D
:107EA00062E070E0E60EF71E73E0E035F70781F65A
:107EB0008091880190E08170907022E030E0281B72
:107EC000390B80E090E02817390721F0FC01EA57D0
:107ED000FC4F1082019684309105A9F786E00E943C
:107EE0000E5881E00E94E86DC05CDF4F0FB6F89439
:107EF000DEBF0FBECDBFCF91DF911F910F91FF90DD
:107F0000EF9008952F923F924F925F926F927F92DF
:107F10008F929F92AF92BF92CF92DF92EF92FF9299
:107F20000F931F93DF93CF930F92CDB7DEB71091CE
:107F300086011F70813809F477C0823888F4833253
:107F4000F1F1843230F48032E1F0823209F07EC007
:107F500045C0813609F45DC0803809F077C01BC088
:107F60008438F9F0853838F4823809F44AC0833807
:107F700009F06CC040C08538E1F08F3B09F066C065
:107F800059C0153009F062C08091A20491E08927A0
:107F90008093A2044DC00E9437150E94761580E898
:107FA00005C082E691E30E94761584E80E9429626A
:107FB0004DC080E19BE40E94761585E8F7CF812FC4
:107FC0008F5F80938601863010F01092860181E0E9
:107FD0000E940E5883E10E94E86D38C0112319F009
:107FE000812F815001C085E08093860181E00E944D
:107FF0000E5884E1F0CF8EE79AE10E94661583E87F
:10800000D5CF0E945F6F81E192E70E94661582E8FA
:10801000CDCF80914706823021F483E080934706DC
:1080200007C0153099F402C00E94CD300E94B515EA
:1080300087E1D1CF81E00E94296283E00E9429621A
:1080400082E00E94296281E0809337088091B80124
:1080500060E040E00E94D510882331F0809137081D
:10806000882311F40E94073F8091B80160E040E04E
:108070000E94D5108093370880918601803108F0E6
:10808000D3C09091080180917301981710F496E085
:1080900001C094E0B4EAEB2EB1E0FB2E0AE0D70178
:1080A0004D917D01802F60E024E099830E942A5D3C
:1080B000055F9981083799F7492F406884E260E1AC
:1080C0000E94A50F84E268E146E50E94E95D809187
:1080D0004706882399F0823011F406E001C004E0DD
:1080E00040914806509149068EE560E1202F0E949C
:1080F000260F83E368E140E00E944A104091B601F8
:1081000083E04802A00111244C5D574F84E260E1F6
:1081100023E000E00E94ED5D8091B5018F7031F0A9
:1081200089E360E140E258E00E944C5EAEE0EA2E56
:10813000A1E0FA2EF0E0CF2EF1E0DF2E66247724C6
:10814000EFE19E2EF70101917F01D601ED91FD91A6
:108150006D01808187FD8D5F85958595843E0CF44A
:1081600084EEA82E8D3114F07CE1A72E862D81504F
:108170008230F8F4802F64E046E30E94CE5E2091C6
:10818000880130E02625372520FD04C08091B50107
:108190008F7061F4802F81506EE143E00E94CE5ECB
:1081A000802F8F5F6EE143E00E94CE5E992D9A1979
:1081B00014C0802F8B516BE346E30E94CA5E802E71
:1081C0008A94882D6AE343E00E94CA5E882D6CE39E
:1081D00043E00E94CA5E0A0D9BE36DEF862E800E7F
:1081E0005DEFA52EA90E882D6A2D47E099830E9488
:1081F000CE5E9981692F6D5F882D47E00E94CA5E2F
:10820000802F8D5F6A2D47E00E94CE5E882D6A2DFB
:1082100047E00E94CA5E0894611C711CB4E06B16B2
:10822000710409F08FCF27C080E060E044EA51E09C
:108230002AE001E10E94ED5D9091080180917301B7
:10824000981710F442E001C040E084E560E00E942D
:10825000A50F80914706882371F0823011F402E067
:1082600001C000E040914806509149068FE660E069
:10827000202F0E94260F123008F085C045E2E42E20
:1082800045E0F42E00E039E1A32EB12C2BE1922E33
:1082900090E2692E712C80E8482E512CF701219034
:1082A00031907F01113011F1802F8370899DC02C96
:1082B0001124D02ED694D694DD0CDD0CDD0CF8E222
:1082C000DF0EC101B3010E9453729B01C101B201D3
:1082D0000E945372AB01421B530B420D531D8C2D58
:1082E0008F5D6D2D20E20E94606048C0043018F45C
:1082F000B2E2CB2E02C0AEE5CA2E802F8370D82EFC
:10830000DD0CDD0CD80E26E2D20EC10137FE04C012
:1083100088279927821993098A9DA0018B9D500D6A
:108320009A9D500D112440505E4F452F550F550B0F
:1083300045954595842E4A3114F0E9E18E2E8C2D19
:1083400089516D2D43E325E50E949C5E6D2D6250A1
:108350008C2D45E00E94CE5E1214130414F4C394D5
:1083600001C0C8186D2D6F5F8C2D482D0E94CA5E0C
:108370006D2D61508C2D482D0E94CA5E0F5F083014
:1083800009F08CCF8AC0153008F07DC00E94F5201E
:10839000123061F0812F880F810F880F8950912F43
:1083A0009150192F110F190F110F02C080E016E024
:1083B000C82E992787FD90952C01440C551C480E1A
:1083C000591E60E2D62EEE24FF2452E0852E912C19
:1083D000880E991E3C011AC00E9447105C018C2D2A
:1083E00060E040E00E94D510082FA501440D551D06
:1083F0008AE06D2D23E00E94ED5D0894E11CF11CE4
:1084000083E090E0480E591E98E0D90EC394C7014E
:10841000860D971D88169906FCF6812F992787FDF2
:1084200090952C01440C551C480E591E30E2D32E59
:10843000EE24FF2422E0822E912C880E991E3C010E
:108440001AC00E9447105C01812F60E040E00E944A
:10845000D510082FA501440D551D85E66D2D23E08F
:108460000E94ED5D0894E11CF11CA3E0B0E04A0E0F
:108470005B1EB8E0DB0E1F5FC701860D971D8816D7
:108480009906FCF60AC04091A4045091A5048CE31F
:1084900068E224E004E00E94260F0F90CF91DF9164
:1084A0001F910F91FF90EF90DF90CF90BF90AF9012
:1084B0009F908F907F906F905F904F903F902F9004
:1084C000089518161CF010921F050895282F3327C1
:1084D00027FD309590911F05291B3109462F50E04B
:1084E0004217530724F4861B80931F0508954650B6
:1084F00050402417350724F48A5F861B80931F059C
:108500000895AF92CF92DF92EF92FF920F931F9355
:10851000DF93CF930F92CDB7DEB7182F83EB9BE09D
:108520000E94771A81E998E0612F42E020E038E06C
:108530000AE07EEBE72E7BE0F72ECC2456E0A52E5A
:108540000E94EF1BF09091088F2D67E00E9461421E
:1085500088E068EA7BE00E94445E31E08F2D813044
:1085600009F030E08091BA0182958695877090E09D
:10857000AC01440F551F480F591F440F551F475753
:10858000544F84E568E026E0032F39830E94ED5DB7
:108590003981332399F06091BA01629566956770CD
:1085A000812F40E024E00E9419158295880F807E7B
:1085B0009091BA019F71982B9093BA0180E16EE778
:1085C0007BE00E94445E01E0EF2DE23009F000E024
:1085D00084E560E14091BB01202F0E94AB0F002396
:1085E00049F0812F6091BB0140E024E20E941915FF
:1085F0008093BB0188E163E77BE00E94445E409189
:10860000BC01FF2DF33011F421E401C020E484E526
:1086100068E150E00E9460608F2D833049F4812F23
:108620006091BC0140E024E60E9419158093BC01D2
:108630000091BA0106950695017080E265E67BE03F
:108640000E94445ECF2CDD24C7FCD09421E0E4E0FE
:10865000CE16D10409F020E084E560E2402F0E94AC
:10866000BA1BFF2DF43079F4812F602F40E021E018
:108670000E9419158170880F880F9091BA019B7F15
:10868000982B9093BA010091BA010695069506952C
:10869000017088E267E57BE00E94445E21E085E0AE
:1086A000C816D10409F020E084E568E2402F0E945A
:1086B000BA1BEF2DE53081F4812F602F40E021E0DF
:1086C0000E9419158170880F880F880F9091BA0148
:1086D000977F982B9093BA010091BA01029501708F
:1086E00080E369E47BE00E94445E21E0F6E0CF167F
:1086F000D10409F020E084E560E3402F0E94BA1B1A
:108700008F2D863079F4812F602F40E021E00E9488
:10871000191581708295807F9091BA019F7E982B68
:108720009093BA010F90CF91DF911F910F91FF901D
:10873000EF90DF90CF90AF900895AF92BF92CF921D
:10874000DF92EF92FF920F931F93DF93CF930F92DD
:10875000CDB7DEB7D82E82E19DE00E94771A83E97B
:1087600098E06D2D41E020E038E00AE0A8E1EA2E33
:10877000ADE0FA2EFBE0CF2EE0E1AE2E0E94EF1B23
:1087800010919308F0909408812F67E00E94614255
:108790002091710130E02F5F3F4F442737FD409516
:1087A000542F8AE260E001E172E0E72E0E942A5F26
:1087B0002D2D253451F0263418F4243401F511C040
:1087C0003D2D343671F03536D1F41130C1F4FF202F
:1087D000B1F080912005882391F080919408815018
:1087E0000CC0113061F44F2D493048F480912005C0
:1087F000882329F0809194088F5F8093940880915A
:108800001F05882309F088C088E06DE07DE00E94A4
:10881000445E113031F481E090E020912005222364
:1088200011F080E090E0082F00618CE368E044EAFA
:1088300051E02AE00E94ED5D80912005882359F4E3
:108840008091230587FF07C081E080932005109267
:1088500023051092940880912005882381F02091AF
:108860002305332727FD30958F2D90E0821793073E
:1088700034F41092200510922305109294081130C0
:1088800009F04DC080912005882309F448C08091EB
:10889000940890912305891B8093940887FF02C058
:1088A00010929408809194088A301CF089E080939B
:1088B000940810922305AF2CBB24F501EC55FE4F14
:1088C00080810E94F92D682F20919C0430919D0495
:1088D0002115310549F47D2D723631F0733621F0C2
:1088E000723411F0733431F48D2D40E021E40E9494
:1088F0001915682F862F0E94092E482FF501EC5577
:10890000FE4F80838F2D880F8F0D880F845C68E069
:1089100021E00E942A5D03C098E0E92E02C080E1B8
:10892000E82E80911F05823008F084C08E2D67E00C
:108930007DE00E94445E4091B1015091B20112303D
:1089400099F4FF2039F480912005882309F01AC496
:1089500021E019C48F2D813039F4809120058823BE
:1089600029F020E002E004C020E00DC420E001E096
:1089700087E46E2D0E94260F123009F059C08091B5
:108980002005882339F480919C0490919D040097E0
:1089900009F44EC0FF2029F09F2D913009F048C006
:1089A00022C08091B1019091B2010CE3A02EB12CB4
:1089B000B5010E943F728D2D40E02BE30E941915F6
:1089C0002CE3482F4203900111248091B101909132
:1089D000B201B5010E943F72280F391F3093B201D6
:1089E0002093B10125C08091B1019091B2016CE357
:1089F00070E00E943F72082F0E5F8D2D602F41E0C6
:108A00002EE30E941915081B602F772767FD7095CC
:108A10002091B1013091B201261B370B3093B20186
:108A20002093B10137FF04C01092B2011092B1013E
:108A300068E0E60E80911F058330F8F48E2D6FEF0D
:108A40007CE00E94445E01E0133009F000E08CE31A
:108A50006E2D402F0E944A10002349F08D2D609109
:108A6000AF0147EC29E30E9419158093AF0178E02C
:108A7000E70E8E2D893308F088C380911F0584305E
:108A8000C8F58E2D68EF7CE00E94445E91E01430C2
:108A900009F090E08091B001282F217030E0A90109
:108AA000440F551FA3E0220F331FAA95E1F7420F91
:108AB000531F4D51534F8CE36E2D2AE0092F99839C
:108AC0000E94ED5D9981992379F06091B001617008
:108AD0008D2D40E021E00E94191581709091B00128
:108AE0009E7F982B9093B00198E0E90EEE2DE9332C
:108AF00008F04BC380911F05853030F50091B5011A
:108B00000F708E2D6CED7CE00E94445E21E01530EC
:108B100009F020E08CE36E2D402F0E94AA1B153037
:108B200069F48D2D602F40E021E00E9419158F70AF
:108B30009091B501907F982B9093B501F8E0EF0EDE
:108B40002E2D293308F021C380911F05863040F572
:108B50000091B50102950F708E2D65ED7CE00E94AD
:108B6000445E21E0163009F020E08CE36E2D402FAA
:108B70000E94AA1B163071F48D2D602F40E021E079
:108B80000E9419158295807F9091B5019F70982B56
:108B90009093B50138E0E30E4E2D493308F0F5C24D
:108BA00080911F05873050F58E2D6CEC7CE00E9483
:108BB000445E91E0173009F090E04091B60186E004
:108BC0004802A00111244355534F8CE36E2D26E03B
:108BD000092F99830E94ED5D9981992349F08D2D8C
:108BE0006091B60140E024E00E9419158093B6011F
:108BF00068E0E60E7E2D793308F0C7C280911F052C
:108C0000883008F58E2D65EA7CE00E94445E01E024
:108C1000183009F000E086E36E2D4091B801202F56
:108C20000E94F70F002349F08D2D6091B8014AEEA4
:108C300026E10E9419158093B80188E0E80E9E2D68
:108C4000993308F0A2C280911F05893008F051C005
:108C50008E2D6CE97CE00E94445E9CE3AA24BB2438
:108C6000A5014C56534FFA1411F4193061F02091BC
:108C7000B90130E00A2C02C0359527950A94E2F735
:108C8000022F017001C002E0892F6E2D21E099832F
:108C90000E94ED5D0894A11CB11C99819A5F9636E3
:108CA000F9F6193001F5ED2DE03631F080919C0494
:108CB00090919D040097B9F08D2D0E942962109229
:108CC000200581E090E00F2C02C0880F991F0A94C4
:108CD000E2F72091B90128272093B90182E00E9490
:108CE0000E580E94AA58F8E0EF0E2E2D293308F0F6
:108CF0004CC280911F058A3008F0E3C08E2D6EE8CB
:108D00007CE00E94445E4091B30186E0489FA00150
:108D100011244B58534F1A3041F4FF2031F4809105
:108D20002005882321F002E003C000E001C001E03B
:108D300084E26E2D26E00E94ED5D8091B3018823D0
:108D400021F0833009F04DC009C086E66E2D40E762
:108D50005CE020E00E941D5E9CE308C082E76E2D6F
:108D60004DE65CE020E00E941D5E98E44091B40175
:108D7000552747FD5095440F551F440F551F485A1E
:108D8000534F1A3049F43F2D313031F48091200592
:108D9000882321F002E003C000E001C001E0892F38
:108DA0006E2D24E099830E94ED5D9981892F865D67
:108DB0004091B70192E34902A0011124445D5E4F46
:108DC0001A3049F46F2D623031F4909120059923C7
:108DD00021F022E003C020E001C021E06E2D0E94BE
:108DE00060608091B301813001F582E46E2D49E429
:108DF0005CE020E00E941D5E4091B401552747FDD4
:108E000050954F5F5F4F1A3049F47F2D713031F428
:108E100080912005882321F022E003C020E001C0DA
:108E200021E08EE76E2D0E9460601A3009F043C089
:108E300080912005882331F480919C0490919D04B9
:108E40000097C9F18F2D813079F0813018F0823090
:108E500091F522C08D2D6091B30140E023E00E9486
:108E600019158093B30127C08091B301882311F0B5
:108E7000833031F48D2D6091B4014EEF24E007C0B2
:108E80008130C9F48D2D6091B40140E02CE70E943F
:108E900019158093B4010FC08091B301882311F09C
:108EA000833049F48D2D6091B7014CEF2AE00E9488
:108EB00019158093B70198E0E90EEE2DE93308F01B
:108EC00064C180911F058B3008F07AC08091B30196
:108ED000882311F0833019F58E2D6AE37CE00E941F
:108EE000445E4091BD0185E04802A00111244F512C
:108EF0005F4F1B3011F421E201C020E28EE46E2DA1
:108F00000E9460601B3009F055C08D2D6091BD013D
:108F10004CEE24E10E9419158093BD014BC08130B5
:108F2000B9F401E01B3009F000E080E06E2D44E26E
:108F30005CE0202F0E941D5E0023E1F1FD2DF03842
:108F4000C9F581E080936D0E80E00E94E86D32C02B
:108F50008E2D6BE17CE00E94445E8091B40187FD20
:108F600003C083301CF403C080E001C082E0809322
:108F7000B40149E08402A00111244150544F1B3038
:108F800031F480912005882321F002E003C000E045
:108F900001C001E08CE36E2D29E00E94ED5D1B30E5
:108FA00049F48D2D6091B40140E022E00E94191532
:108FB0008093B40128E0E20E3E2D393308F0E5C07D
:108FC00080911F058C3098F58E2D65EF7BE00E9417
:108FD000445E31E01C3009F030E08091BA018170CC
:108FE00090E0AC01440F551F480F591F4251544F98
:108FF0008CE36E2D23E0032F39830E94ED5D3981D0
:10900000332379F06091BA0161708D2D40E021E049
:109010000E94191581709091BA019E7F982B9093B0
:10902000BA0148E0E40E6E2D693308F0AEC08091BD
:109030001F058D3040F50091BA01069501708E2D07
:1090400064EE7BE00E94445E21E01D3009F020E0E8
:109050008CE36E2D402F0E94AA1B1D3071F48D2DC4
:10906000602F40E021E00E9419158170880F9091D7
:10907000BA019D7F982B9093BA0178E0E70E8E2D70
:10908000893308F082C080911F058E3040F5009131
:10909000B001069501708E2D6CED7BE00E94445E60
:1090A00021E01E3009F020E08CE36E2D402F0E945D
:1090B000AA1B1E3071F48D2D602F40E021E00E942C
:1090C00019158170880F9091B0019D7F982B909316
:1090D000B00198E0E90EEE2DE93308F056C080911A
:1090E0001F058F3048F50091B00106950695017077
:1090F0008E2D63ED7BE00E94445E21E01F3009F07D
:1091000020E08CE36E2D402F0E94AA1B1F3079F4C3
:109110008D2D602F40E021E00E9419158170880F8D
:10912000880F9091B0019B7F982B9093B001F8E04D
:10913000EF0E2E2D293348F580911F05803128F53B
:1091400080912105882319F421E0103109F020E0F5
:1091500080E06E2D4FEB5BE00E941D5E1031A9F4A4
:109160003D2D303891F41092200589E1809321053E
:1091700080E80E94296210923B0680EE90E30E94F4
:10918000761503C022E000E0F3CB0F90CF91DF9182
:109190001F910F91FF90EF90DF90CF90BF90AF9015
:1091A00008956F927F928F929F92AF92BF92CF92CB
:1091B000DF92EF92FF920F931F93DF93CF930F9263
:1091C000CDB7DEB7B82E8DE59FE00E94771A89EA09
:1091D00098E06B2D47E020E038E00AE07DE6E72EDE
:1091E0007FE0F72ECC24C3945CE0A52E0E94EF1BF9
:1091F0008090A9088A94D090AA08882D66E00E94E1
:10920000614218E0CC24992487FC909490911F052A
:109210009C0D9C3009F44FC1E92EFF248E149F044D
:1092200039F480912005882329F022E0A22E04C081
:10923000AA2402C0AA24A39480E0612F4AE55FE03B
:1092400022E000E099830E94ED5D9981993010F051
:1092500048E301C041E3490F8CE0612F0E94E95DC2
:10926000F701EE0FFF1FEE0DFF1DE450FC4F408194
:1092700087E0489FA00111244950514FDD2011F093
:1092800000E001C00A2D88E1612F27E00E94ED5D1A
:10929000C701880F991F8E0D9F1D8C559E4FFC0195
:1092A000E85AFD4F2081253008F4F6C0FC01EA5A47
:1092B000FD4F283008F4F9C040819D2D9130D1F543
:1092C0003BC020E001C02A2D88E4612F0E94AB0F33
:1092D000F701EE0FFF1FEE0DFF1DE550FC4F408123
:1092E000552747FD5095ED2DE23011F020E001C0EB
:1092F0002A2D88E7612F0E94606000E035C020E0E1
:1093000001C02A2D88E4612F0E94F70FF701EE0FAC
:10931000FF1FEE0DFF1DE550FC4F4081FD2DF2308B
:1093200011F020E001C02A2D80E6612F0E94F70F86
:1093300001E01AC020E001C02A2D88E4612F0E94BC
:10934000AB0FF701EE0FFF1FEE0DFF1DE550FC4FB9
:1093500040818D2D823011F020E001C02A2D86E65B
:10936000612F0E94AB0F02E080912005882339F421
:1093700080919C0490919D04009709F486C0AA20D6
:1093800009F483C09D2D9130D1F1913020F09230BD
:1093900009F07BC046C03701660C771C6E0C7F1C41
:1093A000ECEFF3E06E0E7F1E8B2DF301608140E049
:1093B0002DE00E941915F3018083202F30E08530C5
:1093C00028F0883030F481E090E005C080E090E043
:1093D00002C082E090E02817390709F456C0C7019F
:1093E000880F991F8E0D9F1D8C559E4FFC01EA5AC8
:1093F000FD4F1082895A9D4FFC01108246C00130FA
:1094000041F0C701880F991FE80EF91E8AEF93E01B
:1094100031C03701660C771C6E0C7F1C8AEF93E01D
:109420001AC0013089F0C701880F991F0230F1F08E
:10943000E80EF91E8BEF93E0E80EF91E8B2DF70175
:10944000608143E82DE71DC03701660C771C6E0C68
:109450007F1C8BEF93E0680E791E8B2DF3016081EA
:109460004AEE26E10E941915F3010EC0E80EF91E1E
:109470008BEF93E0E80EF91E8B2DF701608140E041
:1094800024E20E941915F7018083C394185FFC2D14
:10949000F73009F0BBCE0FC08A5A9D4FFC014081C6
:1094A000FD2DF13009F00DCF0ECF40818D2D813093
:1094B00009F025CF26CF0F90CF91DF911F910F910B
:1094C000FF90EF90DF90CF90BF90AF909F908F90E4
:1094D0007F906F9008956F927F928F929F92AF923C
:1094E000BF92CF92DF92EF92FF920F931F93CF9391
:1094F000DF93982E8FE69FE00E94771A8BEA98E020
:10950000692D48E020E038E00AE01FE7E12E1FE087
:10951000F12ECC24C394B0E1AB2E0E94EF1B6090DF
:10952000AB086A948090AC08862D66E00E94614288
:10953000A8E0FA2EDD24772467FC709440911F0583
:109540004D0D403109F45DC0A42EBB244F5F80E077
:109550006F2D20E00E94D70FEE24E501CC0FDD1F18
:10956000CE5DDB4F8501000F111F0F5D1B4F6A148D
:109570007B0471F48E1461F480912005882359F4E2
:1095800080919C0490919D04009739F421E001C0E2
:1095900020E0CC2405C022E001C021E0CC24C3940B
:1095A000EE2091F48EE16F2DF80140810E94F70FBB
:1095B000CC20D9F0892DF80160814AEE26E10E9485
:1095C0001915F801808311C04881552747FD509532
:1095D00080E66F2D0E946060CC2039F0892D688173
:1095E00043E82DE70E9419158883E394FE2DF3309C
:1095F00009F0BDCFD39488E0F80EED2DE73009F0E7
:109600009DCFDF91CF911F910F91FF90EF90DF9051
:10961000CF90BF90AF909F908F907F906F90089564
:10962000AF92BF92CF92DF92EF92FF920F931F9370
:10963000DF93CF9300D0CDB7DEB7182F8091930181
:10964000813019F048E1C42E02C03AE1C32E2BEF5D
:10965000B22EBC0C8EE49AE00E94771A88E498E05F
:10966000612F40E024E138E006E0EC2C0E94781FF6
:10967000F0904808D09049088F2D67E00E94614221
:1096800060911F058C2D90E0462F50E09C012750E3
:1096900030404217530761F42F2D30E0049728170C
:1096A000390714F48FEF01C081E0680F60931F0544
:1096B000113629F1123678F4143409F448C01534FF
:1096C00020F4123408F46AC063C0153419F110365E
:1096D00009F064C009C0143608F45AC01436B9F150
:1096E000153609F05BC016C0FF2009F457C081E0B1
:1096F00090912005911180E0809320054FC08091CA
:109700002005882309F44AC01092200581E60E94B2
:10971000296244C02F2D213059F4DD2049F0809179
:109720002005882329F080914908815080934908B9
:109730002F2D30E08B2D992787FD9095281739071D
:1097400069F5DD2059F18091490881501EC03F2DF7
:10975000313061F48D2D893048F4809120058823C3
:1097600029F0809149088F5F809349082F2D30E0C0
:109770008B2D992787FD90952817390779F49D2D12
:10978000973060F4809149088F5F8093490806C044
:1097900080912005882311F41092490880911F05BB
:1097A000882309F089C088E063E47AE00E94445E7F
:1097B000EF2DE13031F481E090E02091200522236B
:1097C00011F080E090E0082F006182E468E045E954
:1097D00051E02AE00E94ED5D80912005882359F434
:1097E0008091230587FF07C081E0809320051092B8
:1097F00023051092490880912005882381F020914B
:109800002305332727FD30958D2D90E08217930790
:1098100034F4109220051092230510924908FF2D70
:10982000F13009F04CC080912005882309F447C02D
:109830008091490890912305891B8093490887FFEF
:1098400002C010924908809149088A301CF089E0D2
:109850008093490810922305AD2CBB24F501EB56EB
:10986000FE4F80810E94F92D682F20919C04309139
:109870009D042115310541F4123631F0133621F0E3
:10988000123411F0133431F4812F40E021E40E94AE
:109890002815682F862F0E94092E482FF501EB56B8
:1098A000FE4F80838D2D880F8D0D880F8E5B68E0B5
:1098B00021E00E942A5D03C098E0E92E02C080E109
:1098C000E82E80911F058230A0F5C0908701C694D4
:1098D000C694C69427E0C2228E2D6CE37AE00E94E3
:1098E000445E91E03F2D323009F090E046E08C2D4F
:1098F000849FA00111244F5E554F8CE56E2D26E00C
:10990000092F9A830E94ED5D9A81992381F0812F1E
:109910006C2D40E026E00E9428158770880F880F84
:10992000880F90918701977C982B9093870198E0FE
:10993000E90E80911F05833058F5C09093018E2D5C
:1099400066E07AE00E94445E91E0EF2DE33009F09A
:1099500090E046E0FC2DF49FA00111244750564FA3
:109960008CE56E2D26E0092F9A830E94ED5D9A8189
:10997000992341F0812F6C2D40E021E00E942815B1
:109980008093930128E0E20E3E2D393308F0FFC3A7
:1099900080919301813041F580911F05843030F52D
:1099A0008E2D6BEE79E00E94445E409191018F2DE7
:1099B000843011F421E401C020E486E66E2D50E0ED
:1099C0000E9460609F2D943049F4812F6091910135
:1099D00041E024E60E94281580939101E8E0EE0E14
:1099E000FE2DF93318F0D3C304E001C005E08091E7
:1099F00093018150823038F580911F05801710F552
:109A00008E2D6BED79E00E94445E40919201F0163C
:109A100011F421E401C020E486E66E2D50E00E949E
:109A20006060F01649F4812F6091920140E025E0DA
:109A30000E9428158093920128E0E20E3E2D3933D2
:109A400008F0A5C30F5F80911F05801720F58E2DAC
:109A500062ED79E00E94445E40917201F01611F4CB
:109A600021E401C020E486E66E2D50E00E94606093
:109A7000F01659F4812F609172014AE02DE20E94A4
:109A80002815809372010E94C06088E0E80E9E2D28
:109A9000993308F07CC3C02EC39480911F058C15A8
:109AA00008F58E2D62EC79E00E94445E40917301CE
:109AB000FC1411F421E401C020E486E66E2D0E941E
:109AC000910FFC1449F4812F6091730148E228E75B
:109AD0000E94281580937301E8E0EE0EFE2DF93305
:109AE00008F055C3C39480911F058C1560F58E2D29
:109AF00061EB79E00E94445E40918901552747FD62
:109B00005095465F5F4FFC1411F421E401C020E43E
:109B100086E66E2D0E9460608091A90D6E2D4DE647
:109B20000E94E95DFC1449F4812F6091890146EFA0
:109B30002EE60E9428158093890128E0E20E3E2D32
:109B4000393308F024C3C39480911F058C1550F558
:109B50008E2D66EA79E00E94445E91E0FC1090E070
:109B600040918B0150E0440F551F440F551F47563D
:109B7000564F86E66E2D24E0092F9A830E94ED5DF4
:109B80009A81992349F0812F60918B0140E022E076
:109B90000E94281580938B0188E0E80E9E2D993352
:109BA00008F0F5C2C39480911F058C15C8F480910C
:109BB0008A01817021E0FC1020E06E2D48E859E018
:109BC000012F0E94132E817090918A019E7F982B05
:109BD00090938A01E8E0EE0EFE2DF93308F0D7C22B
:109BE000C39480911F058C15D8F480918A018695C5
:109BF000817021E0FC1020E06E2D4CE759E0012F30
:109C00000E94132E8170880F90918A019D7F982B5E
:109C100090938A0128E0E20E3E2D393308F0B7C256
:109C2000C39480911F058C15E8F480918A01869574
:109C30008695817021E0FC1020E06E2D4DE659E004
:109C4000012F0E94132E8170880F880F90918A0136
:109C50009B7F982B90938A0188E0E80E9E2D993384
:109C600008F095C2C39480911F058C15F8F480917B
:109C70008A01869586958695817021E0FC1020E00A
:109C80006E2D4FE559E0012F0E94132E8170880F31
:109C9000880F880F90918A01977F982B90938A0163
:109CA000E8E0EE0EFE2DF93308F071C2C394809106
:109CB0001F058C1500F58E2D62E579E00E94445E4B
:109CC00001E0FC1000E080E66E2D40917501202F30
:109CD0000E94F70F002349F0812F609175014AEE31
:109CE00026E10E9428158093750128E0E20E3E2DA2
:109CF000393308F04CC2C394BB2480911F058C15E6
:109D000008F048C0BB2019F462E479E002C062E3C5
:109D100079E08E2D0E94445EBB2019F4A0908C0146
:109D200002C0A0909401AA20A9F08A2D95E0899FF5
:109D3000A0011124FC1411F421E401C020E486E602
:109D40006E2D0E9460608091A90D6E2D43E70E94E8
:109D5000E95D0AC001E0FC1000E086E66E2D4EE2EF
:109D600059E023E00E94ED5DFC1439F4812F6A2D47
:109D700040E028E70E942815A82EBB2019F4A092E5
:109D80008C0102C0A0929401E8E0EE0EFE2DF933A2
:109D900008F0FDC1C394B3942B2D223009F0ADCF50
:109DA00080911F058C15F8F480918A0182958F703F
:109DB0008095817021E0FC1020E06E2D40E259E09A
:109DC000012F0E94132E809581708295807F909143
:109DD0008A019F7E982B90938A0138E0E30E8E2DA6
:109DE000893308F0D4C1C39480911F058C15F8F411
:109DF0008091900182958F708095817021E0FC1098
:109E000020E06E2D44E159E0012F0E94132E809531
:109E100081708295807F909190019F7E982B909386
:109E2000900198E0E90EEE2DE93308F0B0C1C3943B
:109E300080911F058C15D8F48091870180958170E1
:109E400021E0FC1020E06E2D43E059E0012F0E943C
:109E5000132E80958170909187019E7F982B90930F
:109E60008701F8E0EF0E2E2D293308F090C1C3943E
:109E700080911F058C15E8F4809187018695809567
:109E8000817021E0FC1020E06E2D44EF58E0012F9E
:109E90000E94132E80958170880F909187019D7F7D
:109EA000982B9093870138E0E30E8E2D893308F0CC
:109EB0006EC1C39480911F058C1508F086C08E2D4D
:109EC00069EE78E00E94445E92E4AA24BB24A501D6
:109ED0004052574FE0919F01F0E00A2C02C0F595E7
:109EE000E7950A94E2F7E170F070892F6E2D21E07A
:109EF0000E2F9A830E94ED5D0894A11CB11C9A81DB
:109F00009A5F923721F7FC1409F059C080914908F3
:109F100090912305891B8093490887FF02C0109206
:109F20004908809149088A301CF089E080934908EB
:109F3000109223058D2D880F8D0D880F4D2D50E02B
:109F40004952574F8E5B6E2D21E002E00E94ED5D7D
:109F5000103631F080919C0490919D04009779F126
:109F6000812F0E9429621092200581E090E002C0BA
:109F7000880F991FDA94E2F790919F0198279093A8
:109F80009F01803151F0803271F0883099F493FF55
:109F900002C09F7C0DC098600BC094FF02C0977DEB
:109FA00007C0906105C095FF02C0977E01C0906216
:109FB00090939F0181E00E940E580E94AA5898E059
:109FC000E90EEE2DE93308F0E2C0C39480911F053D
:109FD0008C15F8F48091870186958695809581701F
:109FE00021E0FC1020E06E2D48EC58E0012F0E948B
:109FF000132E80958170880F880F909187019B7F29
:10A00000982B90938701F8E0EF0E2E2D293308F05E
:10A01000BEC0C39480911F058C1500F590918701F7
:10A02000991F9927991F81E0891B21E0FC1020E0EE
:10A030006E2D4AEB58E0012F0E94132E80958795D4
:10A0400088278795909187019F77982B9093870118
:10A0500038E0E30E8E2D893308F099C0C3948091C7
:10A060001F058C1508F580918A0182958695877069
:10A070008095817021E0FC1020E06E2D40EB58E0CF
:10A08000012F0E94132E809581708295880F807E0B
:10A0900090918A019F7D982B90938A0198E0E90E18
:10A0A000EE2DE93308F073C0C39480911F058C1521
:10A0B00018F580918A0182958695869583708095A2
:10A0C000817021E0FC1020E06E2D48EA58E0012F5D
:10A0D0000E94132E809581708295880F880F807C56
:10A0E00090918A019F7B982B90938A01F8E0EF0E64
:10A0F0002E2D293308F04BC0C39480911F058C1579
:10A1000008F045C086E06E2D43EA58E00E944C5EA0
:10A110003E2D383390F434E290E0832F6E2D45EBE2
:10A1200057E0292F00E039839A830E94CB5C9A8103
:10A130009F5F3981385E943081F788E0E80E9E2D6C
:10A14000993328F5DD24D394FC10DD244091880157
:10A150004F5C82E16E2D2D2D0E942A5D94E200E07D
:10A160000F5F892F6E2D402F20E09A830E94AB0F46
:10A170009A81985E0430A1F7DD2049F0812F60912B
:10A18000880140E023E00E942815809388010F9009
:10A190000F90CF91DF911F910F91FF90EF90DF9083
:10A1A000CF90BF90AF9008958F929F92AF92BF9241
:10A1B000CF92DF92EF92FF920F931F93DF93CF9393
:10A1C0000F92CDB7DEB7C82E88EA9FE00E94771ABB
:10A1D0008DEA98E06C2D49E020E038E00AE0FAE0F2
:10A1E000EF2E0E94781F1091AD081150812F66E06C
:10A1F0000E9461422C2D203899F480E80E94296247
:10A2000089E180932105193019F40E94E86205C0A4
:10A21000183018F4812F0E945A6381E00E94E86D83
:10A22000DD24E8E0FE2EA12EBB24A7FCB094809193
:10A230001F058D0D883081F1882E992494012F5FA0
:10A240003F4F442737FD4095542FA814B90411F40B
:10A2500001E101C000E182E16F2D72E0E72E0E9472
:10A260002A5FF401EE0FFF1FE45DF54E8591949196
:10A27000AC0180912105882321F421E0A814B904C0
:10A2800009F020E088E16F2D0E941D5E38E0F30E9A
:10A29000D3948D2D873059F6EF2DE93308F04FC058
:10A2A00080912105882321F4DD24D394183009F00E
:10A2B000DD2486E06F2D4AE95FE00E944C5E9AE55E
:10A2C00056E0A52EB12CE0918D01F0E0E85FFA4F49
:10A2D000449150E00A2C02C0559547950A94E2F744
:10A2E000437050704B56504F892F6F2D21E00D2D2C
:10A2F00099830E94ED5D2EEF3FEFA20EB31E998170
:10A300009A5F923701F7DD2049F08C2D60918D0125
:10A3100040E027E10E94281580938D016F2D685F32
:10A32000693368F480912105882319F421E01930FC
:10A3300009F020E086E041E85FE00E941D5E0F909A
:10A34000CF91DF911F910F91FF90EF90DF90CF9011
:10A35000BF90AF909F908F9008954F925F926F92B1
:10A360007F928F929F92BF92CF92DF92EF92FF9255
:10A370000F931F93DF93CF9300D0CDB7DEB7182F85
:10A3800086EE9FE00E94771A81EC98E0612F46E00C
:10A3900020E038E00AE050E1E52E0E94781F60904E
:10A3A000C1086A94862D66E00E946142103611F061
:10A3B000143641F467FC06C06092A6088AE493E371
:10A3C0000E947615CC24DD24EE24E39418E0F12ECF
:10A3D000772467FC709430911F053C0DBB24B39427
:10A3E000383028F4BB248E2D883028F074C09E2D80
:10A3F000973008F070C0032F10E091E060167106EE
:10A4000009F090E0DD2019F0DD24D39401C0D92EAD
:10A4100080E06F2D43EE5FE0292F3A8399830E94FD
:10A420001D5E3A819981393010F482E101C087E1E3
:10A43000A8014F5F5F4F6F2D292F0E946060BB20E6
:10A4400079F0085010402801B3E0440C551CBA952F
:10A45000E1F7400E511EE2EBF3E04E0E5F1E0BC023
:10A460002801440C551C440C551C400E511E8AE812
:10A4700093E0480E591E42010AE2F40141914F0156
:10A48000552747FD5095802F6F2D20E00E9460607A
:10A490000B5E033991F7F8E0FF0EE394BB20B1F0B7
:10A4A00085E090E0480E591E0AE2F20141912F0129
:10A4B000552747FD5095802F6F2D20E00E9460604A
:10A4C0000B5E0E3791F7F8E0FF0EE394C3948C2DEA
:10A4D000873009F080CFDD2029F480911F058F5F40
:10A4E00080931F050F900F90CF91DF911F910F91D7
:10A4F000FF90EF90DF90CF90BF909F908F907F90D4
:10A500006F905F904F900895AF92BF92CF92DF927D
:10A51000EF92FF920F931F93CF93DF93F82E87EA6A
:10A5200098E06F2D4DE00E94E92080919F088823DC
:10A5300019F08BEE9EE002C081EE9EE00E94771A39
:10A54000182F8091A0080E940A0FEC01812F8A5FCA
:10A5500060E0488120E00E94D70FA090A7088A2DD4
:10A5600066E00E94614218E0EE24BB24A7FCB09490
:10A5700020911F052E0D822F90E0DD24D394A81684
:10A58000B90609F0DD24263009F4FAC0273090F42A
:10A59000223009F457C0233030F4222309F121304E
:10A5A00009F0E8C134C0243009F499C0253008F01E
:10A5B000BAC069C02A3009F46BC12B3038F4283096
:10A5C00009F420C1293008F044C1F1C02C3009F44D
:10A5D0009CC12C3008F47AC12D3009F0CBC1B2C136
:10A5E0008CE0612F4AED5EE00E944C5E84E5612FB5
:10A5F00049812D2D0E94AB0FDD2009F4BBC18F2DA9
:10A60000698141E024E20E9419158983B3C18CE07D
:10A61000612F43ED5EE00E944C5E4A81552747FD65
:10A6200050952D2D206484E5612F0E946060DD200F
:10A6300009F4A0C18F2D6A8143E82DE70E94191506
:10A640008A8398C18F8186FF03C049EC5EE002C017
:10A6500042EC5EE08CE0612F0E944C5E48855527FD
:10A6600047FD50952D2D206484E5612F0E94606088
:10A67000DD2009F47FC18F2D688543E82DE70E9416
:10A680001915888777C1CF80C294C694C694E3E039
:10A69000CE2281E0C8228CE0612F47EB5EE00E9471
:10A6A0004C5E43E09C2D949FA00111244055514FD6
:10A6B00084E5612F23E00D2D0E94ED5DDD2009F47E
:10A6C00059C18F2D6C2D40E021E00E941915817039
:10A6D0008295880F880F807C9F819F7B90C08CE043
:10A6E000612F4BEA5EE00E944C5E8F81817090E0AA
:10A6F000AC01440F551F480F591F4C55514F84E56D
:10A70000612F23E00D2D0E94ED5DDD2009F432C1A3
:10A710006F8161708F2D40E021E00E9419158170DA
:10A720009F819E7F6CC08CE0612F4DE95EE020E050
:10A730000E941D5E4C8183E0489FA00111244F5E62
:10A740005F4E84E5612F23E00D2D0E94ED5DDD203D
:10A7500009F410C18F2D6C8140E026E10E9419158B
:10A760008C83873008F406C19F2D903609F002C112
:10A7700087508093A6088AE493E30E947615FAC076
:10A780008CE0612F46E95EE00E944C5E8EE4612F12
:10A790004B812D2D0E94F70FDD2009F4EBC08F2D8A
:10A7A0006B814AEE26E10E9419158B83E3C08CE091
:10A7B000612F4EE85EE00E944C5E0F8102950370AF
:10A7C00049F02D2D206484E5612F402F50E00E9438
:10A7D000606007C084E5612F4AE85EE02D2D0E948D
:10A7E0001D5EDD2009F4C6C08F2D602F40E023E000
:10A7F0000E94191583708295807F9F819F7C982B82
:10A800009F83B8C08CE0612F43E85EE00E944C5EFD
:10A810004F814695477050E063E0440F551F6A959D
:10A82000E1F74659514F84E5612F28E00D2D0E9434
:10A83000ED5DDD2009F49EC06F81669567708F2DF8
:10A8400040E022E00E9419158770880F9F81917F58
:10A85000D6CF8CE0612F4FE55EE00E944C5E4D81CB
:10A8600042954F7080E6612F50E02D2D0E94606070
:10A87000DD2009F47FC06D8162956F708F2D40E0FF
:10A880002FE00E9419158295807F9D819F701BC0CB
:10A890008CE0612F46E55EE00E944C5E4D814F707A
:10A8A00080E6612F50E02D2D0E946060DD2009F4CC
:10A8B00061C06D816F708F2D40E02FE00E941915EF
:10A8C0008F709D81907F982B9D8354C08CE0612F69
:10A8D0004BE45EE00E944C5E4E8142954F7080E6F4
:10A8E000612F50E02D2D0E946060DD2009F442C0F0
:10A8F0006E8162956F708F2D40E02FE00E941915D8
:10A900008295807F9E819F701AC08CE0612F42E407
:10A910005EE00E944C5E4E814F7080E6612F50E0F9
:10A920002D2D0E946060DD2029F16E816F708F2DCA
:10A9300040E02FE00E9419158F709E81907F982B28
:10A940009E8318C08CE0612F40E35EE02D2D0E94B5
:10A950001D5EDD2079F08F2D803861F40E94296220
:10A960008091A0080E94062381E00E94E86D80E0AB
:10A970000E944115E394185F9E2D973009F0F8CDA1
:10A98000DF91CF911F910F91FF90EF90DF90CF90CB
:10A99000BF90AF9008955F926F927F928F929F9237
:10A9A000AF92BF92CF92DF92EF92FF920F931F93DD
:10A9B000CF93DF93D82E8AEC9FE00E94771A8FEB1B
:10A9C00098E06D2D45E020E038E00AE071EDE72EDB
:10A9D0007FE0F72E51E1C52E11E1A12E0E94EF1B61
:10A9E000F090BF08FA948090C0088F2D66E00E9416
:10A9F00061428D2D803821F59F2D903108F5EF2D86
:10AA0000FF27E7FDF09580911F05E81BF109EE0F88
:10AA1000FF1FEB5DFA4FC081D1818F2D0E941A0F6D
:10AA2000FC01882069F48281882319F0D095C195B2
:10AA3000DF4FD483C38382E00E940E580E94AA583D
:10AA400018E09924552453946F2C772467FC709454
:10AA500000911F05090D003109F4E1C0802F0E940B
:10AA60001A0FEC018A816B817C81882319F0709523
:10AA700061957F4FA02EBB24F501EE0FFF1FEB5D0C
:10AA8000FA4F20813181261B370B2333310524F007
:10AA9000F501E155F74F08C09FEF2E3C39072CF424
:10AAA000F501E155F74F85258083402F4F5F80E00A
:10AAB000612F20E00E94D70FF501E155F74F80810B
:10AAC000882311F04FE701C04EE78BE4612F20E0AF
:10AAD0000E942A5DEE246A147B0471F48E1461F4E2
:10AAE00080912005882359F480919C0490919D04C5
:10AAF000009739F401E001C000E0CC2405C002E079
:10AB000001C001E0CC24C3948E2D823009F43FC0F3
:10AB1000833009F45DC08130C1F04B815C81202F0E
:10AB2000206280E3612F0E946060CC2009F46BC03A
:10AB30006B817C818D2D48E15CEF28EE33E002E0F3
:10AB40000E9455149C838B835EC0488144565527D0
:10AB500047FD509588E4612F202F0E946060CC2033
:10AB600009F451C06881645668838091BA0181FFFD
:10AB700004C08D2D43E82DE703C08D2D4CE924E65C
:10AB80000E941915888388818C5988833CC049812B
:10AB90004C59552747FD509586E6612F202F0E947E
:10ABA0006060CC2081F169816C5969838091BA0120
:10ABB00081FF04C08D2D43E82DE703C08D2D4CE9A6
:10ABC00024E60E94191589838981845689831BC0D4
:10ABD0008A8190E0AC01440F551F480F591F4D5317
:10ABE000504F8CE6612F23E00E94ED5DCC2059F0A0
:10ABF0008D2D6A8140E021E00E94191591E08823A3
:10AC000009F490E09A83E3949E2D943009F063CF89
:10AC10009394185F892D873009F01ACF1FC001E087
:10AC20009F2D903109F000E080912105882311F0DB
:10AC300020E001C0202F82E1612F42EB5FE00E9403
:10AC40001D5E002359F08D2D803841F489E18093F9
:10AC5000210580E80E9429620E94073FDF91CF9181
:10AC60001F910F91FF90EF90DF90CF90BF90AF902A
:10AC70009F908F907F906F905F900895F8942091AF
:10AC8000D70D3091D80D7894C9010895CF93DF93F3
:10AC9000C4E4D1E080E6FE0111928A95E9F78AE0EA
:10ACA0008093440189E1809372018AE58093730166
:10ACB00081E0809388012196FE0120E032E080E867
:10ACC00091E02193319395878487938F828F41E020
:10ACD000E335F407B1F785E991E063EB70E14AE011
:10ACE00050E00E94A97280E090E029913991820F92
:10ACF000931FE1E0CD35DE07C1F79093700180939B
:10AD00006F01DF91CF9108951F93CF93DF938AEC6A
:10AD100098E060E00E946A5A64E471E080E6FB011A
:10AD200011928A95E9F78AEC98E040E650E00E949B
:10AD3000F65A182FC5E9D1E088810E94F92D0E94AA
:10AD4000092E8993F1E0CF39DF07B1F780914401F3
:10AD50008A3028F4809181048160809381048AE0A4
:10AD6000809344011D3468F0E5E4F1E020E030E038
:10AD700081919191280F391F81E0ED35F807C1F7D6
:10AD800002C020E030E081E040916F0150917001FD
:10AD90004217530709F080E0DF91CF911F9108958A
:10ADA0001F93182FE4EAF1E025EA32E0DF01C90140
:10ADB0001D920197E9F7CF0168EA70E14AE050E09F
:10ADC0000E94A972812F90E001966AE070E00E94D3
:10ADD0005372605D6093A901805D8093AA018AE04F
:10ADE0008093AE0180E00E945A631F910895CF9234
:10ADF000DF92EF92FF920F931F93DF93CF930F9207
:10AE0000CDB7DEB76B01803160F5682F6F5F8AECDC
:10AE100098E049830E946A5A4981042F10E0C601D4
:10AE200060E270E050E00E94CA728AEC98E0B601DD
:10AE30004AE050E00E94F65A8A30910591F48AEC7B
:10AE400098E00E945C5AF601E00FF11F2AE030E022
:10AE500006C0B9010E943F72805D8293CB010097CA
:10AE6000C1F70F90CF91DF911F910F91FF90EF905D
:10AE7000DF90CF9008958F5F0E94ED5908951F9342
:10AE8000CF93DF93182F803168F5682F6F5F8AECBE
:10AE900098E00E946A5A64EA71E025EA32E0FB0118
:10AEA000C90111920197E9F78AEC98E045EA52E06E
:10AEB0000E94F65A8F3F910509F018F4812F0E94E5
:10AEC000D056C4EAD1E088810E94F92D0E94092E53
:10AED000899391E0CE3AD907B1F78AE08093AE0129
:10AEE0000E94B515DF91CF911F9108950F931F9385
:10AEF000DF93CF93CDB7DEB760970FB6F894DEBF80
:10AF00000FBECDBF682F6F5F062F0AC0102F1F5FC7
:10AF1000812F688B0E94ED596889882329F0012FC1
:10AF20000031A0F3003139F18AEC98E00E946A5AAE
:10AF3000602F6F5F83ED98E042E028E532E00E94E9
:10AF4000DC5B8E010F5F1F4F06C083ED98E0B801F8
:10AF50000E94575BA8958AEC98E0B8014FE050E05A
:10AF60000E94855A482F882381F783ED98E00E943C
:10AF7000055C81E001C080E060960FB6F894DEBF0A
:10AF80000FBECDBFCF91DF911F910F910895EF922A
:10AF90000F931F930E94D859882341F00E94435970
:10AFA00087FD04C00E948456882381F588E990E1DA
:10AFB00061E00E94241386E890E10E940B130E9436
:10AFC000B2590E9446568AEC98E060E041E024E4E1
:10AFD00031E000E610E078ECE72E0E94345C803629
:10AFE000910529F087E790E160E00E94241380E05A
:10AFF0000E94D0568AEC98E061E042E024EA31E019
:10B0000005EA12E058ECE52E0E94345C8091710153
:10B010000E943F571F910F91EF900895882359F098
:10B020009091E608982B9093E6080E94020F909367
:10B03000E8088093E7080895EF920F931F93CF934A
:10B04000DF931091E608112309F47EC0882309F0EC
:10B0500076C00E94020F2091E7083091E808AC0109
:10B06000421B530B4436510508F46EC068C081E0A2
:10B070008093E508812F90E0EC01C470D07012FF3E
:10B0800003C023E02093E5081092E60880FF1CC06F
:10B090008CED98E061E141E024E431E000E610E06D
:10B0A000F4E1EF2E0E94345C8036910511F480E0CB
:10B0B00020C08091E208823021F48091E60881600E
:10B0C00029C087E690E135C081FF36C08CED98E05D
:10B0D00061E142E024EA31E005EA12E0E4E1EE2E2B
:10B0E0000E94345C52E0853A950739F480917101F1
:10B0F0008F5F61E10E94FB591FC08091E20882309E
:10B10000A1F48091E608982F92609093E60820972A
:10B1100019F086608093E6080E94020F84569040E2
:10B120009093E8088093E70807C0209729F487E503
:10B1300090E160E00E9424131092E50805C0809120
:10B14000E508882309F493CFDF91CF911F910F91E8
:10B15000EF9008950AC081E00E941C5880916B0E08
:10B16000833019F4A89510926B0E8091E60888231D
:10B1700091F70895DF93CF930F92CDB7DEB7682F85
:10B1800070E084E0660F771F8A95E1F7CE010196A3
:10B1900041E050E00E94D17289810F90CF91DF9100
:10B1A0000895DF93CF930F92CDB7DEB76983682FF1
:10B1B00070E094E0660F771F9A95E1F7CE01019653
:10B1C00041E050E00E94FD600F90CF91DF91089523
:10B1D00089EE98E060E070E040E450E00E94FD609D
:10B1E00008958BEE98E062E070E041E050E00E944C
:10B1F000FD6008950F931F93182F082F04C0802F10
:10B200000E94BA58082F802F0E94BA588823B9F795
:10B21000802F6091EB080E94D1581093EB080E9498
:10B22000F1581F910F9108951F931091EB0811236E
:10B2300059F0812F0E94BA588093EB080E94F15870
:10B24000812F60E00E94D158812F1F910895F894BA
:10B250002091D70D3091D80D7894C9010895EF92BF
:10B26000FF92CF93DF938091EB08C0E0D0E003C062
:10B270002F960E94BA588823D9F7CE01DF91CF913B
:10B28000FF90EF900895CF92DF92EF92FF920F938D
:10B290001F93CF93DF9380E8E9E2F9E0DF011D928D
:10B2A0008A95E9F70DEE18E0C0E0D0E08C2FC431AC
:10B2B00039F4D090EB083BEEE32E38E0F32E0BC0D0
:10B2C0007E01EE0CFF1CEC0EFD1E2DEE38E0E20EB2
:10B2D000F31ED801DC9090E0C82EC3941DC08D2DC4
:10B2E00084508C3738F4ED2DF0E0E75DF64F808127
:10B2F000882361F0992329F0892F60E00E94D158BA
:10B300000DC0F70110820E94E85808C0C0828D2D40
:10B310000E94BA589D2DD82EDD2009F721960D5F89
:10B320001F4FC531D10511F604E0E02FF0E0E75DD5
:10B33000F64F8081882349F4802F6091EB080E94AA
:10B34000D1580093EB080E94F1580F5F003869F75D
:10B3500080E0DF91CF911F910F91FF90EF90DF90F0
:10B36000CF9008951F9380E4E9EEF8E0DF01982F75
:10B370001D929A95E9F794E09093E9088093EA0882
:10B3800080E18093EC0884E001C0812F182F1F5FBB
:10B39000612F0E94D1581038C1F78FE760E00E94FA
:10B3A000D15884E08093EB080E94E8581F910895DB
:10B3B00089EE98E060E070E040E450E00E94D172D5
:10B3C0008091E908843039F481E09091EA08903462
:10B3D00019F080E0089580E0089590E0FC01EE0F00
:10B3E000FF1FE80FF91FE751F74F81E09481992380
:10B3F00009F480E00895DF93CF9300D00F92CDB78A
:10B40000DEB790E0FC01EE0FFF1FE80FF91FDE0131
:10B410001196E351F74F23E001900D922150E1F78F
:10B4200070E0DC01AA0FBB1FA80FB91FFB01EE0FD4
:10B43000FF1FE60FF71FA351B74FE351F74F83E00C
:10B4400001900D928150E1F7FB01EE0FFF1FE60F17
:10B45000F71FE351F74FDE01119683E00D90019243
:10B460008150E1F70E94E8580F900F900F90CF9114
:10B47000DF910895DF93CF930F92CDB7DEB790E0C1
:10B480009C01220F331F280F391FF901E751F74F95
:10B4900084812351374F93E0D9011D929A95E9F7A2
:10B4A00089830E94E8588981882311F00E94FA5804
:10B4B0000F90CF91DF910895FC01808190E0FC0115
:10B4C000EE0FFF1FE80FF91FE251F74F91818081C6
:10B4D0009F700895FC0160831282118270E0CB019D
:10B4E000880F991F860F971FDC01A751B74F14963D
:10B4F0002C91149723831482158216828151974FC1
:10B50000FC01808182958F7008958F929F92AF92F7
:10B51000BF92CF92DF92EF92FF920F931F93DF9330
:10B52000CF930F92CDB7DEB78C015B01FC01808118
:10B5300090E0FC01EE0FFF1FE80FF91FE251F74FFB
:10B5400080812181922F9F70F80121813281821B9D
:10B55000930BE42EF52E8E159F0508F47C016701F0
:10B560004E010894811C911C25C0F801638166235B
:10B5700021F184818F5F848370E0B4E0660F771FD0
:10B58000BA95E1F7680F711DC40141E050E00E94D7
:10B59000D1728981F50181935F01F80184818F3037
:10B5A00030F0148283810E94BA58F8018383089492
:10B5B000C108D108C114D104C1F6F801818192817A
:10B5C0008E0D9F1D8C199D09928381838E2D8C1960
:10B5D0000F90CF91DF911F910F91FF90EF90DF902F
:10B5E000CF90BF90AF909F908F9008958F929F9231
:10B5F000AF92BF92DF92EF92FF920F931F93CF9380
:10B60000DF938C015B017A01C0E0D0E045E0842E3D
:10B61000912C880E991E3BC0F801858190E08F77B0
:10B620009070009741F4C801B40141E050E00E94DD
:10B63000855A813079F5F80145813FE7D32ED42230
:10B640002D2D30E0C7018C1B9D0B8217930710F442
:10B65000DE2CDC1AB5016C0F7D1F47FF08C0CB0143
:10B6600060E070E04D2D50E00E94CA720AC0C8012F
:10B670004D2D50E00E94855A8D1519F0C80FD11D2F
:10B6800009C0CD0DD11DF80185818D198583CE1599
:10B69000DF0510F2CE01DF91CF911F910F91FF9046
:10B6A000EF90DF90BF90AF909F908F9008959F9202
:10B6B000AF92BF92CF92DF92EF92FF920F931F93C0
:10B6C000CF93DF93EC018B01C42E8B81882389F407
:10B6D00089819A81009769F4E880FF240E941459B7
:10B6E0008B83F701EE0FFF1FEE0DFF1DE751F74FA4
:10B6F0008483DC2C6FE0962E44C0EF80F8840E9497
:10B70000020FE81AF90AF7FE02C082E004C08B813A
:10B71000882319F481E08E8337C09C819F3080F0AC
:10B720001C820E94BA58882339F4EB800E94145975
:10B73000682F8E2D0E94D1588B810E94BA588B831E
:10B740008B81882339F36C81992D961BED2C9D15E7
:10B7500008F4E92EAE2CBB2470E06F5F7F4F90E0C1
:10B7600054E0880F991F5A95E1F7680F791FC801B7
:10B77000A5010E94FD600A0D1B1D8C818E0D8C831E
:10B78000DE18DD2009F0B9CF2C2D30E02D1931095C
:10B7900089819A81820F931F9A8389838C2D8D19B9
:10B7A000DF91CF911F910F91FF90EF90DF90CF909D
:10B7B000BF90AF909F9008950F931F93CF93DF9307
:10B7C000EC01890168831A82198270E0CB01880F2D
:10B7D000991F860F971FFC01E751F74F24812B8398
:10B7E0001C821D821E82FC01E251F74F108242959D
:10B7F000407F41830E94020F080F191F18870F8393
:10B80000DF91CF911F910F9108951F93CF93DF93F5
:10B81000EC01888190E0FC01EE0FFF1FE80FF91F9B
:10B82000E251F74F898180839A819F708181807F67
:10B83000892B81838B81882389F00E94BA58182F25
:10B84000882361F08B8160E00E94D1580E94E85803
:10B85000112331F0812F0E94FA5802C010E0F6CF78
:10B86000DF91CF911F9108954F925F926F927F92D7
:10B870009F92AF92BF92CF92DF92EF92FF920F937F
:10B880001F93DF93CF930F92CDB7DEB75C012901F1
:10B8900068012E2D30E00E94DC5B1982720100E00D
:10B8A00010E081E03E010894611C711CF701919148
:10B8B0007F01992341F4882349F49081992349F425
:10B8C000992493941EC0882371F403C099249394FF
:10B8D00001C0992499819F3718F40C151D0561F555
:10B8E000882379F001C099248981882321F1806817
:10B8F0008983C501B30141E00E94575B8130D1F0DB
:10B9000025C089818823B9F0C501B30141E00E94B7
:10B91000575B8130D9F44981B801641B7109640D0A
:10B92000751DC5010E94575B9981891719F0981BF5
:10B9300099830CC01982892D99819F5F99830F5F2C
:10B940001F4FC016D10608F0B1CF05C089818F778F
:10B950006801C81AD108C5010E94055CC6010F9094
:10B96000CF91DF911F910F91FF90EF90DF90CF90DB
:10B97000BF90AF909F907F906F905F904F90089591
:10B9800080E094E0E9EAF9E0DF019C011D9221509A
:10B990003040E1F708950F931F93CF93DF93DA01BF
:10B9A0001196FA014491ED012196FD01A491B0E0B8
:10B9B000179613E0B595A7951A95E1F71A2FDE01B2
:10B9C0001196FE019491929FE0011124AC0FBD1FCE
:10B9D00000FD08C001FF08C09091D90D51E096FD0F
:10B9E00004C002C051E001C050E0669566956695BE
:10B9F00070E09B013695322F22273795279590E0EE
:10BA0000280F391F610F711D7695762F6627779560
:10BA10006795680F791F042F10E014C0E901C7551E
:10BA2000D64F80E090E008C0FD01E80FF91FE491D7
:10BA30005111E095E99301968417B0F3A00FB11F5F
:10BA400020583F4F2617370749F7DF91CF911F91B5
:10BA50000F910895FF920F931F93CF93DF93942F2D
:10BA600046313CF4440F490F440F22FFABC0440F52
:10BA7000A9C0482F4A5F092F112707FD109520FD07
:10BA800009C021FF0AC03091D90DFF24F39436FD7F
:10BA900005C003C0FF24F39401C0FF24669566959A
:10BAA000669570E07695762F662777956795680F8F
:10BAB000711DEB01C755D64F22FF4FC09E3209F0D2
:10BAC0004A5FC801809760E170E00E94537280EA8B
:10BAD00090E0689F9001699F300D789F300D112490
:10BAE000C801880F991F53E0000F111F5A95E1F705
:10BAF000800F911F280F391F2C593E4E85E0882357
:10BB000069F0F9019491E056FF4F54912F5F3F4F38
:10BB1000F9016491E056FF4F749104C060E050E079
:10BB200090E070E0FF2021F0909560955095709521
:10BB3000DE01AF57BF4FFDE0A93ABF0740F498833D
:10BB40006983FE01E058FF4F50837C932296815019
:10BB50008F3FC1F12F5F3F4FD2CF23FF0DC0FF209A
:10BB600011F08FEF01C080E06755764FFB018083B5
:10BB700021964F5F91E001C090E09801220F331FA2
:10BB8000220F331F200F311F2F5D3F4E85E0F9013B
:10BB90002F5F3F4FE491992311F0843039F0FDE09D
:10BBA000C93ADF0718F4F110E095E993815079F76D
:10BBB0005DE0C93AD50730F4FF2011F08FEF01C0E6
:10BBC00080E08883842FDF91CF911F910F91FF90A8
:10BBD000089520E00E942A5D0895CF92DF92EF92AF
:10BBE000FF920F931F93CF93DF93162FF22EF0E166
:10BBF000EF2EE022C42EE6016E01D52EE6010CC028
:10BC0000EE2011F0488102C0FE014491612F202FE7
:10BC10000E942A5DFA942196FF2091F7DF91CF913F
:10BC20001F910F91FF90EF90DF90CF9008950F93A9
:10BC300000E00E94ED5D0F910895CF92DF92FF9298
:10BC40000F931F93CF93DF93162F022FA0E1FA2EAD
:10BC5000F222C42EE6016E01D52EE601FF2011F07E
:10BC6000488102C0FE0144912196442329F0612FAE
:10BC7000202F0E942A5DF2CFDF91CF911F910F916B
:10BC8000FF90DF90CF900895982FAB0180E0692F4F
:10BC900020E00E941D5E089520E00E941D5E089530
:10BCA000EF92FF920F931F93DF93CF930F92CDB735
:10BCB000DEB7182F062F7A01982F9C5E95504E2DD7
:10BCC0004F704A301CF0495C28E002C0405D20E023
:10BCD000892F602F99830E942A5D9981911731F0F5
:10BCE000B4E0F694E794BA95E1F7E8CF0F90CF91DE
:10BCF000DF911F910F91FF90EF900895E62FE69549
:10BD0000E695E695F0E0F695FE2FEE27F795E79598
:10BD1000E80FF11DE755F64F8DE0E93AF80758F4C2
:10BD2000677081E090E002C0880F991F6A95E2F782
:10BD3000208128272083089547FF02C0840F419562
:10BD4000E62FE695E695E695F0E0F695FE2FEE27D0
:10BD5000F795E795E80FF11DE755F64F6770A1E0FD
:10BD6000B0E001C0AA0F6A95EAF711C08DE0E93A88
:10BD7000F80778F4822F90E09C013595279580FF95
:10BD800004C080818A2780832068415031964423F3
:10BD900069F708952FEF0E949C5E08950F931F93FB
:10BDA000CF93DF93C82FD0E0E62FE695E695E69592
:10BDB000F0E0F695FE2FEE27F795E795EC0FFD1FC7
:10BDC000E755F64F062F10E0242F332727FD309537
:10BDD000200F311FC90168E070E00E945372769510
:10BDE000762F6627779567956C0F7D1F6755764F81
:10BDF0000770107081E090E002C0880F991F0A95CB
:10BE0000E2F781959081892708C0E058FF4F8DE0C7
:10BE1000E93AF807D0F4808180958083E617F70728
:10BE2000A0F38DE0E93AF80780F4C90168E070E01A
:10BE30000E94537221E030E002C0220F331F8A9526
:10BE4000E2F72195808182278083DF91CF911F9136
:10BE50000F9108952F923F924F925F926F927F922F
:10BE60008F929F92AF92BF92CF92DF92EF92FF920A
:10BE70000F931F93DF93CF9300D00F92CDB7DEB710
:10BE8000182F662E59016A01F02E802F05FF04C07D
:10BE900004FF04C002E003C000E001C001E0E7FECF
:10BEA00004C0E1942224239401C02224D7FE0BC0B5
:10BEB000D094C094B094A094A11CB11CC11CD11CFE
:10BEC0004424439401C0442482FF06C09CE0909324
:10BED000A90D3AE0932E05C096E09093A90D25E0B8
:10BEE000922E86FF2FC04110190D28EEA21623E0D6
:10BEF000B20620E0C20620E0D20614F0190D06C0FA
:10BF000034E6A316B104C104D10414F0190D06C01F
:10BF10008AE0A816B104C104D1040CF0190D002365
:10BF200091F0023039F4E4E6AE16B104C104D10454
:10BF300054F4190DFAE0AF16B104C104D1041CF495
:10BF4000190D01C0191B8091A90D810F8093A90DB6
:10BF5000023011F420EFF20E5524539492E0792E22
:10BF600088242E2D332727FD3095862D8A5F8983DF
:10BF70003B832A8370C0C601B5012AE030E040E06F
:10BF800050E00E948872E62E80E3382E3E0C812F0E
:10BF9000662D432D2F2D0E942A5D0515D9F5F2FE41
:10BFA00023C08E2D8150833008F47394C601B501EF
:10BFB0002AE030E040E050E00E948872CA01B901F6
:10BFC0002AE030E040E050E00E948872623011F0D8
:10BFD0006430C1F4E32DE43319F4812E839413C04B
:10BFE000812E8A9473940FC01250812F8F5FF0FEC0
:10BFF00005C0662D47E00E94CE5E05C069810E94A3
:10C000007E5E01C0812EFAE0AF16B104C104D104F6
:10C010000CF000E0C601B5012AE030E040E050E05D
:10C020000E94887259016A012115310541055105A7
:10C0300081F4002331F0023059F4252D223040F4F0
:10C0400008C0F4FE10C0222021F430EFF30E01C02E
:10C0500000E019195394852D90E0EA81FB81E817DF
:10C06000F9070CF088CF882061F0662D645F882D79
:10C07000472D0E94CA5E662D635F882D472D0E9462
:10C08000CA5E442039F0812F8919662D4DE22F2D8B
:10C090000E942A5D0F900F900F90CF91DF911F911A
:10C0A0000F91FF90EF90DF90CF90BF90AF909F9057
:10C0B0008F907F906F905F904F903F902F9008955A
:10C0C000EF920F93022FFA019F01442737FD40950D
:10C0D000542F75E0E72E0E942A5F0F91EF9008958C
:10C0E00020E00E9460600895A998AB98AC988BBB43
:10C0F000AD9AAD98AB9AA99A089520E030E006C0B9
:10C1000045E04A95F1F700002F5F3F4F28173907A8
:10C11000BCF30895AA9885E08A95F1F7000085E0C0
:10C120008A95F1F70000AA9A8CED95E00E947D6057
:10C1300082EE0E9474608EEA0E94746081EA0E941E
:10C14000746086EA0E94746084EA0E94746082EAE5
:10C150000E94746080EC0E9474608FE20E947460A0
:10C1600085E20E94746081E80E94746082E20E940D
:10C1700074608FEA0E94746082E280937201089575
:10C180001F93182F81E80E947460812F0E947460B1
:10C190001F9108951F93CF93DF9310E0C9EAD9E070
:10C1A00084E00E94746080E10E947460812F806B43
:10C1B0000E947460A998AB9AAC98FE0180E29081CD
:10C1C0009BBBAD9AAD9891819BBBAD9AAD98928186
:10C1D0009BBBAD9AAD9893819BBB3496AD9AAD98BD
:10C1E000815069F7C058DF4FAB9AA99A1F5F18308A
:10C1F000B9F6DF91CF911F910895BF92CF92DF9250
:10C20000EF92FF920F931F93CF93DF93EA01E82EF3
:10C21000F92E062F172F21C0F701B1907F01680179
:10C220000894C11CD11C04C0009739F00E943C192D
:10C230008091E50890E082709070E199F5CF1FBB86
:10C240000EBBE09A8DB3B81631F0BDBA8FB7F89433
:10C25000E29AE19A8FBF219786012097E9F6DF9154
:10C26000CF911F910F91FF90EF90DF90CF90BF90F3
:10C2700008958093DA0D08958091DA0D1092DA0D09
:10C280000895FC018081982F990F9E70807F892BE3
:10C290008083662321F09160807F892B8083818158
:10C2A0008F5F81839281992391F020812F7079F49F
:10C2B000933659F0242F20622093DA0D903111F437
:10C2C000803118F080818F7C80831182128282817C
:10C2D000883009F443C0893058F4813009F446C0ED
:10C2E0008130A0F08230D1F1843009F052C036C0E4
:10C2F0008F3549F1803620F4803109F04AC02EC0D4
:10C30000813689F0823609F044C03DC08081982F83
:10C310009F709F30F1F591E6928391819131E0F029
:10C320008F7C808319C040664093DA0D9081892FFD
:10C3300082958F708F5F83708295807F9F7C982B12
:10C3400090838FE508C08181883111F4406818C05E
:10C350008832F9F480E182831182089591819033CB
:10C3600028F090E09595879582831182828190E0F4
:10C370000197218130E082239323009751F4406498
:10C380004093DA0D08958181803418F088E082832B
:10C39000118208958E3091056CF4FC01EE0FFF1FA1
:10C3A000E80FF91FE355F24F90819F7081E09F30B5
:10C3B000E9F53FC0823131F1833160F48F30C9F04B
:10C3C000803118F48E3091F52AC0803161F08131CE
:10C3D00069F513C0843151F08431D0F08531E1F03A
:10C3E000863121F51EC091B194701DC093B3907831
:10C3F0001AC090916300917016C09091630090955F
:10C40000987011C08091630083FF12C091B102C087
:10C4100091B19095907407C091B1907104C093B39D
:10C42000F9CF91B1907281E0992319F480E00895D9
:10C4300080E008958F708E3058F490E0FC01EE0F8C
:10C44000FF1FE80FF91FE355F24F82E68283118246
:10C4500008958F708E3068F490E0FC01EE0FFF1F9E
:10C46000E80FF91FE355F24F83E6828380818F7CCA
:10C47000808308950F931F93CF93DF938091D70DFF
:10C480009091D80D01969093D80D8093D70D8091FF
:10C49000D90D8F5F8093D90D06B3009540E050E031
:10C4A00010E001C0AE01EA012196CA01880F991F70
:10C4B000840F951FB8010C2E02C0759567950A94DC
:10C4C000E2F7617070708355924F50E00E944161B5
:10C4D000C630D10539F700B30095C0E0D0E0FE01C9
:10C4E000EC5DF54EE4919E012A5F3F4FC901880F34
:10C4F000991F820F931F8355924FE02361E009F447
:10C5000060E09E012A5F422F50E00E944161219627
:10C51000C830D10521F7DF91CF911F910F91089578
:10C52000FF920F931F93CF93DF93F82EEEEBF1E082
:10C5300080E090E0582F9C014081F41638F04423AD
:10C5400029F001963A9681329105A1F75032B9F15E
:10C55000E901CC0FDD1FC901A3E0880F991FAA953F
:10C56000E1F7C80FD91F8E0102541E4FA9014F5F7A
:10C570005F4FCA01880F991FE3E0440F551FEA95EA
:10C58000E1F7840F951F20953095205E3F4FA9015C
:10C59000440F551F63E0220F331F6A95E1F7420FE6
:10C5A000531F82549E4FB8010E94B8728AE0D8018E
:10C5B0001D928A95E9F7CC55DE4FFA8E02C00EEB3C
:10C5C00011E0C801DF91CF911F910F91FF90089565
:10C5D00080E491E0EEEBF1E0DF019C011D9221503F
:10C5E0003040E1F70895EAE8F3E088E2DF011D92C8
:10C5F0008A95E9F7B89688E4DF011D928A95E9F7F4
:10C600000895282F30E08830C0F4462F572FDA01E4
:10C61000F901EE0FFF1FEE0FFF1FE20FF31FE657AA
:10C62000FC4F95E0899FC001112481579C4F2D91AB
:10C630002193E817F907D9F70895462F572FDA0104
:10C6400028503040F90193E0EE0FFF1F9A95E1F773
:10C65000E20FF31FEE54FC4F99E0899FC0011124B3
:10C660008D589C4F2D912193E817F907D9F708951C
:10C6700090E00197FC01EE0FFF1FE80FF91FEC554A
:10C68000FE4FDF01A85ABD4F6C93DF01AA5ABD4F80
:10C690004C93E95AFD4F20830895E0918801F0E022
:10C6A000EE0FFF1FEE0FFF1FE80FF11DE15EFA4FC7
:10C6B000849108958F929F92AF92BF92CF92DF9212
:10C6C000EF92FF920F931F93DF93CF93CDB7DEB717
:10C6D0006D970FB6F894DEBF0FBECDBFF82EDE010A
:10C6E0001596E6E2F1E085E001900D928150E1F7C8
:10C6F000DE011A96E1E2F1E085E001900D928150B1
:10C70000E1F7DE011F96ECE1F1E085E001900D928A
:10C710008150E1F7DE015496E7E1F1E085E0019018
:10C720000D928150E1F7DE015996E2E1F1E085E0FA
:10C7300001900D928150E1F719821A821B821C82AE
:10C74000E0918D01F0E0E85FFA4F26E030E011E083
:10C75000E491CE2EDD24BE016F5F7F4F0FC04F5F8F
:10C760005F4FA417B50711F4FC0110834430510545
:10C77000B1F71F5F22503040153081F040E050E0AB
:10C78000C601022E02C0959587950A94E2F7837040
:10C790009070DC011196860F971FE1CFFF2041F5C5
:10C7A0000E94E86289810E9490628C0181E00E946F
:10C7B0004D63F801818374E6F72EF2828A810E942C
:10C7C00090628C0182E00E944D63F8018183F282C5
:10C7D0008B810E9490628C0183E00E944D63F8017E
:10C7E0008183F2828C810E9490628C0184E07EC001
:10C7F000FF2DF13071F48B810E949062FC0188E082
:10C8000081838CE98283F3828781817F846087833F
:10C81000D7C18F2D8230E9F58B810E949062FC0197
:10C8200008E001836CE9F62EF28285E1838387813B
:10C83000817F846087838EE00E949062FC0182E2A7
:10C84000818314E612838EE00E949062FC010183D2
:10C85000F28284E183838781817F846087838EE095
:10C860000E949062FC010183128381E083838781AF
:10C87000817F8460878383E00E944D63482F8BE033
:10C8800062E02DE90E9438638CE061E042E220E042
:10C8900095C1EF2DE33081F50E94E862E9808E2D8D
:10C8A0000E9490628C0181E00E944D63F8018183B7
:10C8B00054E6F52EF2828E2D0E9490628C0182E069
:10C8C0000E944D63F80181838CE98283EA808E2D7A
:10C8D0000E9490628C0181E00E944D63F801818387
:10C8E000F2828E2D0E9490628C0182E00E944D6344
:10C8F000F8018183F28264C1FF2DF43081F50E943A
:10C90000E862EA808E2D0E9490628C0182E00E9493
:10C910004D63F801818344E6F42EF2828E2D0E944D
:10C9200090628C0184E00E944D63F8018183F28261
:10C93000EC808E2D0E9490628C0182E00E944D63FB
:10C94000F8018183F2828E2D0E9490628C0184E036
:10C950000E944D63F80181838CE9828331C1FF2DF0
:10C96000F53009F0D0C00E94E8620E94F36281E0D5
:10C970000E949062FC013AE0C32EC18224E6B22EEE
:10C98000B28282E00E949062FC019BE0D92ED182AB
:10C99000B28283E00E949062FC018CE0E82EE1828A
:10C9A000B28284E00E9490628C0181E00E944D631B
:10C9B000F8018183B28285E00E9490628C0183E05D
:10C9C0000E944D63F8018183B28204E0A02EA3820D
:10C9D00087E0848387818160878385E00E949062FD
:10C9E0008C0183E00E944D63F8018183B282F3825F
:10C9F00018E0812E848287818160878385E00E9490
:10CA000090628C0183E00E944D63F8018183B282C1
:10CA1000B6E0BB2EB382A9E09A2E94828781816012
:10CA2000878385E00E949062FC0181828CE9828389
:10CA300081E083838781817F8460878386E00E9491
:10CA40009062FC0191828EE1828388EF83838BE088
:10CA50000E9490628C0183E00E944D63F801818303
:10CA600076E4972E9282A382C48287818160878335
:10CA70008BE00E9490628C0183E00E944D63F8017C
:10CA800081839282F382D4828781816087838BE065
:10CA90000E9490628C0183E00E944D63F8018183C3
:10CAA0009282B382E4828781816087838091BA0118
:10CAB0008F7180628093BA018FE18093BB0180E027
:10CAC000BE016B5F7F4F0E94016381E0BE01665F24
:10CAD0007F4F0E94016382E0BE01615F7F4F0E9431
:10CAE000016383E0BE016C5E7F4F0E9401638E0193
:10CAF000075E1F4F84E0B8010E94016385E0B80122
:10CB00000E9401635DC0FF2DF630B1F486E00E9403
:10CB10009062FC01F18282E3828388EF838314E6D2
:10CB2000108786E00E949062FC01F1828EEC828385
:10CB300088E08383108744C08F2D873009F040C080
:10CB40008FE00E949062FC0184E2818384E682830C
:10CB500088E8868380E10E949062FC0189E08183FD
:10CB60000EE602838AE0838380E10E949062FC01EA
:10CB700018E0118382E982838BE083838781817F40
:10CB80008460878380E10E949062FC0111830283AC
:10CB90008CE083838781817F8460878381E06BE081
:10CBA00043E224E20E94386382E061E043E229E646
:10CBB0000E94386383E062E043E227E90E94386321
:10CBC00082E00E940E580E94AA586D960FB6F89403
:10CBD000DEBF0FBECDBFCF91DF911F910F91FF90B0
:10CBE000EF90DF90CF90BF90AF909F908F9008957F
:10CBF0006F927F928F929F92AF92BF92CF92DF926D
:10CC0000EF92FF920F931F93CF93DF938091BA011E
:10CC100081FF03C060E075E002C060E074E09091C5
:10CC2000B70184E69802C0011124885A9D4FE09113
:10CC3000BD01FF27E7FDF09548EE53E0E49F90012A
:10CC4000E59F300DF49F300D112428533045AA2460
:10CC5000BB24A81AB90A281B390BF5E2EF2EF5E020
:10CC6000FF2E4091B401440F485F50E0440F551F20
:10CC7000440F551F4552524FEBEDFDE0CC24DD240F
:10CC8000C61AD70AA8E5B2E0A81BB90B1CC0E70179
:10CC9000699079907E014B01661677060CF443018A
:10CCA00084018C149D040CF48601005A164FE50192
:10CCB000C01BD10B2C0F3D1F0A0F1B1F11830083BC
:10CCC000938382833496E417F50709F73183208331
:10CCD0009383828315821482DF91CF911F910F91EC
:10CCE000FF90EF90DF90CF90BF90AF909F908F908C
:10CCF0007F906F900895E0912B01F0912C0181932A
:10CD0000F0932C01E0932B010895FF920F931F9352
:10CD1000CF93DF93B9E0FB2E90E120E0C82FD0E065
:10CD20008E0101701070201711F4905F07C0892FD9
:10CD300090E001970E947B66202F90E1FA9431F0F9
:10CD4000D595C795AE014068842FE8CF892F90E034
:10CD50000F960E947B66DF91CF911F910F91FF90FC
:10CD600008951F93CF93DF93182F2BED3DE0309361
:10CD70002C0120932B0180913101877471F08091F7
:10CD8000B401882319F0813029F402C080E803C07F
:10CD900080E901C088E9809331018091310187FFEA
:10CDA0000BC086E190E00E94CA61882329F480913B
:10CDB00031018F77809331018091310187FD5AC015
:10CDC00085E160E040E00E94D510882309F452C05C
:10CDD00080913101806280933101809171018F5F78
:10CDE00080933201E3E3F1E0A5E2B5E080E01CC00E
:10CDF0002D913D913595279520503E4F37FD05C02B
:10CE000093E02F3F390724F405C020E030E002C052
:10CE10002FEF33E0932F9370482F440F440F942B40
:10CE2000908321838F5F3296811711F7C1E3D1E0A0
:10CE300089910E94856681E0CF33D807C9F7809138
:10CE40002B0190912C01019790932C0180932B0141
:10CE50008FEF90E00E947B6680E090E00E947B660E
:10CE60008BED9DE09093300180932F01DF91CF9166
:10CE70001F910895809131018F7DADCF1F920F9248
:10CE80000FB60F9211242F938F939F93EF93FF93DD
:10CE900088B391E0892788BBE0912F01F0913001A0
:10CEA0002191F0933001E0932F01822F90E097BD04
:10CEB00086BD293C08F0C09A80916B0E81608093FA
:10CEC0006B0EFF91EF919F918F912F910F900FBE5D
:10CED0000F901F9018951F920F920FB60F9211246A
:10CEE0002F933F938F939F93EF93FF9388B391E09A
:10CEF000892788BBE0912B01F0912C01208130E043
:10CF000020FD04C088B599B5809603C088B599B551
:10CF1000409699BD88BDC90195958795009791F474
:10CF2000CF01019690932C0180932B01818188235E
:10CF300051F480917800909179008053984F99BD79
:10CF400088BD01C0808380916B0E816080936B0EE1
:10CF5000FF91EF919F918F913F912F910F900FBE75
:10CF60000F901F901895EDE7F0E08081857E80831B
:10CF700017981F9AAAE8B0E01C9210928B0082E8E2
:10CF80008C938081806280830895EDE7F0E080815A
:10CF90008F7D8083179AAAE8B0E01C9210928B00D4
:10CFA0008AE08C9380818861808308951F920F921C
:10CFB0000FB60F9211248F939F93AF93BF93EF936C
:10CFC000FF938091770E882321F01F9A1092770E9D
:10CFD00004C01F9881E08093770EA0912D01B0913D
:10CFE0002E01FD018191919190938700809386009D
:10CFF000F0932E01E0932D0180916E0E90916F0EB3
:10D00000909385008093840012968D919C91139744
:10D01000009759F483E29EE090932E0180932D01B6
:10D020008091BA0181708093770E80916B0E816040
:10D0300080936B0EFF91EF91BF91AF919F918F9174
:10D040000F900FBE0F901F901895AF92BF92CF9286
:10D05000DF92EF92FF920F931F93CF93DF93809114
:10D06000BA0181FF03C040E055E002C040E054E057
:10D07000F090B401FF0C80E1F80E2091B70184E636
:10D08000280290011124285A3D4FE091BD01FF274D
:10D09000E7FDF09568EE73E0E69FC001E79F900D15
:10D0A000F69F900D112488539045CC24DD24C21A9C
:10D0B000D30A821B930B68EFE62EEF0CE3E2FEE04F
:10D0C00000271127041B150B68E572E0621B730B28
:10D0D00021C0AE2DB0E0AA0FBB1FAB5DBA4FAC9024
:10D0E0001196BC90D5014A175B070CF4DA01A01722
:10D0F000B1070CF4D801A05AB64FE601CA1BDB0BEE
:10D100008C0F9D1F31832083A60FB71FB383A2838B
:10D110003496E394EF14E8F231832083938382837F
:10D12000885E934090936F0E80936E0E15821482EA
:10D13000DF91CF911F910F91FF90EF90DF90CF90F3
:10D14000BF90AF9008951F920F920FB60F921124C7
:10D150002F933F934F935F936F937F938F939F93FF
:10D16000AF93BF93EF93FF9378940E942568FF914C
:10D17000EF91BF91AF919F918F917F916F915F914F
:10D180004F913F912F910F900FBE0F901F901895C8
:10D190002091740E3091750E90E082279327907045
:10D1A000880F991F8057954EFC0145915491232F6C
:10D1B0003327422753275093750E4093740E0895DA
:10D1C0009091700E96959695982B9093700E8091F5
:10D1D000710E8F5F8093710E843068F0E091720E53
:10D1E000F091730E9193F093730EE093720E109280
:10D1F000700E1092710E089503C080E00E94E068E6
:10D200008091710E8823C9F7E091720EF091730E30
:10D2100010820895882339F08091760E8F5F809375
:10D22000760E80E803C01092760E80EC0E94E068D3
:10D230008091760E8530B8F708950F931F93182FBD
:10D240000E94C86808E0812F81700E940A691695C3
:10D250000150C9F71F910F91089580EC0E94E0687A
:10D2600080E80E94E06880E80E94E06880E80E9410
:10D27000E06880E80E94E06880E80E94E06880E85A
:10D280000E94E06880EC0E94E0680895AF92BF922F
:10D29000CF92DF92EF92FF920F931F93CF93DF9382
:10D2A0008BED9DE090932C0180932B019093730E56
:10D2B0008093720E1092750E1092740E1092700E72
:10D2C0001092710E1092760E0E942D698091B40119
:10D2D0000E941D6980916D0E0E941D6980E00E9470
:10D2E0001D6910926D0E05E215E054E0C52ED12C9B
:10D2F000F80120813181C901880F991F820F931F86
:10D30000B6010E945372EB0122813381C901880F5B
:10D31000991F820F931FB6010E94537260507C4F79
:10D32000C050DC4FF8E0C030DF0710F0CFEFD7E09F
:10D330007B0128E06030720720F0AFEFEA2EA7E013
:10D34000FA2E8C2F0E941D695E019B2D9F708E2DE1
:10D350008295807F892B0E941D69C701F4E0969514
:10D360008795FA95E1F70E941D690C5F1F4F25E034
:10D370000533120709F0BCCF0091750E8091740E31
:10D380000E941D69802F0E941D690E942D690E94C4
:10D39000FC688091780090917900805C934690932E
:10D3A000790080937800C09ADF91CF911F910F91FF
:10D3B000FF90EF90DF90CF90BF90AF900895809155
:10D3C000B30190916C0E981709F494C080936C0E81
:10D3D0008130F9F0813030F08230F1F1833009F0A2
:10D3E00089C05EC00E94B3671EBC80E49CE99BBDFF
:10D3F0008ABD1DBC1CBC87B7837C87BF8CE386BFFE
:10D400008FE380937C0087B7806187BF1FBC8AE071
:10D4100021C00E94B3671EBC1DBC1CBC80E797E105
:10D4200099BD88BD80EA9FE0909379008093780051
:10D4300087B7837C87BF8CE386BF8FE380937C00B4
:10D4400087B7886087BF80917D00816080937D0071
:10D450001FBC82E08EBD4EC00E94B3671EBC88EC2C
:10D4600090E090937900809378008CE291E09DBDEC
:10D470008CBD80EE9BEA97BD86BD87B7837C87BF56
:10D480008CE386BF8FE380937C0087B7806287BF81
:10D4900080917D00816080937D001FBC8AE1DACF9E
:10D4A0001EBC80E49CE99BBD8ABD1DBC1CBC87B72B
:10D4B000837C87BF80917D008E7F80937D008CE38D
:10D4C00086BF8FE380937C0087B7806187BF1FBCD6
:10D4D0008AE08EBD0E94256880E593EC90938700DA
:10D4E0008093860088E893E1909385008093840080
:10D4F0000E94C5678091B301813051F0813028F0DE
:10D50000823051F0833079F40CC00E94F8650895A0
:10D5100078940E9446690895789486E00E94B166E6
:10D5200008950E94F86508951F920F920FB60F920A
:10D5300011242F933F934F935F936F937F938F9318
:10D540009F93AF93BF93EF93FF938091B30182308A
:10D55000C1F480E492EA97BD86BD809178009091F5
:10D5600079008F3F910538F488E598E99093790028
:10D570008093780008C088EC90E0909379008093C5
:10D5800078000E94DF69FF91EF91BF91AF919F9169
:10D590008F917F916F915F914F913F912F910F905C
:10D5A0000FBE0F901F9018951F920F920FB60F92FB
:10D5B00011242F933F934F935F936F937F938F9398
:10D5C0009F93AF93BF93EF93FF938CB59DB520913D
:10D5D000780E222321F0C09A1092780E04C0C098D1
:10D5E00021E02093780EA0913F01B0914001FD0110
:10D5F000219131913BBD2ABDF0934001E0933F0161
:10D600002091C5063091C6062817390720F490935B
:10D61000C6068093C50620910C0130910D0182173A
:10D62000930720F490930D0180930C0112968D9135
:10D630009C9113970097D9F48BED9DE09093400156
:10D6400080933F018091BA01809581708093780E1C
:10D6500087B78F7E87BF0E94DF698091B3018823DF
:10D6600011F0833021F487B7806187BF789480916F
:10D670006B0E816080936B0EFF91EF91BF91AF9124
:10D680009F918F917F916F915F914F913F912F91DA
:10D690000F900FBE0F901F9018959091870198736F
:10D6A000903121F463E00E9433720895983111F4AF
:10D6B00086950895983211F4880F0895903319F4DF
:10D6C000982F990F890F0895FC01A5E6B0E08C9181
:10D6D0008B7F8C93148215821082118216A617A656
:10D6E00008950E94646B089521E0FC0184818823E1
:10D6F00009F420E0822F0895FC0181819081891B2B
:10D70000877098E0981B81E0933008F480E00895DA
:10D71000FC0184818823F9F0815084838281938184
:10D72000890F828386A5882309F44CC087A5982F8A
:10D73000915097A7882331F0809165008460809391
:10D7400065000895809165008B7F809365008091CE
:10D75000920187A708951B98809165008B7F809325
:10D7600065008581882319F0815085830895808123
:10D770009181891739F190E0DF01A80FB91F169642
:10D780002C911697228356962C91569724831E9699
:10D790002C911E9723835E962C915E972583D096BD
:10D7A0002C91D09726A717A696962C919697322F54
:10D7B000315096963C939697222321F401968770D8
:10D7C0009070808308958F929F92AF92BF92CF9274
:10D7D000EF92FF920F931F93DF93CF9300D0CDB7BB
:10D7E000DEB74C01122F4A8369830E947C6B4A8109
:10D7F0006981882331F180918701887311F1F401E7
:10D80000A180BB24C501019697E0F92EF822808102
:10D81000F816B9F0662329F080919101865F860F92
:10D8200001C080E0A80CB91CF5018683842F0E94FA
:10D830004D6BF501868B168FE0AA06A3C686F40110
:10D84000F1820F900F90CF91DF911F910F91FF9078
:10D85000EF90CF90BF90AF909F908F900895AF9230
:10D86000BF92CF92EF920F93DF93CF9300D00F929E
:10D87000CDB7DEB75C012B834A8369830E947C6B42
:10D880002B814A816981882329F1809187018873DE
:10D8900009F1662329F080919101865F860F01C00E
:10D8A00080E0F5018283842F2B834A8369830E9461
:10D8B0004D6BF50184832B812583E6A617A6C382D1
:10D8C000808181834A816981002321F00150C50153
:10D8D0000E94E36B0F900F900F90CF91DF910F910B
:10D8E000EF90CF90BF90AF900895CF92EF920F93AB
:10D8F000CF93DF93EC01809187018695869586957D
:10D90000877028819981291709F05CC1E62FF0E022
:10D91000E132F10508F056C1EA5BFF4FEE0FFF1F41
:10D920000590F491E02D0994CE0166E44AE0DEC052
:10D93000CE0166E444E1DAC0CE0166E44EE1D6C031
:10D94000CE0164E64AE022E002E0EE24E39452E0F5
:10D95000C52E36C1CE016FE545E022E00AE0EE2497
:10D96000E394CC240E94E36BCE016FE545E02AE00E
:10D9700001E00E94E36BCE016FE545E022E00AE0A2
:10D980001FC1CE0160E54AE023E002E0EE24CC2492
:10D99000CA940E94E36BCE016CE34AE023E0CC24FE
:10D9A000C3940E94E36BCE0166E44AE021E000E00C
:10D9B00032E0E32E96C0CE0166E445E021E001E0CE
:10D9C000EE24E394CC240E94E36BCE0162E34FE0AB
:10D9D00022E00E94E36BCE0160E54FE022E0F0C060
:10D9E000CE016EE645E021E002E0EE24E394CC2493
:10D9F0000E94E36BCE016CE745E021E02AC0CE0136
:10DA000062E345E025E000E0EE24CC240E94E36BD5
:10DA1000CE016AE545E025E00E94E36BCE016EE6AB
:10DA200043E024E002E0CCC0CE0160E545E02AE01E
:10DA300003E0EE24E394CC240E94E36BCE0160E586
:10DA400045E024E101E00E94E36BCE0160E545E0A2
:10DA50002AE003E0B5C0CE016AE044E125E002E03F
:10DA6000EE24E394CC24C394ABC0CE0162E344E043
:10DA70002AE002E0EE24E394CC240E94E36BCE0182
:10DA800066E448E024E101E00E94E36BCE0162E33A
:10DA900048E02AE002E00E94E36BCE0166E444E045
:10DAA00024E101E08DC0CE0168E745E02AE00AE00C
:10DAB00016C0CE0168E745E022E30AC0CE0160E06F
:10DAC00044E12AE001E00BC0CE0160E044E12AE03D
:10DAD00002E005C0CE0160E044E12AE003E0EE246C
:10DAE000E394CC246DC0CE0166E448E221E000E07E
:10DAF00048C0813009F466C0CE016BE405C08130B6
:10DB000009F460C0CE0161E44AE021E000E041C0D8
:10DB1000CE01642F46E0F9CFCE0166E44AE022E070
:10DB2000E6CF813009F44EC0CE0166E44AE022E03F
:10DB3000EDCFCE0168E7E8CFCE0168E74AE021E00B
:10DB40001FC0CE016AE74AE021E00FC0CE016CE7BA
:10DB50004AE021E004C0CE0168E74FE023E003E0A3
:10DB600010C0CE0168E74FE023E002E00AC0CE011A
:10DB700068E74FE023E004C0CE0166E444E129E118
:10DB800001E0EE24E39406C0CE0166E44AE022E020
:10DB900002E0EE24CC240E942F6C14C0CE016CE372
:10DBA00044E123E002E0EE24CC24C3940E94E36B22
:10DBB000CE0160E544E123E0EE24E394CC24CA9452
:10DBC0000E94E36BDF91CF910F91EF90CF9008957A
:10DBD000682F89E494E046E40E94756C08951F92D2
:10DBE0000F920FB60F9211241F932F933F934F93D1
:10DBF0005F936F937F938F939F93AF93BF93CF93D5
:10DC0000DF93EF93FF934CB18BB18C7161F0109265
:10DC10007E0E10927D0E1092800E10927F0E81E08B
:10DC200080937A0E40E08AB180917A0E90E001975D
:10DC30008831910508F018C189599F4FFC01EE0FFA
:10DC4000FF1F0590F491E02D09944B3291F04C3276
:10DC500040F4433281F0453281F0413209F004C191
:10DC600006C0403571F0483509F0FEC008C083E0B9
:10DC7000BEC086E0BCC089E0BAC08CE0B8C08FE00E
:10DC8000B6C082E1B4C0413209F0B0C084E0AFC098
:10DC9000413209F0ABC084E180937A0E40937C0E50
:10DCA00081E080937B0E80E006C0E82FF0E0EF5724
:10DCB000F14F10828F5F8230C0F384C04B3209F085
:10DCC00095C087E094C04B3209F090C084E1809306
:10DCD0007A0E40937C0E81E080937B0E80E006C03C
:10DCE000E82FF0E0EF57F14F10828F5F8230C0F3E2
:10DCF00069C0433209F07AC08AE079C0433209F042
:10DD000075C088E180937A0E40937C0E81E0809309
:10DD10007B0E80E006C0E82FF0E0EF57F14F108255
:10DD20008F5F8230C0F34EC0453209F05FC08DE096
:10DD30005EC0453209F05AC088E180937A0E409364
:10DD40007C0E81E080937B0E80E006C0E82FF0E03F
:10DD5000EF57F14F10828F5F8230C0F333C04835E8
:10DD600009F044C080E143C0483509F03FC088E174
:10DD700080937A0E40937C0E81E080937B0E80E04E
:10DD800006C0E82FF0E0EF57F14F10828F5F82302E
:10DD9000C0F318C0403551F583E129C0403531F555
:10DDA00088E180937A0E40937C0E81E080937B0E15
:10DDB00080E006C0E82FF0E0EF57F14F10828F5F50
:10DDC0008230C0F38093790E4FC085E110C086E1A8
:10DDD0000EC087E10CC04A3349F488E108C04A32DA
:10DDE00029F070917B0E4C3261F404C081E0809385
:10DDF0007A0E3AC084E180937A0E7F5F70937B0E37
:10DE000033C010917C0E50E02BE030E029C0852F0C
:10DE100090E0FC01E158F14F6081161701F5FC011B
:10DE2000E358F14F60817617D1F4EC01CF57D14F11
:10DE300068816A30A0F4829FF001839FF00D929F69
:10DE4000F00D1124DF01A60FB11DAD57B14F4C935A
:10DE50006F5F6883E60FF11DED57F14F10825F5F32
:10DE60005230A8F25093790EFF91EF91DF91CF914C
:10DE7000BF91AF919F918F917F916F915F914F91E2
:10DE80003F912F911F910F900FBE0F901F901895EB
:10DE9000109818981092900089E189B959981AB889
:10DEA00086E08093950001C08CB15F99FDCF089505
:10DEB00053980895539A089554985798089540E0B8
:10DEC0002BE030E019C0842F90E0FC01EF57F14FB8
:10DED0001082829FF001839FF00D929FF00D11241C
:10DEE000ED57F14F1082FC01E158F14F1082835839
:10DEF000914FFC0110824F5F423028F34093790E1E
:10DF000081E080937A0E549A579A08951F93182FA0
:10DF100080E060E040E95CE121E00E941D5E86E671
:10DF200060E0412F21E00E942A5D1F91089590E05A
:10DF3000FC01E158F14F2081261731F4FC01E35830
:10DF4000F14F20812417D9F02BE030E0829FF001BF
:10DF5000839FF00D929FF00D1124ED57F14F108229
:10DF6000FC01EF57F14F1082FC01E158F14F608343
:10DF70008358914FFC01408381E080937A0E08958D
:10DF8000823641F0833619F0813669F406C089E0A3
:10DF900090E707C08FEB91E704C00E945C6F82E8B6
:10DFA0009FE30E94661580E063E241E00E94976F64
:10DFB00081E065E241E00E94976F88E30E94866FEE
:10DFC00086E068E044EB5CE10E944C5E8091830E49
:10DFD000882319F043E85EE002C041E451E08CE0A0
:10DFE00060E124E10E941D5E86E060E246EA5CE1B9
:10DFF0000E944C5E80918E0E882319F04EE85EE000
:10E0000002C041E451E08CE068E224E10E941D5E20
:10E010000895823641F0833619F0813669F406C0DE
:10E0200082E590E707C080EC9FE604C00E945C6F29
:10E0300082E89FE30E94661580E06BE243E00E9465
:10E04000976F81E06BE244E00E94976F87E30E9444
:10E05000866F86E068E041ED5CE10E944C5E809155
:10E06000830E882319F043E85EE002C041E451E0EA
:10E070008CE060E124E10E941D5E86E060E244ECF9
:10E080005CE10E944C5E80918E0E882319F04EE870
:10E090005EE002C041E451E08CE068E224E10E94CD
:10E0A0001D5E0895823641F0833619F0813669F499
:10E0B00006C08BE990E707C089E090E704C00E94A2
:10E0C0005C6F82E89FE30E94661580E06BE241E0AE
:10E0D0000E94976F81E06BE242E00E94976F86E3B7
:10E0E0000E94866F86E068E04AEE5CE10E944C5E2A
:10E0F0008091830E882319F043E85EE002C041E47A
:10E1000051E08CE060E124E10E941D5E86E060E267
:10E110004DED5CE10E944C5E80918E0E882319F0DB
:10E120004EE85EE002C041E451E08CE068E224E1A8
:10E130000E941D5E0895823641F0833619F08136C3
:10E1400069F406C084EE90E707C082E590E704C05A
:10E150000E945C6F82E89FE30E94661580E061E2A6
:10E1600049E00E94976F81E061E24AE00E94976F68
:10E1700085E30E94866F86E068E041E05DE10E94F1
:10E180004C5E8091830E882319F043E85EE002C064
:10E1900041E451E08CE060E124E10E941D5E86E0F4
:10E1A00060E246EF5CE10E944C5E80918E0E882317
:10E1B00019F04EE85EE002C041E451E08CE068E214
:10E1C00024E10E941D5E0895823641F0833619F0E5
:10E1D000813669F406C08DE291E707C08BE990E7CC
:10E1E00004C00E945C6F82E89FE30E94661580E095
:10E1F00061E247E00E94976F81E061E248E00E949F
:10E20000976F84E30E94866F86E068E048E15DE1F5
:10E210000E944C5E8091830E882319F043E85EE0F3
:10E2200002C041E451E08CE060E124E10E941D5E07
:10E2300086E060E24FE05DE10E944C5E80918E0ED0
:10E24000882319F04EE85EE002C041E451E08CE022
:10E2500068E224E10E941D5E0895823641F0833613
:10E2600019F0813669F406C086E791E707C084EEAD
:10E2700090E704C00E945C6F82E89FE30E946615ED
:10E2800080E061E245E00E94976F81E061E246E054
:10E290000E94976F83E30E94866F86E068E04FE2FA
:10E2A0005DE10E944C5E8091830E882319F043E863
:10E2B0005EE002C041E451E08CE060E124E10E94B4
:10E2C0001D5E86E060E240E25DE10E944C5E80916E
:10E2D0008E0E882319F04EE85EE002C041E451E062
:10E2E0008CE068E224E10E941D5E0895823641F0D0
:10E2F000833619F0813669F406C08FEB91E707C0C9
:10E300008DE291E704C00E945C6F82E89FE30E9467
:10E31000661580E061E243E00E94976F81E061E270
:10E3200044E00E94976F82E30E94866F86E068E077
:10E3300045E45DE10E944C5E8091830E882319F0D4
:10E3400043E85EE002C041E451E08CE060E124E19A
:10E350000E941D5E86E060E249E35DE10E944C5E42
:10E3600080918E0E882319F04EE85EE002C041E4F1
:10E3700051E08CE068E224E10E941D5E089582363F
:10E3800061F0833628F4803659F08136A1F40DC04F
:10E39000833689F480EC9FE60CC086E791E709C0DC
:10E3A0000E945C6F8EE79AE104C00E945C6F82E875
:10E3B0009FE30E94661580E061E241E00E94976F52
:10E3C00081E061E242E00E94976F81E30E94866FE4
:10E3D0008EE168E04EE55DE10E944C5E8091830E27
:10E3E000882319F043E85EE002C041E451E08CE08C
:10E3F00060E124E10E941D5E8EE160E243E55DE1A3
:10E400000E944C5E80918E0E882319F04EE85EE0EB
:10E4100002C041E451E086E068E224E10E941D5E12
:10E4200008950E94BF710895629FD001739FF0010B
:10E43000829FE00DF11D649FE00DF11D929FF00D94
:10E44000839FF00D749FF00D659FF00D9927729FCB
:10E45000B00DE11DF91F639FB00DE11DF91FBD0156
:10E46000CF0111240895991B79E004C0991F9617D4
:10E4700008F0961B881F7A95C9F780950895AA1B06
:10E48000BB1B51E107C0AA1FBB1FA617B70710F09F
:10E49000A61BB70B881F991F5A95A9F780959095D1
:10E4A000BC01CD01089597FB092E07260AD077FD00
:10E4B00004D0E5DF06D000201AF4709561957F4FF7
:10E4C0000895F6F7909581959F4F0895A1E21A2E31
:10E4D000AA1BBB1BFD010DC0AA1FBB1FEE1FFF1F08
:10E4E000A217B307E407F50720F0A21BB30BE40B58
:10E4F000F50B661F771F881F991F1A9469F760959F
:10E500007095809590959B01AC01BD01CF01089558
:10E5100097FB092E05260ED057FD04D0D7DF0AD071
:10E52000001C38F450954095309521953F4F4F4F42
:10E530005F4F0895F6F790958095709561957F4FA0
:10E540008F4F9F4F0895EE0FFF1F0590F491E02D20
:10E550000994FB01DC014150504048F005900D92B8
:10E560000020C9F701C01D9241505040E0F70895C6
:10E570006817790768F4FB01DC01E40FF51FA40FAD
:10E58000B51F02C002900E9241505040D8F7089536
:10E590000C94E172DC0101C06D9341505040E0F7F2
:10E5A0000895DC01CB01FC01E199FECF06C0FFBB61
:10E5B000EEBBE09A31960DB20D9241505040B8F743
:10E5C0000895FB01DC0102C001900D9241505040C2
:08E5D000D8F70895F894FFCF7D
:10E5D80086038703880389034AF0004DFF07220456
:10E5E8007C5E9CCE003264E2F1003264645A505A78
:10E5F8006450463C46649CEC1E465ADB0D230EDBF9
:10E608000DFF0000AA05FF09FF0DFF135414AADB34
:04E618000D3F0000B2
:00000001FF
